:100000000C94850A0C94A60A0C94A60A0C94FD0F75
:100010000C9437100C94A60A0C94A60A0C94A60A09
:100020000C94A60A0C94A60A0C94A60A0C94A60A90
:100030000C94A60A0C94A60A0C94A60A0C945213CB
:100040000C94A60A0C94A60A0C94A60A0C94A60A70
:100050000C94A60A0C9495650C94A60A0C94A60A16
:100060000C94A60A0C9410660C94A60A0C94A60A8A
:100070000C94A60A0C94A60A0C94A60A0C94A60A40
:100080000C9496790C94A60A0C94A60A0C94A60AD1
:100090000C943F660C94A60A0C94A60A0C94A60A2B
:1000A0000C94A60A0C94A60A0C94A60A0C94A60A10
:1000B0000C94A60A0C94A60A0C94A60A0C94A60A00
:1000C0000C94A60A0C94A60A0C94A60A0C94A60AF0
:1000D0000C94A60A0C94A60A0C94A60A0C94A60AE0
:1000E0000C94A60A0C94D06C0C94DA6C0C94C66C2C
:1000F0000C94866C0C94066D0C94FC6C0C94F06C57
:100100000C94E46C0C94A60A0C94A60A0C94A60A0F
:100110000C94A60A0C94A60A0C94A60A0C94A60A9F
:100120000C94A60A0C94A60A0C94A60A0C94A60A8F
:100130000C94A60AC47FE37F5C804E816E818E8121
:1001400096814381084AD73B3BCE016E84BCBFFDFC
:10015000C12F3D6C74319ABD56833DDA3D00C77F97
:1001600011BED9E4BB4C3E916BAAAABE0000008030
:100170003F07634236B79BD8A71A39685618AEBAFC
:10018000AB558C1D3CB7CC5763BD6DEDFD753EF690
:10019000177231BF000000803F08000000BE9224AB
:1001A00049123EABAAAA2ABECDCCCC4C3E000000E0
:1001B00080BEABAAAAAA3E00000000BF00000080DB
:1001C0003F0000000000084178D3BB4387D1133DB6
:1001D000190E3CC3BD4282AD2B3E68EC8276BED97F
:1001E0008FE1A93E4C80EFFFBE01C4FF7F3F0000BE
:1001F000000000000C94845B0C94C47F0C94068671
:100200000C9402110C9446780C947F820C94F8663E
:100210000C94216D0C945E760C94B2680C94497821
:100220000C94A9890C948E810C9488740C941116EA
:100230000C948D740C94AA370C948B0E0C945C80E7
:100240000C9492740C94391D0C9468790C94598315
:100250000C94710E0C949F740C94A7860C94977454
:100260000C946D4C0C946E810C941E150C946D695D
:100270000C94E36A0C944B740C94286A0C94717976
:100280000C94E37F0C94A0660C94704D0C94168330
:100290000C9461730C94436E0C940D6C0C94D68783
:1002A0000C944E810C94CF820C9424670C9455735B
:1002B0000C94BB680C9496810C94AA820C94E86709
:1002C0000C9443810C94EF730C94F3670C949C741E
:1002D0000C94124D0C9441780C9418740C94906A00
:1002E0000C94E5780C9400796E616E00696E66007E
:1002F000256300496E76616C6964206932632073FE
:100300007065656420696E20454550524F4D2E2022
:1003100053657474696E67203130206B6269742F85
:10032000730025730A005854414C5F5452494D3DA7
:1003300025640025730A0025730A00546573742030
:10034000362025730A005465737420352025730AFE
:10035000005465737420342025730A005465737447
:1003600020332025730A00546573742032202573CE
:100370000A005465737420312025730A0063686194
:100380006E3D25640A0074787077723D25640A001A
:100390003530306B0A003235306B0A003131356B45
:1003A0000A0035366B0A0033386B0A0025730A00E1
:1003B000765F6C6F773D252D332E32660A002573EC
:1003C0000A0073656E743D252D75206475703D259A
:1003D0002D752069676E6F7265643D252D752074DB
:1003E000746C5F7A65726F3D252D750A0025372E76
:1003F00033662025372E33660025352E32662000E1
:100400004572726F72203020566F6C74004E6F749C
:1004100020737570706F727465640A004572726F34
:1004200072203020566F6C74004572726F722030EB
:1004300020566F6C740062756C6B5F64656C6179DB
:100440003D252D750062756C6B3D252D750056613F
:100450006C7565206E6F7420616C6C6F77656400DD
:1004600062756C6B3A206D61783D257520737461FF
:1004700072743D25752C20656E643D25752C2069B0
:100480006E5F7573653D25750A007062323D257398
:100490000A007062313D25730A00256C7500416CBD
:1004A0006C6F77656420737065656420312F31301F
:1004B0002F3130302F343030206B6269742F73004D
:1004C00025630074746C3D252D64200074746C3DAC
:1004D000252D6420004E65772074746C3D252D64B5
:1004E00020002563004D533536313120503D252DF8
:1004F000372E326620252D372E32666D0A00424D8A
:100500005030383520256C642050612020252D374F
:100510002E32666D00256300545F484541545F49A3
:1005200044583D252D352E32662000545F444557F2
:100530003D252D352E3266200041483D252D352E96
:1005400032662000545F53485432583D252D352ED5
:100550003266200052485F53485432583D252D35AD
:100560002E32662000545F52483D252D342E3166D0
:10057000200052483D252D342E3166200025630091
:100580002563002563002563002563007265706F95
:1005900072745F616C6C3D007265706F72743D00C7
:1005A000256300256300256300256300204F534326
:1005B00043414C3D2564200020467573653A206513
:1005C000653D253032782068663D25303278206CD4
:1005D000663D25303278206C623D25303278004D02
:1005E00043553D2530366C780025630074785F6C88
:1005F000656E3D252D6C752C765F6C6F773D252DD6
:100600006C752C73687432783D252D6C752C627571
:100610006C6B3D252D6C75002563004F4B0A002542
:1006200063002563002563002563002563002563BF
:100630000025630025630064656275675F616C6C0B
:100640003D0064656275673D0064656275673D00E5
:1006500025730A00646565700A006E6F6E650A0096
:10066000707772733D007062323D25730A007062CC
:10067000313D25730A00696E74725F7365635F7044
:10068000313D252D372E33660A00696E74725F7016
:10069000313D252D6C640A00696E74725F73656369
:1006A0005F70303D252D372E33660A00696E7472F7
:1006B0005F70303D252D6C640A00765F6D63753D7B
:1006C000252D352E32660A00745F6D63753D252D2C
:1006D000352E32660A00707077723D25730A006409
:1006E000656275673D0072636D643D25730A002580
:1006F000730A006175746F0A006C6F675F6D6F64D9
:10070000653D007573625F7077723D25730A0072F4
:10071000656C61793D25730A0074746C3D252D6408
:100720000A0052494D455F616464723D252D642E77
:10073000252D640A006E65696768626F725F746177
:10074000626C655F73697A653D25640A00765F6C4B
:100750006F773D252D332E32660A00747870773D11
:1007600025640A006368616E3D25640A0069643D82
:10077000006932635F6275733D006932635F737055
:100780006565643D252D6C750A007478743D25738C
:100790000A0053797374656D2053756D6D617279BC
:1007A0000A002530366C780041744D65676132353A
:1007B00036524652320041744D65676131323852CB
:1007C0004652320041744D656761363452465232AA
:1007D0000041744D65676131323852464131004DF8
:1007E00043553D006D61736B3D002C00696E74656F
:1007F0007276616C3D252D750023252D642C0070CB
:1008000062320070623100745F686561745F6964B0
:100810007800745F64657700616800705F6D7335A0
:100820003631310072685F736874327800745F73B8
:100830006874327800706100700061643400616433
:100840003300616432006164310061330061320061
:10085000613100765F696E007268006572720075C2
:100860007074696D650070315F6C73740070315F16
:10087000740070310070305F6C73740070305F749E
:1008800000703000765F6D637500745F6D63750096
:100890007431007400696400653634007478740043
:1008A0002D002B006175746F006E6F6E65006275B0
:1008B0006C6B00706F7765725F736176655F6C65F6
:1008C0006472790072656C61795F6C65647900634C
:1008D0006F6D7061737300616363656C0070726546
:1008E0007300705F707772006165730070315F6CC8
:1008F0006564790070305F6C656472006576656E62
:1009000074006C6564006F7700706B740074785FBE
:100910006C6564790072785F6C656472006F7065F5
:1009200072006E6F6E65002530327800765F61640C
:10093000343D252D382E3666002000765F61643305
:100940003D252D382E3666002000765F6164323DED
:10095000252D382E3666002000765F6164313D25F6
:100960002D382E3666002000765F6C696768743D0E
:10097000252D382E3666002000765F61323D252D0C
:10098000372E3366002000765F61313D252D372EEE
:100990003366002000765F696E3D252D352E326668
:1009A00000204E657665722D7573656420737461E1
:1009B000636B203E2025642062797465730A00759C
:1009C0007074696D653D252D642D646179732D25E5
:1009D0003032643A253032643A253032642D686F03
:1009E0007572730A0074657374205B6F66667C3180
:1009F0007C327C337C347C355D20202020202020FC
:100A0000202D2074657374206D6F6465730A0D006A
:100A10007478205B706B74207061796C6F61645DB9
:100A20002020202020202020202020202D20736521
:100A30006E6420726164696F20706B74206B6579DD
:100A4000626F6172640A0D00776474205B6F6E7C64
:100A50006F66667C746573745D20202020202020E2
:100A6000202020202D207761746368646F670A0D51
:100A700000765F6C6F77205B765F6C6F775D202010
:100A8000202020202020202020202020202D206C0D
:100A90006F77657374207265706F727420766F6CF7
:100AA000746167650A0D0075706772202020202030
:100AB0002020202020202020202020202020202036
:100AC0002020202D207265626F6F7420766961206E
:100AD000626F6F746C6F616465720A0D007561728C
:100AE00074205B33386B7C35366B7C3131356B7CF5
:100AF0003235306B7C3530306B5D202D2073657462
:100B0000207465726D2F75617274207370656564F1
:100B10000A0D00626F6F74202020202020202020EA
:100B20002020202020202020202020202020202DB8
:100B3000207265626F6F740A0D0070777273205BAC
:100B4000646565707C6E6F6E655D202020202020BE
:100B50002020202020202D206D637520736C65657A
:100B600070206D6F64650A0D007265737420656591
:100B700070726F6D20202020202020202020202037
:100B800020202020202D20726573746F72652065EF
:100B90006570726F6D0A0D0070707772205B6F6EFA
:100BA0007C6F66665D2020202020202020202020D1
:100BB000202020202D2070726F6772616D6D616240
:100BC0006C65207077720A0D0070623220205B6FB6
:100BD0006E7C6F66665D2020202020202020202053
:100BE00020202020202D2070726F6772616D6D6152
:100BF000626C652070696E2062320A0D007062318D
:100C000020205B6F6E7C6F66665D20202020202098
:100C10002020202020202020202D2062756C6B2099
:100C20004750494F2070696E0A0D00747874205B3C
:100C3000737472696E675D202020202020202020A0
:100C4000202020202020202D2053657420726570E4
:100C50006F7274207465787420737472696E670A99
:100C60000D0074787077205B31352D305D202020A9
:100C700020202020202020202020202020202D2067
:100C80005458205077722E20486967686573742025
:100C90003020283364426D290A0D0074746C205B87
:100CA000302D31355D2020202020202020202020C4
:100CB000202020202020202D2074696D652D746F48
:100CC0002D6C69766520666F72207061636B657448
:100CD000730A0D0073732020202020202020202064
:100CE0002020202020202020202020202020202004
:100CF0002D2073797374656D2073756D6D617279D4
:100D00000A0D007273202020202020202020202087
:100D10002020202020202020202020202020202DC6
:100D200020726164696F2073746174730A0D0072BC
:100D300069205B236E5D205B696E745D202020203E
:100D400020202020202020202020202D20726570AF
:100D50006F727420696E74657276616C0A0D007230
:100D6000636D64205B6F6E7C6F66665D2020202063
:100D700020202020202020202020202D20616C6C8D
:100D80006F7720636D642066726F6D206E65746F7F
:100D9000726B0A0D007265205B236E5D205B2B7CFD
:100DA0002D5D205B6D61736B7C6175746F2C6D6163
:100DB000736B5D202D206D6F7465207265706F728E
:100DC00074207365742F6D6F646966790A0D006F06
:100DD00077202020202020202020202020202020BC
:100DE00020202020202020202020202D206F6E6514
:100DF0002D776972652073656E736F72730A0D00CB
:100E00006C6F67205B6175746F7C6F6E7C6F66665C
:100E10005D20202020202020202020202D206D6FEC
:100E20007465732064617461206F6E205553420AAB
:100E30000D006E65205B666C7573685D2020202058
:100E400020202020202020202020202020202D2095
:100E50006E65696768626F72207461626C650A0D05
:100E600000657272202020202020202020202020B9
:100E7000202020202020202020202020202D206520
:100E800072726F722073746174730A0D006D6375F2
:100E90002020202020202020202020202020202052
:100EA0002020202020202020202D206D6375206907
:100EB0006E666F0A0D00693263205B70726F626547
:100EC0007C737065656420236E5D202020202020C7
:100ED00020202D206932632070726F626520627558
:100EE000737C736574206275732073706565640A22
:100EF0000D006964205B72657365745D202020209D
:100F000020202020202020202020202020202D20D4
:100F100069642068616E646C696E670A0D006875AB
:100F20006D20202020202020202020202020202074
:100F3000202020202020202020202D2068756D6971
:100F4000646974792073656E736F720A0D0072653F
:100F50006C6179205B6F6E7C6F66667C7374617404
:100F6000735D20202020202020202D2072656C61C0
:100F700079206E6574776F726B207265706F727412
:100F8000730A0D006465205B6D61736B5D2020202A
:100F90002020202020202020202020202020202051
:100FA0002D2064656275670A0D006368616E205BC1
:100FB00031312D32365D202020202020202020209D
:100FC0002020202020202D206368616E2031312DCB
:100FD00032362028322E3430352D32343830204D00
:100FE000687A290A0D0063616C69205B5B765F6932
:100FF0006E7C61317C61325D20766F6C747C7265D1
:101000007365747C6E6F6E655D202D2063616C6905
:1010100062726174650A0D0062756C6B205B5B73B4
:10102000686F777C666C7573685D205B7365742090
:1010300074687273682064656C61795D5D20202D31
:101040002062756C6B696E67207061636B65747389
:10105000200A0D0061646320202020202020202011
:101060002020202020202020202020202020202080
:101070002D2073686F7720765F696E2C2061312C8C
:1010800020613220766F6C74616765730A0D00759C
:101090002020202020202020202020202020202050
:1010A00020202020202020202020202D207570743A
:1010B000696D650A0D007620202020202020202048
:1010C0002020202020202020202020202020202020
:1010D00020202D2076657273696F6E0A0D006820DE
:1010E0002020202020202020202020202020202000
:1010F000202020202020202020202D2068656C70BA
:101100000A0D00256300756E6B6E6F776E20636D40
:10111000640A00484D433538383300257300257381
:1011200000202573002025362E326620002530321F
:10113000780074656D705F65787465726E3D252DFD
:10114000362E326600202573002025362E3266208A
:101150004F6E2D426F6172640025303278007465E5
:101160006D705F626F6172643D252D362E326600B0
:101170000A0042756C6B2072656D3A20737461725F
:10118000743D25752C20656E643D25752C20696E97
:101190005F7573653D25750A0042756C6B2061644F
:1011A000643A2073746172743D25752C20656E64F9
:1011B0003D25752C20696E5F7573653D25750A00A8
:1011C00042756C6B207468726573683A2074696D3F
:1011D00065723D25750A00503A20256C64205061E7
:1011E0002020252D372E3266206D0A004932433AE1
:1011F00020004A54414720726573657474210A00C7
:101200005761746368646F67207265736574210A3F
:101210000042726F776E6F7574207265736574210A
:101220000A0045787465726E616C2072657365742E
:10123000210A00506F7765722D6F6E20726573659D
:1012400074212E0A004F6E6C696E650A00526F752C
:1012500074696E6720456E61626C65640A00525065
:101260004C20456E61626C65640A0025732025730D
:101270002C206368616E6E656C202575202C2063C0
:101280006865636B207261746520257520487A203B
:10129000747820706F7765722025750A000A2A2AF3
:1012A0002A2A2A2A2A426F6F74696E672025732AB8
:1012B0002A2A2A2A2A2A0A004A5441472072657398
:1012C0006574210A005761746368646F67207265F2
:1012D000736574210A0042726F776E6F75742072A5
:1012E00065736574210A0045787465726E616C20BF
:1012F0007265736574210A00506F7765722D6F6E89
:101300002072657365742E0A00726E6720697373AC
:101310007565732025640A00454550524F4D20697C
:101320007320636F72727570742C207265777269A6
:1013300074696E6720776974682064656661756C8E
:1013400074732E0A006C6F63616C686F7374004174
:10135000544D454741323536726672320002000004
:10136000FFFE000001452025642E256420636C6F7C
:10137000636B20256C752063707520256C75206C5F
:10138000706D20256C752069727120256C75206741
:101390006C656420256C7520796C656420256C75FE
:1013A00020726C656420256C7520747820256C751E
:1013B000206C697374656E20256C752073656E737F
:1013C0006F727320256C752073657269616C2025BE
:1013D0006C750A0000407A10F35A00A0724E18098A
:1013E0000010A5D4E80000E87648170000E40B548C
:1013F000020000CA9A3B000000E1F505000080965B
:101400009800000040420F000000A086010000008C
:10141000102700000000E803000000006400000046
:1014200000000A00000000000100000000002C760F
:10143000D888DC674F0823DFC1DFAE59E1B1B7962A
:10144000E5E3E453C63AE651997696E8E6C2842687
:10145000EB898C9B62ED407C6FFCEFBC9C9F40F263
:10146000BAA56FA5F490055A2AF75C936B6CF967DF
:101470006DC11BFCE0E40D47FEF520E6B500D0EDA4
:10148000902E0300943577050080841E080000200C
:101490004E0A000000C80C333333330F986E1283AA
:1014A0001141EF8D2114893BE65516CFFEE6DB187E
:1014B000D1844B381BF77C1D901DA4BBE424203243
:1014C00084725E228100C9F124ECA1E53D274E41E2
:1014D0004E494E495459494E46CDCCCC3D0AD723AE
:1014E0003C17B7D13877CC2B329595E6241FB14FF6
:1014F0000A000020410000C84200401C4620BCBE3B
:101500004CCA1B0E5AAEC59D740011241FBECFEFEE
:10151000D1E8DEBFCDBF00E00CBF1AE0A0E0B2E032
:10152000E0EBFDE201E00BBF02C007900D92A63494
:10153000B107D9F729E3A6E4BAE001C01D92AD3F97
:10154000B207E1F70E946F640C94D6960C940000E9
:101550002F923F924F925F926F927F928F929F92C3
:10156000AF92BF92CF92DF92EF92FF920F931F93B1
:10157000CF93DF93CDB7DEB763970FB6F894DEBF96
:101580000FBECDBF6C014B012A01FC0117821682F0
:10159000838181FF43C3AE014F5F5F4F3A01F60184
:1015A0009381F40193FD859193FF81914F018823ED
:1015B00009F430C3853239F493FD859193FF81910D
:1015C0004F01853239F4B60190E00E94A293520196
:1015D0002501E5CF10E0F12C20E02032A0F48B3281
:1015E00069F030F4803259F0833269F420612CC004
:1015F0008D3239F0803339F4216026C022602460B6
:1016000023C0286021C027FD27C030ED380F3A30B5
:1016100078F426FF06C0FAE01F9F300D1124132F27
:1016200013C04AE0F49E300D1124F32E20620CC04A
:101630008E3221F426FDEEC2206406C08C3611F4F1
:10164000206802C0883641F4F40193FD859193FF30
:1016500081914F018111C1CF9BEB980F933018F40A
:101660002061805E06C09BE9980F933008F071C13D
:101670002F7E26FF16E02F73322E853619F4206454
:10168000322E08C0863621F4F22FF0683F2E02C0B9
:101690001111115037FE07C01C3350F4EE24E394AF
:1016A000E10E27E00BC0183038F027E017E005C046
:1016B00027E04CE3E42E02C0212FE12C520144E04C
:1016C000A40EB11CF20160817181828193810E2D83
:1016D000A3010E9419922C01098100FF02C003FF9F
:1016E00007C031FC08C032FE09C030E2232E07C01B
:1016F0002DE2222E04C09BE2292E01C0212C802F36
:101700008C7019F0211068C2A8C237FE0FC0E40C1B
:1017100004FF04C08A81813309F4EA941E1474F52D
:10172000F8E0FE1578F588E0E82E2CC036FC2AC0DB
:10173000812F90E0841595059CF02CEF42162FEF39
:10174000520674F0432D4068342E0AC0E2E0F0E007
:10175000EC0FFD1FE10FF11D8081803319F4115052
:101760001111F4CF37FE0EC0EE24E394E10E812F69
:1017700090E0481659062CF4141904C0EE24E394A2
:1017800001C010E037FE06C01414150434F4C20181
:10179000019605C085E090E002C081E090E0211054
:1017A0000196112331F0212F30E02F5F3F4F820F40
:1017B000931F2F2D30E08217930714F4F81A01C0FD
:1017C000F12C832D897049F4FF2039F0B60180E2B5
:1017D00090E00E94A293FA94F7CF222029F0B6015C
:1017E000822D90E00E94A29333FC09C0FF2039F0C3
:1017F000B60180E390E00E94A293FA94F7CF37FEFF
:101800005AC0942D852D57FE02C090E080E0292E0D
:10181000382E20E030E0A2014E1951095D874C8737
:10182000A201421953095F874E87612F70E0442758
:101830005527461B570B598B488B5FEF25163506EE
:1018400049F4B6018EE290E02A8B3B8B0E94A29372
:101850003B892A89421453046CF04C855D854215FE
:10186000530544F4EE85FF85E20FF31FE60DF71DE7
:10187000818101C080E351E0251A31082F5F3F4F7D
:1018800048895989241635064CF0B60190E02A8B18
:101890003B8B0E94A2932A893B89CFCF2414350425
:1018A00039F49A81963318F4953311F404FF81E3E7
:1018B000B60190E04BC08A81813309F00F7EB601FA
:1018C00090E00E94A293111105C034FC18C085E677
:1018D00090E017C0B6018EE290E00E94A29382E0F1
:1018E000EE24E394E80EF301E80FF11D8081B601C8
:1018F00090E00E94A29311508E2D91F7E6CF85E4DF
:1019000090E0B6010E94A29357FC05C04114510417
:1019100039F404FF05C05194419451088DE201C08F
:101920008BE2B60190E00E94A29380E39AE0491610
:1019300051042CF08F5F5AE0451A5108F7CFB601D9
:1019400090E00E94A293B601C201C0960E94A293A9
:1019500057C1833631F0833779F0833509F058C0A9
:1019600021C05201E2E0AE0EB11CF20180818983F8
:1019700001E010E0230114C05201F2E0AF0EB11CEF
:10198000F2014080518026FF03C0612F70E002C049
:101990006FEF7FEFC2012A8B0E944E938C012A8940
:1019A0002F7715C05201F2E0AF0EB11CF20140805A
:1019B000518026FF03C0612F70E002C06FEF7FEF00
:1019C000C2012A8B0E9403938C012A892068322E3F
:1019D00023FD1AC08F2D90E008171907A8F4B6014F
:1019E00080E290E00E94A293FA94F4CFF20137FCD7
:1019F000859137FE81912F01B60190E00E94A2935C
:101A0000F110FA94015011090115110579F7F8C088
:101A1000843611F0893659F5520127FF09C0F4E0E8
:101A2000AF0EB11CF20160817181828193810AC085
:101A3000F2E0AF0EB11CF20160817181072E000C43
:101A4000880B990B2F76322E97FF09C090958095C1
:101A5000709561957F4F8F4F9F4F2068322E2AE0FF
:101A600030E0A3010E94B394E82EE6183FC0022F95
:101A7000853721F40F7E2AE030E01DC0097F8F36C4
:101A800091F018F4883559F0C5C0803719F08837BF
:101A900011F0C0C0006104FF09C0046007C024FF4A
:101AA00008C0066006C028E030E005C020E130E054
:101AB00002C020E132E0520107FF09C0F4E0AF0E9E
:101AC000B11CF201608171818281938108C0F2E0D2
:101AD000AF0EB11CF2016081718180E090E0A30142
:101AE0000E94B394E82EE6180F77302E36FE0BC016
:101AF000332D3E7FE11650F434FE0AC032FC08C09C
:101B0000332D3E7E05C00E2D332D03C00E2D01C09A
:101B1000012F34FF0CC0FE01EE0DF11D80818033DA
:101B200011F4397E08C032FF05C00E5F04C0832F58
:101B3000867809F00F5F33FD13C030FF06C01E2DFD
:101B40000F1518F41F0D101B0F2D0F1568F4B6019B
:101B500080E290E03B8B0E94A2930F5F3B89F5CF20
:101B60000F1510F4F01A01C0F12C34FF12C0B601A9
:101B700080E390E03B8B0E94A2933B8932FF17C029
:101B800031FD03C088E790E002C088E590E0B6012F
:101B90000CC0832F867859F031FF02C08BE201C060
:101BA00080E237FD8DE2B60190E00E94A293E1163B
:101BB00038F4B60180E390E00E94A2931150F7CF71
:101BC000EA94F301EE0DF11D8081B60190E00E94D0
:101BD000A293E110F5CF14C0F4E0FF1558F584E0AE
:101BE000F81A33FE1EC0211026C003FF2AC008EEDB
:101BF00012E0F32DF0713F2EF8018491811124C081
:101C0000FF2009F4E5CCB60180E290E00E94A293A7
:101C1000FA94F6CFF6018681978126C08FEF9FEF69
:101C200023C0B60180E290E00E94A293FA94F110E2
:101C3000F8CFD9CFF12CB601822D90E00E94A2936B
:101C4000D4CF0CEE12E0D5CF31108052B60190E027
:101C50000E94A2930F5F1F4FCFCF23E02F1510F4E8
:101C600083E0BECFF12CC1CF63960FB6F894DEBFF0
:101C70000FBECDBFDF91CF911F910F91FF90EF90DD
:101C8000DF90CF90BF90AF909F908F907F906F909C
:101C90005F904F903F902F9008958115910511F01E
:101CA0000197F1F7089580E696E09F938F930E9445
:101CB000EE938091660290916702A0916802B091C4
:101CC00069020F900F9093FF03C08AE596E002C06F
:101CD00084E596E09F938F930E94EE930F900F9070
:101CE0000895E091F81CEF73F0E0E75BF24E80831B
:101CF0008091F81C8F5F8093F81C809199358860E3
:101D0000809399354CE452E061E1CA010E948570EC
:101D100080E090E00895CF93DF93EC0180919F13D2
:101D20009091A013A091A113B091A21386FF1DC0A2
:101D30008E811F928F938D811F928F938C811F9222
:101D40008F938B811F928F938A811F928F9389EE3D
:101D500092E09F938F930E94DA938DB79EB70C9673
:101D60000FB6F8949EBF0FBE8DBFBE0181E99AE009
:101D70000E947E71BE0188E092E0DF91CF910C94C9
:101D80000F7252985A981DBAE9E6F0E0808180629D
:101D90008083EA9A53985B98EB9A8081806880836D
:101DA000E8E6F0E08081816080830895EEEAFDE15D
:101DB0001182128210820895CF92DF92EF92FF92E9
:101DC0000F931F93CF93DF93EC019B018091AE1D86
:101DD000843108F0BBC08091B01D64E10E94698825
:101DE0009093B01DC090CB30D090CC30E090CD30EF
:101DF000F090CE30092F10E08DE8989FD00111248B
:101E0000A255B24E1396CD92DD92ED92FC921697AA
:101E10004115510559F0FA018081FD01EA57FF4F44
:101E20008083FA018181A957BF4F8C932097A9F035
:101E300089819DE8909FF001919FF00D1124E2555A
:101E4000F24EDF01A657BF4F8C93E557FF4F8881B5
:101E50008F70808388818F70808321153105E1F137
:101E6000D90116964C9116975DE8509FC001519F7D
:101E7000900D11248255924EFC01E757FF4F40838D
:101E800015964C9115973197408334961B964D913A
:101E90005D916D917C911E97452F562F672F772767
:101EA000518340837C01BEE8EB0EF11CF9012385D0
:101EB000348545855685A4E6B0E00E940489672FE5
:101EC000782F892F992724E630E040E050E00E94E7
:101ED0009D88D7016D937C938DE8809FD001819F71
:101EE000B00D1124AB54B24EFE0132968FE7019033
:101EF0000D928A95E1F78091B01D8F5F8093B01DA0
:101F00009091AE1D9F5F9093AE1D40919F13509195
:101F1000A0136091A1137091A21360FF2DC01F92B6
:101F20009F931F928F938091AF1D1F928F9389E98A
:101F300091E19F938F930E94EE93EDB7FEB7389691
:101F40000FB6F894FEBF0FBEEDBF16C08091DB3018
:101F50009091DC30A091DD30B091DE300196A11D72
:101F6000B11D8093DB309093DC30A093DD30B093D3
:101F7000DE3080E090E002C081E090E0DF91CF9120
:101F80001F910F91FF90EF90DF90CF9008952091D7
:101F9000AE1D222361F18091AF1D8F5F21502093F0
:101FA000AE1D64E10E9469889093AF1D40919F131C
:101FB0005091A0136091A1137091A21360FF1AC0F9
:101FC0001F922F938091B01D1F928F931F929F930A
:101FD00082E791E19F938F930E94EE938DB79EB716
:101FE00008960FB6F8949EBF0FBE8DBF03C080E069
:101FF00090E0089581E090E008951F920F920FB64F
:102000000F9211248F939F93AF93BF938091680099
:1020100080FF24C08091743590917535A0917635FC
:10202000B09177350196A11DB11D809374359093C1
:102030007535A0937635B093773580919F13909145
:10204000A013A091A113B091A21387FF07C07498A9
:1020500082E090E09093920280939102BF91AF91C1
:102060009F918F910F900FBE0F901F9018951F9208
:102070000F920FB60F9211248F939F93AF93BF933C
:102080008091680080FF24C08091783590917935E7
:10209000A0917A35B0917B350196A11DB11D809339
:1020A000783590937935A0937A35B0937B358091CC
:1020B0009F139091A013A091A113B091A21390FF30
:1020C00007C0739882E090E090939202809391020F
:1020D000BF91AF919F918F910F900FBE0F901F9066
:1020E000189580937C0080917B00877F80937B0094
:1020F00080917C00806C80937C0085E080937A00E6
:1021000080917A00806880937A0080917B0087FFBD
:10211000FCCF80917B0085FFFCCF80917A008064AA
:1021200080937A0080917A0086FDFCCF109279002E
:102130001092780084E090E060E070E020917A00F6
:10214000206420937A0020917A0026FDFCCF209114
:10215000780030917900620F731F019779F7109220
:102160007C0080917A008F7780937A0076956795CE
:102170007695679580E090E00E94728C089580E0EB
:102180000E9471102091890230918A0240918B0245
:1021900050918C020E946C8E21EE3AE744E95EE396
:1021A0000E94DD8A08950F931F93CF93DF930FE171
:1021B00010E0CBE5DEE00093510182E991E00E945E
:1021C0004D0E8091510185FD0DC00031110521F0AA
:1021D0002CF0CB54D10903C0C4ECD9E0E2970150F4
:1021E0001109E9CFBE0180E090E00E94728C20E0EE
:1021F00030E04AE754E40E94C08BDF91CF911F91F9
:102200000F910895CF93DF93EC0188819981009716
:1022100099F08031924121F01982188283E011C037
:10222000623171F40E94D3106093C7307093C8304C
:102230008093C9309093CA3080E192E1998388837A
:1022400081E0DF91CF91089580917B008860809339
:102250007B0089EC80937C0085E080937A008091FC
:102260007A00806880937A0080917B0087FFFCCFA2
:1022700080917B0085FFFCCF80917A008064809301
:102280007A0080917A0086FDFCCF80917A0080648C
:1022900080937A0080917A0086FDFCCF609178006F
:1022A0007091790080917A008F7780937A0080E036
:1022B00090E00E94728C27ED33EA40E95FE30E94D0
:1022C0006C8E26E636E648E853E40E94DC8A0895E0
:1022D000CF92DF92EF92FF921F93CF93DF93CDB710
:1022E000DEB729970FB6F894DEBF0FBECDBF6C01E5
:1022F000109299138FEF898781E0E82E8DE1F82EF7
:1023000010E089858823E9F11830D9F1BE016F5FAB
:102310007F4FCE0109960E94465F99859F3F11F03D
:102320009E3F19F4909399132CC0CE010196C114CD
:10233000D10481F40E94605F80939635AEE8B5E3E6
:10234000FE01319688E08E0F91919D938E13FCCF04
:1023500081E018C00E94605FF7018087FE0131961E
:1023600020E030E08191D701A20FB31F8C932F5F43
:102370003F4F28303105B1F71F5FF9E0EF0EF11C38
:10238000C0CF812F29960FB6F894DEBF0FBECDBF08
:10239000DF91CF911F91FF90EF90DF90CF90089544
:1023A00080E791E19F938F930E94EE930F900F909F
:1023B00008952F923F924F925F926F927F928F92E9
:1023C0009F92AF92BF92CF92DF92EF92FF920F93C4
:1023D0001F93CF93DF93EC015B01009711F427E08B
:1023E00003C0019749F426E04AE250E06BE270E056
:1023F00089E290E00E94205ECE010E9468119E0159
:1024000026563C4E6901D9018C93CD2B69F0C1E071
:10241000DDE1E12CF12C85E2282E81E1382E91E2DC
:10242000892E91E1992E9EC08EE895E30E94F15F7E
:10243000BC01990F880B990B0E94748C6B017C0175
:10244000AB2869F020E030E048EC52E40E94C08BF9
:102450009F938F937F936F938EE591E1A4C0CEE815
:10246000D5E309E511E189911F928F931F930F9393
:102470000E94EE930F900F900F900F90B5E3C63926
:10248000DB0789F720E030E048EC52E4C701B601F1
:102490000E94C08B9F938F937F936F9389E491E108
:1024A0009F938F930E94EE930F900F900F900F9039
:1024B0000F900F9080919635811103C08CE893E0C6
:1024C00002C088E193E09F938F9385E491E19F930D
:1024D0008F930E94EE930F900F900F900F906DC00E
:1024E00000E010E0FE01E00FF11F80811F928F934A
:1024F000ADE2B1E1BF93AF930E94EE930F5F1F4F28
:102500000F900F900F900F900830110559F720E0B1
:1025100030E048EC52E4C301B2010E94C08B9F93AB
:102520008F937F936F933F922F920E94EE930F9021
:102530000F900F900F900F900F908885811151C0D0
:102540008CE893E09F938F939F928F920E94EE93DB
:102550000E94D011FFEFEF1AFF0A29960F900F90FB
:102560000F900F90D6018C9190E0E816F906E4F5F3
:10257000CE010E94F15FBC01990F880B990B0E945C
:10258000748C2B013C01A114B10409F4A9CF20E003
:1025900030E048EC52E40E94C08B9F938F937F936E
:1025A0006F9382E391E19F938F930E94EE930F903C
:1025B0000F900F900F900F900F90DF91CF911F9180
:1025C0000F91FF90EF90DF90CF90BF90AF909F90D2
:1025D0008F907F906F905F904F903F902F900C94D2
:1025E000D01188E193E0AECFDF91CF911F910F9191
:1025F000FF90EF90DF90CF90BF90AF909F908F9023
:102600007F906F905F904F903F902F900895CF9361
:10261000DF931F921F92CDB7DEB7EEE8F5E381811D
:10262000898387818A83CE0101960E94B3740F90BB
:102630000F90DF91CF910895CF93DF93EC0120911C
:102640008E3530918F354091903550919135609114
:102650009235709193358091943590919535AFEF87
:102660000E94D08AE1F427E04AE250E06BE270E099
:1026700089E290E00E94205E80E090E00E94681174
:10268000C656DC4E888349E050E06EE070E08EE88C
:1026900095E30E94B996DF91CF910C940713DF91D7
:1026A000CF9108951F920F920FB60F9211240BB67F
:1026B0000F92FF920F931F932F933F934F935F932C
:1026C0006F937F938F939F93AF93BF93CF93DF933A
:1026D000EF93FF9380919935826080939935809133
:1026E000660286FD2B9A8091660287FD2B9A809167
:1026F0009102909192021816190614F4749A739A22
:1027000080919F139091A013A091A113B091A21357
:1027100085FF02C074987398809106029091070219
:1027200001979093070280930602892B09F04CC110
:102730008091540A9091550A01969093550A80937E
:10274000540A8091CB309091CC30A091CD30B09193
:10275000CE300196A11DB11D8093CB309093CC302B
:10276000A093CD30B093CE3080E190E090930702FB
:10277000809306028091660280FD02C01D9B05C009
:1027800010929E1310929D1306C081E090E09093EA
:102790009E1380939D1380919F139091A013A091FD
:1027A000A113B091A21397FF08C080919D1390913F
:1027B0009E13892B49F0749A739808EA1CE1C0EEC5
:1027C000D0E3FF24F39421C0739A7498F6CF8091DC
:1027D000540A9091550A01960E947588892BE1F060
:1027E000F8016085718561157105A1F5F8016085B5
:1027F00071856115710509F03FC0065F1F4F259671
:10280000F0E3C43FDF0709F44CC0F801608571852F
:102810006115710529F3DBCF4281417020E030E082
:1028200050E060E070E080E090E0A0E00E94D08A9C
:10283000B9F2779880919F139091A013A091A11362
:10284000B091A21392FFCCCF749810929202109282
:102850009102C6CF8091540A9091550A01960E9428
:102860007588892B19F61C821B82AE0162E184E215
:1028700092E00E948570BACF8091540A9091550AD7
:102880000E947588892B09F0B8CFF8821A830983D2
:102890001C821B82AE0162E182E492E00E9485709C
:1028A000ACCF60916C0270916D0261157105A1F160
:1028B0008091540A9091550A0E947588892B61F580
:1028C0008091743590917535A0917635B0917735BA
:1028D0004091BD285091BE286091BF287091C028BA
:1028E000841B950BA60BB70B8093D01C9093D11C27
:1028F000A093D21CB093D31C809174359091753500
:10290000A0917635B09177358093BD289093BE28FD
:10291000A093BF28B093C02860916A0270916B02A7
:1029200061157105A1F18091540A9091550A0E9498
:102930007588892B61F58091783590917935A091D2
:102940007A35B0917B354091C1285091C228609171
:10295000C3287091C428841B950BA60BB70B8093DA
:10296000D41C9093D51CA093D61CB093D71C8091F7
:10297000783590917935A0917A35B0917B358093F7
:10298000C1289093C228A093C328B093C4288091F3
:10299000660286FD2B988091660290916702A09155
:1029A0006802B091690291FF0FC00E94AB698A3141
:1029B00019F0C1E0C80F01C0CBE00E94E8678C2F7E
:1029C0000E94C3690E94B26840E050E060E085EB7D
:1029D00092E00E948570FF91EF91DF91CF91BF91BE
:1029E000AF919F918F917F916F915F914F913F91A7
:1029F0002F911F910F91FF900F900BBE0F900FBE64
:102A00000F901F9018958091F81C9091DF30891BD2
:102A100008950E940315882371F0E091DF30EF7371
:102A2000F0E0E75BF24E808190E02091DF302F5F95
:102A30002093DF3008958FEF9FEF0895CF93DF93BA
:102A4000EC011092850A1092840A8881998100977E
:102A5000C1F0863E934021F01982188283E0BDC008
:102A6000613109F0B9C00E94091599279093800A35
:102A700080937F0A8D30910509F444C08F3F910502
:102A800049F40E9403158111EECF86EE93E09983FD
:102A90008883A2C08231910509F45AC08F3791050D
:102AA00009F052C080917D0A90917E0A181619068D
:102AB0000CF56091F7397091F83988E090E00E9448
:102AC000A2936091F7397091F83980E290E00E940A
:102AD000A2936091F7397091F83988E090E00E94F4
:102AE000A29380917D0A90917E0A019790937E0A2D
:102AF00080937D0A80917D0A90917E0A8F3791059F
:102B000009F0BFCF1092DF301092F81C80917D0A3F
:102B100090917E0AFC01EC50FF4C10829093850A44
:102B20008093840A10927E0A10927D0A80919735D4
:102B300090919835009709F4A4CF40E050E060915F
:102B400097130E9485709DCF8830910571F5AACFAB
:102B50006091F7397091F8398DE090E00E94A2936E
:102B600010927C0A10927B0A20917B0A30917C0A99
:102B700080917D0A90917E0A281739070CF0BACF10
:102B8000F901EC50FF4C80816091F7397091F83970
:102B900090E00E94A29380917B0A90917C0A01961A
:102BA00090937C0A80937B0ADFCF6091F739709114
:102BB000F8390E94A29320917D0A30917E0A80917B
:102BC0007F0AF901EC50FF4C80832F5F3F4F309319
:102BD0007E0A20937D0A8ECF81E0DF91CF91089508
:102BE00080919D1390919E13892BD1F08091660264
:102BF00090916702A0916802B091690293FD10C0A4
:102C00000E94E86783B7817F866083BFF89483B7AB
:102C1000816083BF7894889583B78E7F83BF7894D3
:102C20000895CF93DF93FC01208131812115310577
:102C300051F02334324129F0FC011182108283E0EB
:102C400015C0653891F4EC010E94E6660E94F0150B
:102C500040E050E065E88091E1149091E2140E9418
:102C6000857083E492E19983888381E0DF91CF913D
:102C70000895CF93DF931F921F92CDB7DEB7892BB4
:102C800081F05F934F938EE191E19F938F936983DE
:102C90007A830E94EE930F900F900F900F907A819D
:102CA00069817F936F938BE191E19F938F930E9452
:102CB000EE930F900F900F900F900F900F90DF9169
:102CC000CF910895EF92FF920F931F93CF93DF93CD
:102CD0000E94E66680EB0E947B6081111CC00E940E
:102CE000D8608091C52C9091C62C81609093C62CA1
:102CF0008093C52C81E293E09F938F938BE191E1C8
:102D00009F938F930E94EE930F900F900F900F90D0
:102D1000C1E0D0E002C0C0E0D0E01EB11470729AF1
:102D200064E278E680E090E00E9458600E94E666E7
:102D30008EE40E947B60811117C00E94D860809150
:102D4000C52C9091C62C82609093C62C8093C52C84
:102D50007E018FEFE81AF80A48E259E069E273E071
:102D6000CE010E943916E701111101C0729864E288
:102D700078E680E090E00E9458600E94E6668EEE61
:102D80000E947B60811116C00E94D8608091C52C82
:102D90009091C62C84609093C62C8093C52C8E0194
:102DA0000F5F1F4F48E259E061E373E0CE010E94DC
:102DB0003916E80164E278E680E090E00E9458600D
:102DC0000E94E66686EA0E947B60811116C00E941E
:102DD000D8608091C52C9091C62C88609093C62CA9
:102DE0008093C52C8E010F5F1F4F48E259E068E3C6
:102DF00073E0CE010E943916E80164E278E680E0D3
:102E000090E00E9458600E94E6668CE30E947B601E
:102E100081111EC00E94D8608091C52C9091C62C53
:102E200080619093C62C8093C52C8E010F5F1F4F3D
:102E300048E259E060E473E0CE010E94391683E174
:102E400091E19F938F930E94EE930F900F90E80172
:102E500064E278E680E090E00E9458600E94E666B6
:102E600082ED0E947B60811116C00E94D860809123
:102E7000C52C9091C62C80629093C62C8093C52C53
:102E80008E010F5F1F4F48E259E068E473E0CE0106
:102E90000E943916E80164E278E680E090E00E9442
:102EA00058600E94E66680E80E947B60811116C02F
:102EB0000E94D8608091C52C9091C62C916090930F
:102EC000C62C8093C52C8E010F5F1F4F48E259E03E
:102ED00061E573E0CE010E943916E80164E278E60C
:102EE00080E090E00E9458600E94E66680ED0E94BB
:102EF0007B60811116C00E94D8608091C52C909192
:102F0000C62C80689093C62C8093C52C8E010F5FD1
:102F10001F4F48E259E067E573E0CE010E94391681
:102F2000E80164E278E680E090E00E9458600E9448
:102F3000E6668CEE0E947B60811116C00E94D8600C
:102F40008091C52C9091C62C92609093C62C809352
:102F5000C52C8E010F5F1F4F48E259E06FE573E00B
:102F6000CE010E943916E80107E010E064E278E63D
:102F700080E090E00E9458600E94E6668CE70E9424
:102F80007B60811113C00E94D8608091C52C909104
:102F9000C62C80649093C62C8093C52C48E259E0DF
:102FA00066E673E0CE010E94391603C00150110994
:102FB000E9F60E94D860DF91CF911F910F91FF90A9
:102FC000EF900C94D011CF93DF931F921F92CDB747
:102FD000DEB74A8369830E94AF606981862F0E94B1
:102FE000E0604A81842F0E94E0600F900F90DF9193
:102FF000CF910C94D860AF92BF92CF92DF92EF92B4
:10300000FF920F931F93CF93DF9300D0CDB7DEB71E
:10301000182F022F4A835B8369830E94AF60698106
:10302000862F0E94E060812F81600E94D6604A81D5
:10303000A42E5B81B52E10E0E12CF12C680181E01B
:10304000C81AD108E016F10689F0EC14FD0419F451
:103050000E94FB6002C00E94F160F5018083FFEFD7
:10306000EF1AFF0A8FEFA81AB80AECCF0F900F9053
:103070000F90DF91CF911F910F91FF90EF90DF9014
:10308000CF90BF90AF900C94D860BF92CF92DF9258
:10309000EF92FF920F931F93CF93DF93CDB7DEB7DD
:1030A00060970FB6F894DEBF0FBECDBFF82EE42EAA
:1030B0006623D9F18E010F5F1F4F80E1F801119255
:1030C0008A95E9F728E0A80168E980EB0E94FB17E0
:1030D000FF2041F08FE693E09F938F930E94DA9355
:1030E0000F900F9026E7C22E23E0D22E37E0B32EAA
:1030F000B00EF80181918F011F928F93DF92CF92D2
:103100000E94DA930F900F900F900F90B012F1CFB2
:1031100088851F928F938BEC93E09F938F930E94EF
:10312000DA930F900F900F900F90EE20D9F18E014F
:103130000F5F1F4F80E1F80111928A95E9F720E1B6
:10314000A80160E880EB0E94FB17FF2041F08BE7AD
:1031500093E09F938F930E94DA930F900F9086E7EE
:10316000E82E83E0F82E9FE0D92ED00EF801819151
:103170008F011F928F93FF92EF920E94DA930F902C
:103180000F900F900F90D012F1CF88891F928F93DC
:103190008BEC93E09F938F930E94DA930F900F90A4
:1031A0000F900F9060960FB6F894DEBF0FBECDBFA4
:1031B000DF91CF911F910F91FF90EF90DF90CF9013
:1031C000BF9008950F931F93CF93DF931F921F9289
:1031D000CDB7DEB71A82198222E0AE014F5F5F4F92
:1031E0006AEA8EEE0E94FB1709E81DE1898190E0F2
:1031F000982F88272A81822BF8019183808322E0EF
:10320000AE014F5F5F4F6CEA8EEE0E94FB17898123
:1032100090E0982F88272A81822BF801938382835C
:1032200022E0AE014F5F5F4F6EEA8EEE0E94FB1709
:10323000898190E0982F88272A81822BF801958335
:10324000848322E0AE014F5F5F4F60EB8EEE0E9401
:10325000FB17898190E0982F88272A81822BF8011B
:10326000938B828B22E0AE014F5F5F4F62EB8EEE5D
:103270000E94FB17898190E0982F88272A81822B52
:10328000F801958B848B22E0AE014F5F5F4F64EBBA
:103290008EEE0E94FB17898190E0982F88272A8163
:1032A000822BF801978B868B22E0AE014F5F5F4F38
:1032B00066EB8EEE0E94FB17898190E0982F88279D
:1032C0002A81822BF8019783868322E0AE014F5F2B
:1032D0005F4F68EB8EEE0E94FB17898190E0982F7C
:1032E00088272A81822BF8019187808722E0AE010E
:1032F0004F5F5F4F6AEB8EEE0E94FB17898190E073
:10330000982F88272A81822BF8019587848722E0CD
:10331000AE014F5F5F4F6CEB8EEE0E94FB17898111
:1033200090E0982F88272A81822BF801978786873B
:1033300022E0AE014F5F5F4F6EEB8EEE0E94FB17F7
:10334000898190E0982F88272A81822BF801918B20
:10335000808B0F900F90DF91CF911F910F91089567
:103360002F923F924F925F926F927F928F929F9295
:10337000AF92BF92CF92DF92EF92FF920F931F9383
:10338000CF93DF93CDB7DEB76C970FB6F894DEBF5F
:103390000FBECDBF182F042F2D8B19821A821B82CE
:1033A0008091AD1D811107C06C8F0E94E21881E0F1
:1033B0008093AD1D6C8D662309F472C04EE264EFFC
:1033C0008EEE0E94E31762E174E380E090E00E94D9
:1033D000586022E0AE014F5F5F4F66EF8EEE0E94B5
:1033E000FB172981822F90E0A0E0B0E04427582FFE
:1033F000692F7A2F8A81482B80919F1D9091A01D63
:103400009A01AB01281B390B41095109A0919D1D5F
:10341000B0919E1D0E9404896B017C013FE0F594F0
:10342000E794D794C7943A95D1F76091971D70911E
:10343000981DCB01770FAA0BBB0BBC01CD014BE054
:10344000660F771F881F991F4A95D1F72091991D04
:1034500030919A1D4901330FAA08BB08A7019601B4
:10346000280D391D4A1D5B1D0E94BF88C20ED31E48
:10347000D092941DC092931D28E0C20ED11C54E03E
:10348000D594C7945A95E1F70D2C000CEE08FF086F
:10349000C092A11DD092A21DE092A31DF092A41D86
:1034A000812F8295880F880F807C8C5C8887212EE5
:1034B000312CA3E0B0E0012E02C0AA0FBB1F0A947A
:1034C000E2F72AE63AE00E94FD889B01AC012E5FFC
:1034D0003F4F4F4F5F4F29873A874B875C8780E587
:1034E00093ECA0E0B0E09C01AD0104C05595479578
:1034F000379527951A95D2F7298B3A8B4B8B5C8B96
:1035000010E0412C512C320188E090E0AC014219CE
:1035100053095B8F4A8F101709F43EC1488564EF49
:103520008EEE0E94E31769857A858B859C850E94C3
:10353000586023E0AE014F5F5F4F66EF8EEE0E9452
:10354000FB17E091931DF091941DE05AFF409F01FD
:10355000DF010E94E6886C837D838E839F83809148
:103560008B1D90918C1D9E878D872091891D309198
:103570008A1D388B2F8720918D1D30918E1D0E94C2
:10358000E6886B017C01ADE0F594E794D794C7948D
:10359000AA95D1F7A0918F1DB091901D2C813D81EE
:1035A0004E815F818CE055954795379527958A9593
:1035B000D1F70E940F89BB2797FDB095AB2F8C0DDB
:1035C0009D1DAE1DBF1D0296A11DB11D32E0B5951A
:1035D000A795979587953A95D1F79C01AD013058FD
:1035E0004F4F5F4FA0919B1DB0919C1D0E9404897D
:1035F0004B015C014FE0B694A794979487944A9549
:10360000D1F739818A8190E0A0E0B0E0BA2FA92FEC
:10361000982F8827A32B2B81822B9C01AD010A8C2C
:1036200004C055954795379527950A94D2F72E8B68
:103630003F8B488F598F4F8558896A01550FEE0887
:10364000FF0862E0CC0CDD1CEE1CFF1C6A95D1F774
:10365000A091911DB091921D2C813D814E815F8181
:103660000E940F899B01AC0177E1559547953795ED
:1036700027957A95D1F72C833D834E835F832D85E3
:103680003E85DF010E94E688DC01CB01EBE0B595C9
:10369000A79597958795EA95D1F72C813D814E8125
:1036A0005F81820F931FA41FB51FC80ED91EEA1E8B
:1036B000FB1E022C04C0CC0CDD1CEE1CFF1C0A946B
:1036C000D2F732E0C30ED11CE11CF11CF2E0F594FC
:1036D000E794D794C794FA95D1F72E893F89488DFE
:1036E000598D2C193D094E095F0969897A898B89A1
:1036F0009C890E94598897FD0BC0660F771F881F11
:10370000991FA50194010E949D8869017A010AC050
:10371000A50194010E949D8869017A01CC0CDD1CF1
:10372000EE1CFF1C9927F7FC9A958F2D7E2D6D2D91
:103730009B01AC010E9459889B01AC01AEEDBBE03E
:103740000E9404894C01BB2497FCB094AB2CA3E4E9
:10375000B3EEA70196010E941289BB2797FDB09591
:10376000AB2F880E991EAA1EBB1E4FEC840E4EE096
:10377000941EA11CB11C44E0B594A794979487941F
:103780004A95D1F7C80CD91CEA1CFB1C4C0C5D1CDB
:103790006E1C7F1C1F5FBFCE112381F0212F30E0F4
:1037A00040E050E0C301B2010E949D882093A51D16
:1037B0003093A61D4093A71D5093A81D5D895523E6
:1037C00089F16091A51D7091A61D8091A71D909112
:1037D000A81D611571058105910521F10E94748C68
:1037E00020E836EE45EC57E40E94C08B21E03EED28
:1037F00042E45EE30E94D98E9B01AC0160E070E080
:1038000080E89FE30E94DC8A2BE43AE34DEB57E328
:103810000E94C08B6093A91D7093AA1D8093AB1D5D
:103820009093AC1D6C960FB6F894DEBF0FBECDBF63
:10383000DF91CF911F910F91FF90EF90DF90CF908C
:10384000BF90AF909F908F907F906F905F904F90C0
:103850003F902F9008950F931F93CF93DF9300D045
:1038600000D0CDB7DEB78E010F5F1F4F86E0F801A5
:1038700011928A95E9F780919F1C811113C040E055
:1038800061E386EA0E94E3174AE06CE286EA0E945E
:10389000E31781E080939F1C68EF7CE780E090E075
:1038A0000E94586048E06DE286EA0E94E31768EFE4
:1038B0007CE780E090E00E94586026E0A80162E387
:1038C00086EA0E94FB1747E06DE286EA0E94E31752
:1038D0008A8190E0982F88272981822B90939A1CC7
:1038E0008093991C2C8130E0322F22274B81242B8E
:1038F00030939C1C20939B1C4E8150E0542F4427F6
:103900006D81462B50939E1C40939D1C5F934F935B
:103910003F932F939F938F938FE793E09F938F9382
:103920000E94DA930FB6F894DEBF0FBECDBF269685
:103930000FB6F894DEBF0FBECDBFDF91CF911F91C0
:103940000F910895CF92DF92EF92FF920F931F9302
:10395000CF93DF93CDB7DEB72A970FB6F894DEBFCB
:103960000FBECDBF8E010F5F1F4F86E0F801119291
:103970008A95E9F741E062E08CE30E94E31748E5AD
:1039800060E08CE30E94E31764E278E680E090E078
:103990000E94586026E0A80163E08CE30E94FB17B8
:1039A00043E062E08CE30E94E317098110E0102FEE
:1039B00000278A81082BE9E7FCE111830083EB8073
:1039C000F12CFE2CEE248C81E82AF382E282CD8059
:1039D000D12CDC2CCC248E81C82AD582C482B8019B
:1039E000012E000C880B990B0E94748C9B01AC017A
:1039F000B7010F2C000C880B990B2F833887498750
:103A00005A870E94748C2F81388549855A850E9477
:103A10005C8B20EE3EE245E652E40E946C8E20E094
:103A200030E044E353E40E94DD8A9F938F937F93B9
:103A30006F93DF92CF92FF92EF921F930F938DE8D7
:103A400093E09F938F930E94DA930FB6F894DEBFB2
:103A50000FBECDBF2A960FB6F894DEBF0FBECDBF06
:103A6000DF91CF911F910F91FF90EF90DF90CF905A
:103A70000895CF93DF93EC0188819981009759F1E4
:103A80008C32924121F01982188283E071C082E663
:103A90009AE00E94136F892B51F180919F139091AE
:103AA000A013A091A113B091A21393FD22C0809105
:103AB0009F139091A013A091A113B091A21394FD14
:103AC00049C080919F139091A013A091A113B09130
:103AD000A21395FD46C040E850E060E070E082E649
:103AE0009AE00E94F56E8CE292E19983888381E0EE
:103AF0003FC08091C52C82FFDACF21E048E061E031
:103B000083E00E94B0198091AC1D8F938091AB1D12
:103B10008F938091AA1D8F938091A91D8F9380917F
:103B2000A81D8F938091A71D8F938091A61D8F93C1
:103B30008091A51D8F9387ED91E19F938F930E94B4
:103B4000EE938DB79EB70A960FB6F8949EBF0FBE40
:103B50008DBFADCF8091C52C83FFB3CF0E942B1CAE
:103B6000B0CF8091C52C84FFB6CF0E94A21CB3CFEA
:103B7000DF91CF910895CF93DF93C82F8CEE0E94F1
:103B8000D6608C2F0E94E0606AE67AE080E090E0E8
:103B90000E9458608DEE0E94D6600E94F160D82F7E
:103BA0000E94FB60C82F0E94D8608C2F90E09D2B54
:103BB000DF91CF9108951F93CF93DF93C82F8CEEA1
:103BC0000E94D6608C2F0E94E06064E278E680E07C
:103BD00090E00E9458608CEE0E94D66080E00E94C7
:103BE000E0606AE67AE080E090E00E9458608DEE46
:103BF0000E94D6600E94F160D82F0E94F160182FB9
:103C00000E94FB60C82F0E94D860812F90E0A0E046
:103C1000B0E0BA2FA92F982F8827AD2BBC01CD017A
:103C20006C2BDF91CF911F9108952F923F924F926D
:103C30005F926F927F928F929F92AF92BF92CF923C
:103C4000DF92EF92FF920F931F93CF93DF93CDB745
:103C5000DEB7CB54D1090FB6F894DEBF0FBECDBF8F
:103C60008091040290910502892BE1F110920502E6
:103C7000109204028CEE0E94D6608EE10E94E060F9
:103C80000E94D86066E37CE980E090E00E94586082
:103C900082EA0E94BB1D9093530A8093520A84EAE1
:103CA0000E94BB1D9093510A8093500A86EA0E949D
:103CB000BB1D90934F0A80934E0A88EA0E94BB1D59
:103CC00090934D0A80934C0A8AEA0E94BB1D909300
:103CD0004B0A80934A0A8CEA0E94BB1D9093490AC2
:103CE0008093480A88E40E94DB1D6DAB7EAB8FABEE
:103CF00098AF88E50E94DB1D4B015C0180914A0A68
:103D000090914B0A8C0120E030E040E050E0BA0195
:103D100022968FAF229723961FAF239724962FAF1B
:103D2000249725963FAF259726964FAF269727963F
:103D30005FAF279728966FAF289729967FAF29976F
:103D40009C0140E050E060E070E080E090E008E03E
:103D50000E94728A0E942B8A3901B42FA52FF62F58
:103D6000E72F8C019401A50160E070E080E090E015
:103D70005301CB2EDA2EEF2EFE2E0E94A98A2CA301
:103D80003BA349835A831B012C01C20131504109D5
:103D90005F4F6F4F7F4F8F4F9F4F88248394912C9D
:103DA00021153F4F4F4F5140610571058105910528
:103DB00009F010F4812C912C34010091480A1091E3
:103DC000490A5801C12CD12CE12CF12C00E010E063
:103DD0002CA13BA149815A81B101C2010E941789DE
:103DE000F22E032F142FB52FF62FE72FD82EE92E02
:103DF000A0E00E94D08A84F42150310940485F4FEE
:103E00006F4F7F4F8F4F9F4FF22E032F142FB52FE1
:103E1000F62FE72FD82EE92E2F2D302F412F5B2F95
:103E20006F2F7E2F8D2D9E2D07E10E948B8A2B8F69
:103E30003C8F4D8F5E8F6F8F78A389A39AA32053F9
:103E4000384F4F4F5F4F6F4F7F4F8F4F9F4F2B8B91
:103E50003C8B4D8B5E8B6F8B788F898F9A8F205622
:103E6000304F4F4F5F4F6F4F7F4F8F4F9F4F243DCE
:103E7000304341055105610571058105910529F022
:103E800020F03401BFEF6B1A7B0A8090500A9090AB
:103E9000510A940140E050E060E070E080E090E082
:103EA00000E10E94728A2B833C834D835E836F8383
:103EB00078874C0140914C0A50914D0AACA0BBA0B0
:103EC000C980DA80710182019A0140E050E060E02F
:103ED00070E080E090E00E941789F22E032F142FEB
:103EE000B52FF62FE72FD82EE92EA0E00E94D08A1A
:103EF0005CF4AFE70E94B28AF22E032F142FB52F85
:103F0000F62FE72FD82EE92E2F2D302F412F5B2FA4
:103F10006F2F7E2F8D2D9E2D07E00E948B8A5901D9
:103F20006A017B018C012B813C814D815E816F8117
:103F30007885C4010E94A98A2B833C834D835E83CC
:103F40006F8378878F87988B2E5F3F4F434051094F
:103F50006E4F7F4F8F4F9F4F22303105494F5F4F3C
:103F6000644071058105910521F018F0FFEF6F1A8B
:103F70007F0A6091520A7091530A80E090E020E03D
:103F800030E840E050E00E94708929873A874B87EB
:103F90005C876D877E874C0140914E0A50914F0A95
:103FA000ACA0BBA0C980DA80710182019A0140E017
:103FB00050E060E070E080E090E00E941789F22E0F
:103FC000032F142FB52FF62FE72FD82EE92EA0E0C0
:103FD0000E94D08A84F421503F4F4F4F5F4F6F4F64
:103FE0007F4F8F4F9F4FF22E032F142FB52FF62F99
:103FF000E72FD82EE92E2F2D302F412F5B2F6F2F3B
:104000007E2F8D2D9E2D08E00E948B8A59016A011A
:104010007B018C0129853A854B855C856D857E8584
:10402000C4010E94A98A29873A874B875C876D87DC
:104030007E87898B9A8B2F5F3F4F414051096109E1
:10404000710981099109213030484C4F5F47614027
:1040500071058105910521F018F01FEF611A710AB1
:104060002B893C894D895E896F89788D898D9A8DE0
:104070002F3C3740410551056105710581059105CA
:1040800011F00CF09CC1ACA0BBA0C980DA8071011A
:1040900082019501A601B101C2010E941789A12CDC
:1040A000B12CC12CE0E8DE2EE12CF12C00E010E078
:1040B0000E949D8929AF3AAF4BAF5CAF6DAF7EAF29
:1040C0008FAF21969FAF2197AB8CBC8CCD8CDE8CB3
:1040D000EF8CF8A009A11AA19501A601B701C801AA
:1040E0000E94178959016A017B01E82F192F02E00C
:1040F0000E94728A0E2F0E94A98A7901142F452EE0
:10410000F62FE72F6C01922EAF2CB42E052F362EF2
:10411000B72F582E8D2CA0E00E94D08A5CF4A1E02D
:104120000E94B28A922EA32EB42E052F362EB72FC0
:10413000582E892E292D3A2D4B2D502F632D7B2F54
:10414000852D982D01E00E948B8A29A73AA74A0164
:104150002C966FAF2C972B967FAF2B978BA79CA796
:1041600029833A834BA39CA26DA37EA38FA398A718
:10417000B42D9701412F542D6F2F7E2FC601A0E043
:104180000E94D08A4CF4A3E00E94B28A7901142FD5
:10419000B52FF62FE72F6C019701412F5B2F6F2F63
:1041A0007E2FC60102E00E948B8A2DA73EA74FA753
:1041B00058AB69AB7AAB8BAB9CAB2901B42FA52F65
:1041C00022966FAF2297F72F1C012B893C894D89CE
:1041D0005E896F89788D898D9A8D24323A4F4F4F41
:1041E0005F4F6F4F7F4F8F4F9F4F0CF08BC02B8DCA
:1041F0003C8D4D8D5E8D6F8D78A189A19AA124553E
:10420000324F4F4F5F4F6F4F7F4F8F4F9F4F59012F
:104210006A017B018C010E94178919012A01B62FBE
:10422000A72FFC0103E00E94728A51016201EB2E6C
:10423000FA2E8F010E94BE8A59016A017B018C010E
:1042400029A53AA5A4012C966FAD2C972B967FAD8E
:104250002B978BA59CA50E94A98A29833A834BA3FF
:104260005CA36DA37EA38FA398A79101A2016B2FDE
:104270007A2FCF0102E00E94728A51016201EB2E77
:10428000FA2E8F010E94BE8A02E00E94728A0E2FCF
:104290000E94BE8A122FD32EE42EB52FF62FE72FC1
:1042A000F82E092FA0E00E94D08A5CF4A1E00E94C1
:1042B000B28A122FD32EE42EB52FF62FE72FF82E29
:1042C000092F212F3D2D4E2D5B2F6F2F7E2F8F2DF0
:1042D000902F01E00E948B8A59016A017B018C01B9
:1042E0002DA53EA54FA558A969A97AA98BA99CA976
:1042F0000E94A98A2901B42FA52F22966FAF229779
:10430000F72F1C012B813C814D815E816F81788567
:104310008F859889A980BA80CBA0DCA0EDA0FEA0F3
:104320000FA118A50E94BE8A2B833C834D835E8318
:104330006F8378878F87988B29853A854B855C8535
:104340006D857E8589899A895201CB2EDA2E229637
:10435000EFAC2297FF2E81010E94BE8A29873A87FF
:104360004B875C876D877E87898B9A8B2B893C89ED
:104370004D895E896F89788D898D9A8DA9ACBAAC8B
:10438000CBACDCACEDACFEAC0FAD21961FAD2197F4
:104390000E94BE8A2056304F4F4F5F4F6F4F7F4F66
:1043A0008F4F9F4F243D30434105510561057105F5
:1043B0008105910521F018F00FEF601A700A4DA9E0
:1043C0005EA96FA978AD9A01AB0160E070E0CB0106
:1043D00022962FAF229723963FAF239724964FAF75
:1043E000249725965FAF259726966FAF2697279639
:1043F0007FAF279728968FAF289729969FAF299749
:10440000A984BA84CB84DC84ED84FE8409891A896A
:1044100060E070E080E090E00E941789122FD32EB8
:10442000E42EB52FF62FE72FF82E092FA0E00E94DB
:10443000D08A84F421503109404E5F4F6F4F7F4F37
:104440008F4F9F4F122FD32EE42EB52FF62FE72F2D
:10445000F82E092F212F3D2D4E2D5B2F6F2F7E2FF4
:104460008F2D902F05E10E948B8AAB80BC80CD8080
:10447000DE80EF80F8840F8518890E94BE8A122F93
:10448000D32EE42EB52FF62FE72FF82E092FA0E01C
:104490000E94D08A84F4215030484F4F5F4F6F4FB5
:1044A0007F4F8F4F9F4F122FD32EE42EB52FF62F15
:1044B000E72FF82E092F212F3D2D4E2D5B2F6F2F2B
:1044C0007E2F8F2D902F0FE00E948B8A59016A0159
:1044D0007B018C01322E5B2CB42FAD2DF62F4F2C8F
:1044E0004C01285E33404109510961097109810974
:1044F0009109283D304D4140510561057105810507
:10450000910509F010F4672869F09501A601B7013B
:10451000C8010E942B8A322E532EB42FA52FF62FBE
:10452000472E4C01232D352D4B2F5A2F6F2F742DD5
:10453000C4010E946C8C20E030E048EC52E40E9400
:10454000C08BC55BDF4F0FB6F894DEBF0FBECDBF8B
:10455000DF91CF911F910F91FF90EF90DF90CF905F
:10456000BF90AF909F908F907F906F905F904F9093
:104570003F902F9008954F925F926F927F928F920B
:104580009F92AF92BF92CF92DF92EF92FF922B0158
:104590003C0169017A0123EC35EF4CE851E4C70195
:1045A000B6010E946C8E4B015C0128EB3EE143E7B3
:1045B00053E4C701B6010E94DD8A9B01AC01C5012D
:1045C000B4010E94C08B0E943A8C4B015C0120E038
:1045D00030E048EC52E4C301B2010E94C08B21E8F4
:1045E00035E943EC50E40E946C8EA50194010E94D1
:1045F0006C8E4B015C0123E333E948E853E4C701C7
:10460000B6010E94DD8A9B01AC01C501B4010E9484
:10461000C08B23E333EB48E553E40E946C8EFF909C
:10462000EF90DF90CF90BF90AF909F908F907F9052
:104630006F905F904F9008954F925F926F927F922C
:104640008F929F92AF92BF92CF92DF92EF92FF92A2
:1046500069017A010E94E08D20E030E040E050E402
:104660000E94DC8A22E93CE54EED5EE30E94C08BAD
:104670004B015C0123EC35EF4CE851E4C701B60176
:104680000E946C8E2B013C0128EB3EE143E753E492
:10469000C701B6010E94DD8A9B01AC01C301B201D2
:1046A0000E94C08B9B01AC01C501B4010E94DD8A50
:1046B0006B017C0128EB3EE143E753E40E946C8EE2
:1046C0004B015C01A701960163EC75EF8CE891E466
:1046D0000E94DC8A9B01AC01C501B4010E94C08B21
:1046E000FF90EF90DF90CF90BF90AF909F908F9012
:1046F0007F906F905F904F9008954F925F926F926E
:104700007F928F929F92AF92BF92CF92DF92EF9261
:10471000FF922B013C0169017A0123EC35EF4CE853
:1047200051E4C701B6010E946C8E4B015C0128EB7D
:104730003EE143E753E4C701B6010E94DD8A9B01D5
:10474000AC01C501B4010E94C08B0E943A8C4B01A0
:104750005C0120E030E048EC52E4C301B2010E9469
:10476000C08BA50194010E946C8E20E030E040E2F5
:1047700051E40E94DC8A24EE38E34EE05FE30E94BD
:104780006C8E9B01AC01C701B6010E94DD8AFF90CF
:10479000EF90DF90CF90BF90AF909F908F907F90E1
:1047A0006F905F904F90089580E80E94D6608111CD
:1047B0000DC08EEF0E94E060811108C066E37CE9C5
:1047C00080E090E00E9458600C94D8600E94D8600D
:1047D0008091D7309091D830A091D930B091DA3013
:1047E0000196A11DB11D8093D7309093D830A0932E
:1047F000D930B093DA300895FC01DC01AC014E5F92
:104800005F4F90E031E38D91982788E0292F220FA8
:1048100097FF03C0922F932701C0922F8150B1F7C9
:10482000A417B50781F721E030E08281981711F0D5
:1048300020E030E0C9010895DF92EF92FF920F93DC
:104840001F93CF93DF930E94D42380E80E94D66009
:1048500081116DC08AEF0E94E060811168C08FE015
:104860000E94E060811163C06AE67AE080E090E037
:104870000E94586081E80E94D660811158C00E9451
:10488000F160D82F0E94F1600E94F160182F0E9401
:10489000F1600E94F160082F0E94F1600E94FB60AD
:1048A000F82E80E80E94D660811141C08CEF0E94F2
:1048B000E06081113CC089EC0E94E060811137C04A
:1048C0006AE67AE080E090E00E94586081E80E9409
:1048D000D6600E94F160E82E0E94F160D82E0E94FE
:1048E000F1600E94F160C82F0E94FB601F92DF926E
:1048F0001F92EF921F92FF921F920F931F921F938E
:104900001F92DF931F928F931F92CF9382EA93E0BF
:104910009F938F930E94DA930E94D8608DB79EB7C1
:1049200042960FB6F8949EBF0FBE8DBF17C00E946F
:10493000D8608091D7309091D830A091D930B09183
:10494000DA300196A11DB11D8093D7309093D830F5
:10495000A093D930B093DA300E94D42320E030E025
:1049600040E050E060E070E080E090E0DF91CF91C7
:104970001F910F91FF90EF90DF900895EF92FF92BB
:104980000F931F93CF93DF9300D0CDB7DEB78C0189
:1049900080E80E94D660811154C00115110551F0C4
:1049A00085EE0E94E06081114CC062E07EE281E011
:1049B00090E009C083EE0E94E060811142C062E392
:1049C00075E783E090E00E94586081E80E94D6601D
:1049D000811137C00E94F160E82E89830E94F16046
:1049E000F82E8A830E94FB608B830E94D860CE01E0
:1049F00001960E94FC23892B21F16F2D70E07E2906
:104A00006C7F80E090E0012B69F00E94728C20E0C6
:104A100030E04AEF5AE30E946C8E20E030E040EC38
:104A200050E40CC00E94728C22E538EB4FE25BE34D
:104A30000E946C8E26E636E64BE352E40E94DC8A46
:104A40001BC00E94D8608091D7309091D830A0913F
:104A5000D930B091DA300196A11DB11D8093D730C5
:104A60009093D830A093D930B093DA300E94D423F9
:104A700060EF7FEF89E794E40F900F900F90DF9144
:104A8000CF911F910F91FF90EF9008950F931F9377
:104A9000CF93DF93729A8091660283FF08C08EE401
:104AA0000E947B60811165C0C0E5D0E009C0C0E50F
:104AB000D0E08FED97E00E944D0E2197D1F7EFCF18
:104AC0008FED97E00E944D0E2197D1F78FE40E9461
:104AD0007B600E94F160D82FDF730E94F160082F85
:104AE0000E94F160C82F0E94FB60182F0E94D860BE
:104AF0008091660283FF72986D2F70E0762F662793
:104B0000600F711D80E090E00E94728C20E134E023
:104B100048EC5BE30E946C8E6093B9287093BA28CE
:104B20008093BB289093BC286C2F70E0762F66276B
:104B3000610F711D769567957695679580E090E099
:104B40000E94728C24EA3CEF44E25CE30E946C8E8B
:104B500020E030E040E252E40E94DC8A60939A3523
:104B600070939B3580939C3590939D3580E090E0C9
:104B700002C081E090E0DF91CF911F910F910895E5
:104B80007298729A8EE40E947B6080EA0E94E060D4
:104B900080E00E94E06080E00E94E0608FE40E947C
:104BA0007B600E94F1608EE40E947B6080E80E943E
:104BB000E06080E00E94E06080E00E94E0600E948F
:104BC000D86080E090E0089586E091E19F938F9314
:104BD0000E94EE93809180020F900F90882361F0E5
:104BE0001F928F9383E091E19F938F930E94EE93A6
:104BF0000F900F900F900F9008958EED90E19F937E
:104C00008F930E94EE9386EB90E19F938F930E9487
:104C1000EE938FE890E19F938F930E94EE9384E54B
:104C200090E19F938F930E94EE9388E190E19F9390
:104C30008F930E94EE9386EE9FE09F938F930E9446
:104C4000EE938AEA9FE09F938F930E94EE9384E80D
:104C50009FE09F938F930E94EE938EE49FE09F933B
:104C60008F930E94EE938091C52C9091C62C8270F8
:104C700091702DB73EB72E5E3F4F0FB6F8943EBFF2
:104C80000FBE2DBF892B41F08EE19FE09F938F9344
:104C90000E94EE930F900F9082EF9EE09F938F9370
:104CA0000E94EE9386EB9EE09F938F930E94EE937B
:104CB0008DE89EE09F938F930E94EE9381E69EE0A5
:104CC0009F938F930E94EE9382E39EE09F938F9336
:104CD0000E94EE9380E09EE09F938F930E94EE935C
:104CE0008FEC9DE09F938F930E94EE9385E99DE06A
:104CF0009F938F930E94EE938FE59DE09F938F93F8
:104D00000E94EE938FE29DE09F938F930E94EE931B
:104D100083E09DE09F938F930E94EE9384ED9CE04F
:104D20009F938F930E94EE938BE99CE09F938F93C8
:104D30000E94EE9382E69CE09F938F930E94EE93F5
:104D40008BE29CE09F938F930E94EE938DEF9BE00C
:104D50009F938F930E94EE938DB79EB780960FB668
:104D6000F8949EBF0FBE8DBF89EC9BE09F938F93FD
:104D70000E94EE9388E99BE09F938F930E94EE93AD
:104D800089E69BE09F938F930E94EE938AE39BE0DA
:104D90009F938F930E94EE9383E19BE09F938F9369
:104DA0000E94EE938DED9AE09F938F930E94EE9375
:104DB00087EA9AE09F938F930E94EE9381E79AE0AF
:104DC0009F938F930E94EE9388E49AE09F938F9332
:104DD0000E94EE9380E19AE09F938F930E94EE935E
:104DE00085EE99E09F938F930E94EE932DB73EB787
:104DF0002A5E3F4F0FB6F8943EBF0FBE2DBF0895F9
:104E000081ED93E00C9416944F925F926F927F9293
:104E10008F929F92AF92BF92CF92DF92EF92FF92CA
:104E2000CF93DF93CDB7DEB728970FB6F894DEBFE8
:104E30000FBECDBF8091CB309091CC30A091CD30C2
:104E4000B091CE3089839A83AB83BC834090CB30C2
:104E50005090CC306090CD307090CE308091CB307F
:104E60009091CC30A091CD30B091CE308D839E8387
:104E7000AF83B8876091CB307091CC308091CD30CA
:104E80009091CE302CE3822E912CA12CB12CA50137
:104E900094010E949D887F936F9330E1C32E3EE082
:104EA000D32EE12CF12C6D817E818F819885A70115
:104EB00096010E949D88A50194010E949D883F93C0
:104EC0002F9340E8842E41E5942EAA24A394B12C7C
:104ED000C301B201A50194010E949D88A70196011A
:104EE0000E949D883F932F9369817A818B819C8159
:104EF000A50194010E949D883F932F938FEB99E029
:104F00009F938F930E94EE930FB6F894DEBF0FBE6F
:104F1000CDBF28960FB6F894DEBF0FBECDBFDF9190
:104F2000CF91FF90EF90DF90CF90BF90AF909F9088
:104F30008F907F906F905F904F900895EDEFF9E321
:104F4000808191818234924479F0ED5FF943FF933F
:104F5000EF9381EA99E09F938F930E94EE930F90D5
:104F60000F900F900F9008953A96E53F81E8F8076B
:104F700038F30895CF93DF93EC018C9A0E94BF1011
:104F80009F938F937F936F9385E999E09F938F937E
:104F90000E94EE930F900F900F900F900F900F9034
:104FA000209719F00E94D01108C083E999E09F93DF
:104FB0008F930E94EE930F900F9081E00E947110EA
:104FC000209185023091860240918702509188029B
:104FD0000E946C8E9F938F937F936F9387E899E0E5
:104FE0009F938F930E94EE930F900F900F900F90CE
:104FF0000F900F90209719F00E94D01108C085E8FB
:1050000099E09F938F930E94EE930F900F9082E010
:105010000E9471102091810230918202409183029E
:10502000509184020E946C8E9F938F937F936F9315
:1050300089E799E09F938F930E94EE930F900F90D2
:105040000F900F900F900F90209719F00E94D011A1
:1050500008C087E799E09F938F930E94EE930F908B
:105060000F9083E00E9471109F938F937F936F93B3
:1050700088E699E09F938F930E94EE938C980F900F
:105080000F900F900F900F900F90209719F00E94A3
:10509000D01108C086E699E09F938F930E94EE930B
:1050A0000F900F908091C52C87FF83C021E042E1D3
:1050B00061E080ED0E9442629F938F937F936F9394
:1050C00089E599E09F938F930E94EE930F900F9044
:1050D0000F900F900F900F90209719F00E94D01111
:1050E00008C087E599E09F938F930E94EE930F90FD
:1050F0000F9021E042E162E080ED0E9442629F93C6
:105100008F937F936F938AE499E09F938F930E948C
:10511000EE930F900F900F900F900F900F9020979D
:1051200019F00E94D01108C088E499E09F938F93F2
:105130000E94EE930F900F9021E042E163E080ED3A
:105140000E9442629F938F937F936F938BE399E0CA
:105150009F938F930E94EE930F900F900F900F905C
:105160000F900F90CD2B19F00E94D01108C089E349
:1051700099E09F938F930E94EE930F900F9021E000
:1051800042E164E080ED0E9442629F938F937F939F
:105190006F938CE299E09F938F930E94EE930F9010
:1051A0000F900F900F900F900F90DF91CF910C9474
:1051B000D011CD2BD1F3DF91CF9108950F931F9391
:1051C000CF93DF93882389F049E050E06FEF70E0E0
:1051D0008EE895E30E94289349E050E06EE070E08D
:1051E0008EE895E30E94B99613C0CEE8D5E307E2B6
:1051F00019E089911F928F931F930F930E94EE9352
:105200000F900F900F900F9085E3C639D80789F75C
:10521000DF91CF911F910F910C94D011882311F041
:10522000299A089529980895882311F02A9A0895B3
:105230002A980895CF92DF92EF92FF92CF93DF9357
:105240006B017C0160FF11C08EE094E09F938F930F
:105250008BE191E19F938F930E94EE930F900F90BB
:105260000F900F9081E090E002C080E090E0C1FEDE
:1052700009C0EC01219648E259E063E174E00E9424
:105280003916CE01C2FE09C0EC01219648E259E070
:105290006BE174E00E943916CE01C3FE09C0EC0137
:1052A000219648E259E063E274E00E943916CE018B
:1052B000C4FE09C0EC01219648E259E063E975E0BB
:1052C0000E943916CE01C5FE09C0EC01219648E2C4
:1052D00059E067E274E00E943916CE01C6FE09C0AB
:1052E000EC01219648E259E06BE274E00E94391625
:1052F000CE01C7FE09C0EC01219648E259E061E306
:1053000074E00E943916CE01D0FE09C0EC0121964E
:1053100048E259E069E374E00E943916CE01D1FEFB
:1053200009C0EC01219648E259E061E474E00E9472
:105330003916CE01D2FE09C0EC01219648E259E0AF
:1053400065E474E00E943916CE012091C52C30919D
:10535000C62C24703270232B59F0D3FE09C0EC0107
:10536000219648E259E06BE474E00E943916CE01C0
:105370002091C52C23FF0BC0D4FE09C0EC0121965F
:1053800048E259E060E574E00E943916CE012091B0
:10539000C52C24FF0BC0D5FE09C0EC01219648E2C4
:1053A00059E066E574E00E943916CE01D6FE09C0C8
:1053B000EC01219648E259E06EE574E00E9439164E
:1053C000CE01D7FE09C0EC01219648E259E069E61A
:1053D00074E00E943916CE01E0FE0CC048E259E0AC
:1053E0006AE774E0DF91CF91FF90EF90DF90CF906C
:1053F0000C943916CD28CE28CF2841F482E299E0CA
:105400009F938F930E94EE930F900F90DF91CF9117
:10541000FF90EF90DF90CF900895CF92DF92EF92C0
:10542000FF92CF93DF93EC01C12CD12C7601209712
:1054300009F4A3C06DE179E0CE010E94FA92892BB4
:1054400011F46894C0F865E179E0CE010E94FA9207
:10545000892B11F46894C1F86DE079E0CE010E94C7
:10546000FA92892B11F46894C2F869E079E0CE01D0
:105470000E94FA92892B11F46894C3F866E079E0EF
:10548000CE010E94FA92892B11F46894C4F862E06C
:1054900079E0CE010E94FA92892B11F46894C5F844
:1054A0006CEF78E0CE010E94FA92892B11F4689497
:1054B000C6F864EF78E0CE010E94FA92892B11F4CD
:1054C0006894C7F86CEE78E0CE010E94FA92892BBE
:1054D00011F46894D0F868EE78E0CE010E94FA9258
:1054E000892B11F46894D1F862EE78E0CE010E9425
:1054F000FA92892B11F46894D2F86DED78E0CE0120
:105500000E94FA92892B11F46894D3F867ED78E041
:10551000CE010E94FA92892B11F46894D4F86FECB2
:1055200078E0CE010E94FA92892B11F46894D5F8A4
:1055300064EC78E0CE010E94FA92892B11F4689411
:10554000D6F863EB78E0CE010E94FA92892B11F431
:105550006894D7F86EEA78E0CE010E94FA92892B1F
:1055600011F46894E0F860917E0270917F0280E00F
:1055700090E00E940E93EC015ACFC701B601DF9173
:10558000CF91FF90EF90DF90CF900895AF92BF92B0
:10559000CF92DF92EF92FF920F931F93CF93DF93FF
:1055A000D22FC32F8A01F62EC72ED82EE92E2170B6
:1055B00030E040E050E060E070E080E090E0A0E0AB
:1055C0000E94D08A89F08FE794E09F938F938BE1BC
:1055D00091E19F938F930E94EE930F900F900F9005
:1055E0000F90E1E0F0E002C0E0E0F0E08091C52C37
:1055F00080FF19C02D2F247030E040E050E060E0C3
:1056000070E080E090E0A0E00E94D08A61F05F014D
:105610008FEFA81AB80A48E259E063E874E0CF01B6
:105620000E943916F5012D2F227030E040E050E045
:1056300060E070E080E090E0A0E00E94D08A61F03D
:105640005F018FEFA81AB80A48E259E067E874E0F2
:10565000CF010E943916F5012D2F287030E040E06F
:1056600050E060E070E080E090E0A0E00E94D08A2E
:1056700061F05F018FEFA81AB80A48E259E06FE9BC
:1056800074E0CF010E943916F5012D2F207130E012
:1056900040E050E060E070E080E090E0A0E00E9438
:1056A000D08A61F05F018FEFA81AB80A48E259E08A
:1056B0006AE874E0CF010E943916F5012D2F20729F
:1056C00030E040E050E060E070E080E090E0A0E09A
:1056D0000E94D08A61F05F018FEFA81AB80A48E2F1
:1056E00059E06DE874E0CF010E943916F5012D2FC5
:1056F000207430E040E050E060E070E080E090E056
:10570000A0E00E94D08A61F05F018FEFA81AB80A6A
:1057100048E259E063E974E0CF010E943916F501CF
:105720002D2F207830E040E050E060E070E080E035
:1057300090E0A0E00E94D08A61F05F018FEFA81A8C
:10574000B80A48E259E069E974E0CF010E943916CD
:10575000F50120E03C2F317040E050E060E070E067
:1057600080E090E0A0E00E94D08A61F05F018FEFBE
:10577000A81AB80A48E259E06CE974E0CF010E9427
:105780003916F50120E03C2F327040E050E060E037
:1057900070E080E090E0A0E00E94D08A61F05F01BC
:1057A0008FEFA81AB80A48E259E061EA74E0CF0125
:1057B0000E943916F50120E03C2F347040E050E0A3
:1057C00060E070E080E090E0A0E00E94D08A61F0AC
:1057D0005F018FEFA81AB80A48E259E068EA74E05E
:1057E000CF010E943916F50120E03C2F387040E0CF
:1057F00050E060E070E080E090E0A0E00E94D08A9D
:1058000061F05F018FEFA81AB80A48E259E06BEA2D
:1058100074E0CF010E943916F50120E03C2F307171
:1058200040E050E060E070E080E090E0A0E00E94A6
:10583000D08A61F05F018FEFA81AB80A48E259E0F8
:1058400060EB74E0CF010E943916F50120E03C2F97
:10585000307240E050E060E070E080E090E0A0E076
:105860000E94D08A61F05F018FEFA81AB80A48E25F
:1058700059E067EB74E0CF010E943916F50120E092
:1058800030E040E050E06F2D647070E080E090E028
:10589000A0E00E94D08A61F05F018FEFA81AB80AD9
:1058A00048E259E06EEB74E0CF010E943916F50131
:1058B0008091C52C81FF19C020E03C2F307440E05E
:1058C00050E060E070E080E090E0A0E00E94D08ACC
:1058D00061F05F018FEFA81AB80A48E259E062EC64
:1058E00074E0CF010E943916F5018091C52C90918A
:1058F000C62C90FF19C020E030E040E0512F5071DD
:1059000060E070E080E090E0A0E00E94D08A61F06A
:105910005F018FEFA81AB80A48E259E065EC74E01D
:10592000CF010E943916F5018091C52C9091C62CAB
:1059300090FF19C020E030E040E0512F507260E04D
:1059400070E080E090E0A0E00E94D08A61F05F010A
:105950008FEFA81AB80A48E259E068EC74E0CF016A
:105960000E943916F5018091C52C9091C62C90FFAC
:1059700019C020E030E040E0512F507460E070E04A
:1059800080E090E0A0E00E94D08A61F05F018FEF9C
:10599000A81AB80A48E259E06EEC74E0CF010E9400
:1059A0003916F50120E03C2F307840E050E060E00F
:1059B00070E080E090E0A0E00E94D08A61F05F019A
:1059C0008FEFA81AB80A48E259E069ED74E0CF01F8
:1059D0000E943916F50120E030E0402F417050E080
:1059E00060E070E080E090E0A0E00E94D08A61F08A
:1059F0005F018FEFA81AB80A48E259E06EED74E033
:105A0000CF010E943916F50120E030E0402F4270AE
:105A100050E060E070E080E090E0A0E00E94D08A7A
:105A200061F05F018FEFA81AB80A48E259E061EE11
:105A300074E0CF010E943916F50120E030E040E02B
:105A400050E06F2D687070E080E090E0A0E00E9470
:105A5000D08A61F05F018FEFA81AB80A48E259E0D6
:105A600064EE74E0CF010E943916F50120E030E0C9
:105A700040E050E06F2D607170E080E090E0A0E0C9
:105A80000E94D08A61F05F018FEFA81AB80A48E23D
:105A900059E068EE74E0CF010E943916F50180915B
:105AA000C52C87FF19C020E030E0402F487050E03F
:105AB00060E070E080E090E0A0E00E94D08A61F0B9
:105AC0005F018FEFA81AB80A48E259E06CEE74E063
:105AD000CF010E943916F5018091C52C87FF19C0AE
:105AE00020E030E0402F407150E060E070E080E066
:105AF00090E0A0E00E94D08A61F05F018FEFA81AC9
:105B0000B80A48E259E060EF74E0CF010E9439160C
:105B1000F5018091C52C87FF19C020E030E0402FAF
:105B2000407250E060E070E080E090E0A0E00E9411
:105B3000D08A61F05F018FEFA81AB80A48E259E0F5
:105B400064EF74E0CF010E943916F5018091C52CF5
:105B500087FF19C020E030E0402F407450E060E043
:105B600070E080E090E0A0E00E94D08A61F05F01E8
:105B70008FEFA81AB80A48E259E068EF74E0CF0145
:105B80000E943916F5018091C52C82FF19C020E0D2
:105B900030E0402F407850E060E070E080E090E03E
:105BA000A0E00E94D08A61F05F018FEFA81AB80AC6
:105BB00048E259E066E276E0CF010E943916F5012D
:105BC0008091C52C82FF19C020E030E040E0512FC9
:105BD000517060E070E080E090E0A0E00E94D08A28
:105BE00061F05F018FEFA81AB80A48E259E06CEF44
:105BF00074E0CF010E943916F5018091C52C909177
:105C0000C62C90FF19C020E030E040E0512F5270C8
:105C100060E070E080E090E0A0E00E94D08A61F057
:105C20005F018FEFA81AB80A48E259E06FEF74E0FD
:105C3000CF010E943916F5018091C52C9091C62C98
:105C400090FF19C020E030E040E0512F547060E038
:105C500070E080E090E0A0E00E94D08A61F05F01F7
:105C60008FEFA81AB80A48E259E067E075E0CF0163
:105C70000E943916F5018091C52C9091C62C91FF98
:105C80001EC020E030E040E0512F587060E070E02E
:105C900080E090E0A0E00E94D08A89F048E259E0DC
:105CA00060E175E0CF01DF91CF911F910F91FF90DF
:105CB000EF90DF90CF90BF90AF900C9439162D2FBE
:105CC0003C2FA8016F2D7C2D8D2D9E2DA0E00E94D4
:105CD000D08A41F489EA98E09F938F930E94EE93D3
:105CE0000F900F90DF91CF911F910F91FF90EF9048
:105CF000DF90CF90BF90AF900895AF92BF92DF92A8
:105D0000EF92FF920F931F93CF93DF93EC015B0110
:105D1000FB01108264EA78E00E94FA92892B59F51F
:105D20008091C52C3DE4F32E00E882FF03C024E8F7
:105D3000E22E02C094E0E92E10E0D12C81FD00ECAF
:105D400026E04AE250E06BE270E089E290E00E94D7
:105D5000205E81E090E00E946811882311F08DE5BB
:105D6000F82E8091C52C9091C62C90FD16E091FFE5
:105D700007C0186005C0F12C00E0E12C10E0D12C28
:105D800062EA78E0CE010E94FA92892B61F481E008
:105D9000F501808360917E0270917F0280E090E047
:105DA0000E940E93EC0160EA78E0CE010E94FA9224
:105DB000892B61F48FEFF501808360917E027091F1
:105DC0007F0280E090E00E940E93EC01209709F49E
:105DD00038C16CE978E0CE010E94FA92892B19F45F
:105DE000FF2DF160FF2E68E978E0CE010E94FA9263
:105DF000892B19F48F2D8460F82E65E978E0CE01A7
:105E00000E94FA92892B19F4EF2DE260FE2E63E9CD
:105E100078E0CE010E94FA92892B19F4FF2DF860E8
:105E2000FF2E60E978E0CE010E94FA92892B19F4E6
:105E30008F2D8061F82E6AE878E0CE010E94FA92F8
:105E4000892B19F4EF2DE062FE2E64E878E0CE0194
:105E50000E94FA92892B19F4FF2DF064FF2E61E85D
:105E600078E0CE010E94FA92892B19F48F2D806878
:105E7000F82E6CE778E0CE010E94FA92892B09F4A3
:105E8000016065E778E0CE010E94FA92892B09F45F
:105E9000026062E778E0CE010E94FA92892B09F451
:105EA00004606DE678E0CE010E94FA92892B09F435
:105EB000086066E678E0CE010E94FA92892B09F428
:105EC00000616FE578E0CE010E94FA92892B09F417
:105ED00000626BE578E0CE010E94FA92892B19F4FA
:105EE000ED2DE460DE2E68E578E0CE010E94FA92A6
:105EF000892B09F4006463E578E0CE010E94FA92F0
:105F0000892B09F4006860E578E0CE010E94FA92DE
:105F1000892B19F4FE2DF160EF2E6DE478E0CE01AF
:105F20000E94FA92892B19F48E2D8260E82E6AE481
:105F300078E0CE010E94FA92892B19F4EE2DE460EC
:105F4000EE2E66E478E0CE010E94FA92892B19F4D5
:105F5000FE2DF860EF2E62E478E0CE010E94FA9206
:105F6000892B19F48E2D8061E82E6EE378E0CE0146
:105F70000E94FA92892B19F4EE2DE062EE2E6AE36C
:105F800078E0CE010E94FA92892B19F4FE2DF0647C
:105F9000EF2E68E378E0CE010E94FA92892B19F483
:105FA0008E2D8068E82E65E378E0CE010E94FA929B
:105FB000892B09F411606DE278E0CE010E94FA921B
:105FC000892B09F4126064E278E0CE010E94FA9213
:105FD000892B09F414606BE178E0CE010E94FA92FB
:105FE000892B09F4186068E178E0CE010E94FA92EA
:105FF000892B09F4106162E178E0CE010E94FA92E7
:10600000892B09F4106267E078E0CE010E94FA92D1
:10601000892B09F4106463E078E0CE010E94FA92C3
:10602000892B19F4ED2DE860DE2E6FEF77E0CE01BD
:106030000E94FA92892B09F0C0CEFD2DF061DF2E6F
:10604000BCCE2F2D302F4E2D512F6D2D70E080E0C6
:1060500090E0DF91CF911F910F91FF90EF90DF9033
:10606000BF90AF9008955F926F927F928F929F92B0
:10607000AF92BF92CF92DF92EF92FF920F931F9356
:10608000CF93DF93782EC8EADCE100E010E089EFDF
:10609000E82E87E0F82E872D8170582E872D82708C
:1060A000682E94EEC92E97E0D92E2CEEA22E27E072
:1060B000B22E3AEE832E37E0932E772051F01F93C5
:1060C0000F93FF92EF920E94EE930F900F900F901C
:1060D0000F905520A1F089858F9388858F93BF926B
:1060E000AF920E94EE930F900F900F900F9066204A
:1060F000C1F09F928F920E94EE930F900F906620B6
:1061000081F0DF92CF920E94EE93288139814A81FB
:106110005B816C817D818E819F810E94C62A0F9058
:106120000F900E94D0110F5F1F4F2A960430110567
:1061300021F6DF91CF911F910F91FF90EF90DF90AB
:10614000CF90BF90AF909F908F907F906F905F9017
:1061500008958FED97E09F938F930E94EE93809127
:10616000B5289091B628A091B728B091B8280F9083
:106170000F90813027EA92072EE1A207B10519F4AA
:1061800081ED97E01DC0823026EA92072EE1A2073A
:10619000B10519F484EC97E013C0823027EA920726
:1061A0002EE1A207B10519F486EB97E009C0823011
:1061B00028EA92072EE1A207B10549F488EA97E0A0
:1061C0009F938F930E94EE930F900F900895BF932B
:1061D000AF939F938F9382EA97E09F938F930E9450
:1061E000EE930F900F900F900F900F900F900895D7
:1061F00082E997E09F938F930E94EE930E9400277D
:106200000E94A9300E94D0118FE89CE19F938F9348
:106210008AE897E09F938F930E94EE9360916002CB
:1062200070916102809162029091630228EE33E0E6
:1062300040E050E00E949D885F934F933F932F93DF
:106240008AE797E09F938F930E94EE9381E797E010
:106250009F938F930E94EE930E9462168091C52CAB
:106260002DB73EB7225F3F4F0FB6F8943EBF0FBE2B
:106270002DBF80FF05C041E061E081E00E9445182C
:106280008DE697E09F938F930E94EE9380E00E94AB
:10629000DE280E940427809165021F928F9384E676
:1062A00097E09F938F930E94EE9380919C131F928F
:1062B0008F938BE597E09F938F930E94EE9380914D
:1062C00090028F9380918F028F9380918E028F9393
:1062D00080918D028F938DE497E09F938F930E941E
:1062E000EE931F9280E48F9385E397E09F938F93C3
:1062F0000E94EE938091A4371F928F938091A337D1
:106300001F928F9382E297E09F938F930E94EE9368
:10631000809164021F928F9389E197E09F938F93FE
:106320000E94EE938091660290916702A0916802AC
:10633000B09169022DB73EB7225E3F4F0FB6F89479
:106340003EBF0FBE2DBF96FD03C08CE195E002C09D
:1063500089E195E09F938F938FE097E09F938F93D0
:106360000E94EE9383E00E9433300F900F900F90C5
:106370000F901D9903C08CE195E002C089E195E082
:106380009F938F9383E097E09F938F930E94EE9368
:1063900089EF96E09F938F930E94EE93809166021F
:1063A0000F900F900F900F900F900F9081FF09C0EA
:1063B00083EF96E09F938F930E94EE930F900F9040
:1063C00013C080FD03C08CE195E002C089E195E037
:1063D0009F938F938FEE96E09F938F930E94EE93FF
:1063E0000F900F900F900F9080916602909167022E
:1063F000A0916802B091690297FD03C08CE195E01D
:1064000002C089E195E09F938F9386EE96E09F937B
:106410008F930E94EE938FED96E09F938F930E944F
:10642000EE9360919F137091A0138091A1139091AE
:10643000A2130E941A290E94D0110F900F900F9062
:106440000F900F900F90779B03C08CE195E002C0F6
:1064500089E195E09F938F9386ED96E09F938F93CC
:106460000E94EE930E94530E0E9424119F938F93DB
:106470007F936F9388EC96E09F938F930E94EE93A7
:106480000E94D3109F938F937F936F938AEB96E034
:106490009F938F930E94EE9381E090E00E94BA2731
:1064A0008091743590917535A0917635B09177359E
:1064B000BF93AF939F938F938CEA96E09F938F93B4
:1064C0000E94EE93809189358F93809188358F93C8
:1064D000809187358F93809186358F9388E996E0F8
:1064E0009F938F930E94EE938091783590917935A8
:1064F000A0917A35B0917B35BF93AF939F938F93E3
:106500008AE896E09F938F930E94EE938DB79EB793
:1065100082960FB6F8949EBF0FBE8DBF80918D35C9
:106520008F9380918C358F9380918B358F93809151
:106530008A358F9386E796E09F938F930E94EE9320
:1065400061E070E080E090E00E94D91161E070E0CD
:1065500081E090E00E94D9110F900F900F900F9062
:106560000F900F90299903C08CE195E002C089E15A
:1065700095E09F938F938EE696E09F938F930E9472
:10658000EE930F900F900F900F902A9903C08CE11B
:1065900095E002C089E195E09F938F9386E696E0AF
:1065A0009F938F930E94EE930F900F900F900F90F8
:1065B0000895F89491E2E0E0F0E090935700849120
:1065C000E2E0F0E0909357002491E4E0F0E0909353
:1065D0005700E49190E0A0E0B0E0BC0155274427CB
:1065E000822F90E0A0E0B0E0BA2FA92F982F882743
:1065F000840F951FA61FB71F8E0F911DA11DB11DE2
:106600008093B5289093B628A093B728B093B82864
:1066100078940895CF93DF93CDB7DEB761970FB627
:10662000F894DEBF0FBECDBF48E250E062E270E0FA
:1066300088EA9CE10E949B962091A81C3091A91C9D
:106640004091AA1C5091AB1C6091AC1C7091AD1C88
:106650008091AE1C9091AF1CAFEF0E94D08A09F0E0
:106660005DC08DE48093A81C80E88093A91C84E021
:106670008093AA1C1092AB1C1092AC1C1092AD1C03
:106680001092AE1C1092AF1C8CE390E09093B11C62
:106690008093B01C1092B21C1092B31C1092B41CC8
:1066A0001092B51C1092B61C1092B71C1092B81C18
:1066B0001092B91C1092BB1C1092BA1C1092BC1CF8
:1066C0001092BD1C1092BE1C1092BF1C1092C01CD8
:1066D0001092C11C1092C21C1092C31C1092C51CB7
:1066E0001092C41C1092C61C1092C71C1092C81C99
:1066F0001092C91C1092CA1C1092CB1C1092CC1C78
:106700001092CD1C1092CF1C1092CE1C48E250E08B
:1067100062E270E088EA9CE10E94B99644E050E0B1
:106720006EE170E0CE010B960E949B968B859C8556
:10673000AD85BE858F3F2FEF9207A207B207A9F460
:106740008AE090E4A0E0B0E0809366029093670254
:10675000A0936802B093690244E050E06EE170E0FB
:1067600086E692E00E94B99608C0809366029093F4
:106770006702A0936802B0936902809166029091CB
:106780006702A0916802B0916902A2FF02C02A9A32
:1067900003C080E00E94142944E050E06AE570E004
:1067A000CE010B960E949B968B859C85AD85BE8500
:1067B0008F3F2FEF9207A207B20789F410929F1321
:1067C0001092A0131092A1131092A21344E050E073
:1067D0006AE570E08FE993E10E94B99608C0809362
:1067E0009F139093A013A093A113B093A21349E019
:1067F00050E06EE070E08EE895E30E949B960E9468
:10680000071344E050E06EE470E0CE010B960E9466
:106810009B968B859C85AD85BE8544E050E06EE4FB
:1068200070E08F3F9F4FAF4FBF4F29F485E892E054
:106830000E94B99604C085E892E00E949B9644E0CD
:1068400050E06AE470E0CE010B960E949B968B8527
:106850009C85AD85BE8544E050E06AE470E08F3FE2
:106860009F4FAF4FBF4F29F481E892E00E94B99645
:1068700004C081E892E00E949B9644E050E062E50B
:1068800070E0CE010B960E949B968B859C85AD8512
:10689000BE8544E050E062E570E08F3F9F4FAF4F10
:1068A000BF4F29F489E892E00E94B99604C089E8B4
:1068B00092E00E949B9641E050E06DE170E0CE01D5
:1068C00041960E949B96898941E050E06DE170E01D
:1068D0008F3F29F48CE993E10E94B99604C08CE9BA
:1068E00093E10E949B9641E050E06CE170E0CE01A4
:1068F00041960E949B96898941E050E06CE170E0EE
:106900008F3F29F485E692E00E94B99604C085E69F
:1069100092E00E949B9641E050E06BE170E0CE0176
:1069200041960E949B96898941E050E06BE170E0BE
:106930008F3F29F484E692E00E94B99604C084E671
:1069400092E00E949B964AE050E064E070E0CE0145
:1069500001960E949B9689814AE050E064E070E0D5
:106960008F3F29F48FE89CE10E94B99604C08FE81C
:106970009CE10E949B9644E050E066E570E0CE0109
:106980000B960E949B968B859C85AD85BE8544E0C9
:1069900050E066E570E08F3F9F4FAF4FBF4F29F447
:1069A0008DE892E00E94B99604C08DE892E00E94C2
:1069B0009B9644E050E067E170E0CE010B960E94A8
:1069C0009B968B859C85AD85BE8544E050E067E154
:1069D00070E08F3F9F4FAF4FBF4F29F480E692E0AA
:1069E0000E94B99604C080E692E00E949B96809136
:1069F000600290916102A0916202B09163028138BD
:106A00009A41A640B105A0F083EF92E09F938F9347
:106A10000E94EE9380E197E2A0E0B0E080936002F4
:106A200090936102A0936202B09363020F900F9063
:106A300060916002709161028091620290916302A4
:106A40000E94656042E050E062E070E0CE010F9687
:106A50000E949B968F85988942E050E062E070E04A
:106A60008F3F910529F485E993E10E94B99604C00E
:106A700085E993E10E949B9642E050E060E070E07F
:106A8000CE010F960E949B968F85988942E050E038
:106A900060E070E08F3F910529F483E993E10E9463
:106AA000B99604C083E993E10E949B9661960FB664
:106AB000F894DEBF0FBECDBFDF91CF910895CF9286
:106AC000DF92EF92FF9260917E0270917F0280E0F0
:106AD00090E00E940E9360E275E00E942F93892B54
:106AE00009F03BC18DE48093A81C80E88093A91C29
:106AF00084E08093AA1C1092AB1C1092AC1C1092E4
:106B0000AD1C1092AE1C1092AF1C8CE390E09093E1
:106B1000B11C8093B01C1092B21C1092B31C109246
:106B2000B41C1092B51C1092B61C1092B71C109297
:106B3000B81C1092B91C1092BB1C1092BA1C109277
:106B4000BC1C1092BD1C1092BE1C1092BF1C109257
:106B5000C01C1092C11C1092C21C1092C31C109237
:106B6000C51C1092C41C1092C61C1092C71C109217
:106B7000C81C1092C91C1092CA1C1092CB1C1092F7
:106B8000CC1C1092CD1C1092CF1C1092CE1C48E24F
:106B900050E062E270E088EA9CE10E94B9968AE0E7
:106BA00090E4A0E0B0E08093660290936702A09327
:106BB0006802B093690244E050E06EE170E086E65E
:106BC00092E00E94B99610929F131092A013109217
:106BD000A1131092A21344E050E06AE570E08FE93F
:106BE00093E10E94B99682E2C82EDD24DA948CECFF
:106BF000E82E8BE3F82EC0928502D0928602E092B6
:106C00008702F092880244E050E06EE470E085E88C
:106C100092E00E94B996C0928102D0928202E092E4
:106C20008302F092840244E050E06AE470E081E87C
:106C300092E00E94B99687ED94E3AFEEBCE38093B7
:106C4000890290938A02A0938B02B0938C0244E055
:106C500050E062E570E089E892E00E94B9968AE926
:106C600099E9A9E1B0E480938D0290938E02A093FC
:106C70008F02B093900244E050E066E570E08DE84A
:106C800092E00E94B99610929C1380E00E94D56A0F
:106C900041E050E06DE170E08CE993E10E94B9962B
:106CA0008AE1809365020E94AE6941E050E06CE1A8
:106CB00070E085E692E00E94B9968FE080936402CE
:106CC00041E050E06BE170E084E692E00E94B9960A
:106CD0008AE0EFE8FCE1DF011D928A95E9F74AE0DE
:106CE00050E064E070E0CF010E94B99680E197E245
:106CF000A0E0B0E08093600290936102A0936202F2
:106D0000B093630244E050E067E170E080E692E017
:106D10000E94B996109296131092951342E050E09B
:106D200062E070E085E993E10E94B99610929413B5
:106D30001092931342E050E060E070E083E993E149
:106D40000E94B99681E00E94DE2880E090E0FF90EA
:106D5000EF90DF90CF900C941C13FF90EF90DF909A
:106D6000CF9008950E94CC666C9A6B9A6A9A6F9A3B
:106D7000729A749A739A779A809880B3897F80BB4D
:106D80008398849887E080937E00549A0E94D93239
:106D90000E940A330E94C10E80E090E00E941C1302
:106DA0006091600270916102809162029091630231
:106DB0000E9465600E94D3106093C7307093C83002
:106DC0008093C9309093CA308091660286FD239AE1
:106DD000219A229A239A0E94D60E1D9B05C01092DA
:106DE0009E1310929D13089581E090E090939E135E
:106DF00080939D130895CF93DF9390E040919F136C
:106E00005091A0136091A1137091A21341FD08C08D
:106E10002091660220FD04C021FF8CC01D9B8AC00A
:106E20002DE8289FE001299FD00D1124CE018B541D
:106E3000924E9F938F9387E295E09F938F930E944A
:106E4000DA93FE01E255F24EDF01AA57BF4F2C91B3
:106E50000F900F900F900F90438154816581768140
:106E60008091CB309091CC30A091CD30B091CE308C
:106E7000841B950BA60BB70B2223D1F1BF93AF93C5
:106E80009F938F93DF01A257BF4F11968C9111975B
:106E90008F938C918F93129711968C9111978F935A
:106EA0008C918F9313978C911F928F9311978C9144
:106EB0001F928F9313968C911F928F9311978C91A1
:106EC0001F928F93E957FF4F80811F928F931F92DC
:106ED0002F938DE295E09F938F930E94DA938DB765
:106EE0009EB746960FB6F8949EBF0FBE8DBF10C0DA
:106EF000BF93AF939F938F9384E795E09F938F9376
:106F00000E94DA930F900F900F900F900F900F90B8
:106F10000E94D01180918002882361F01F928F938C
:106F200080EF92E09F938F930E94EE930F900F90CB
:106F30000F900F90DF91CF9108958091AE1D88231F
:106F400041F08091AF1D90E00E94FB360E94C70F78
:106F5000F4CF0895CF93DF93EC0188819981893F25
:106F60002EE09207F1F018F4892BC1F04BC081306C
:106F70002FE0920709F44CC085309F4009F042C0D1
:106F800086E59AE00E94136F892B09F43FC086E5DD
:106F90009AE00E94FF6E80E00E940E2989EF9EE039
:106FA0002EC0623199F5299A409193135091941310
:106FB0005695542F44275795479560E070E086E535
:106FC0009AE00E94F56E80919F139091A013A0917A
:106FD000A113B091A213A0FF10C0809194138F93BE
:106FE000809193138F9380EC91E19F938F930E94F4
:106FF000EE930F900F900F900F9081E09FE0998398
:10700000888304C01982188283E019C081E017C008
:1070100086E59AE00E94136F892BC1F386E59AE01A
:107020000E94FF6E0E949D3740E250E060E070E0F9
:1070300086E59AE00E94F56E85E09FE0E0CFDF9163
:10704000CF9108952F923F924F925F926F927F92CD
:107050008F929F92AF92BF92CF92DF92EF92FF9268
:107060000F931F93CF93DF93CDB7DEB72B970FB658
:10707000F894DEBF0FBECDBF9B878A873A01FC0123
:1070800080819181892B11F00C944F4C60917E028C
:1070900070917F02CA010E940E9360E870E0C30104
:1070A0000E944E93009759F46091F7397091F83926
:1070B0008AE090E00E94A29381E00C94544C8130CD
:1070C000910561F4F3011081912E990C9908892C96
:1070D000092D292C392C492C592CB9C08230910505
:1070E000B9F4F3018081082E000C990B982F8827A2
:1070F0002181820F911D27FD9A95182F992E892E97
:10710000880C8808082D282C382C482C582C9FC017
:1071100083309105B1F5F3012081922F990F990BDE
:10712000392F492F592F692F792F892F00E10E947C
:10713000728A19012A014B01B82FA92F2181922FA0
:10714000990F990B392F492F592F692F792F892F93
:1071500008E00E94728A59016A017B018C01910149
:10716000A201B4018B2F9A2F0E94A98AA2801A2D06
:10717000110F110BB12EC12ED12EE12EF12E012FA8
:1071800055C004970CF45BC0F3012081922F990F36
:10719000990B392F492F592F692F792F892F08E102
:1071A0000E94728A19012A014B01B82FA92F21814F
:1071B000922F990F990B392F492F592F692F792F1A
:1071C000892F00E10E94728A59016A017B018C01BA
:1071D0009101A201B4018B2F9A2F0E94A98AA3804A
:1071E0001A2D110F110BB12EC12ED12EE12EF12E21
:1071F000012F0E94A98A19012A014B01B82FA92F3A
:107200002281922F990F990B392F492F592F692FCE
:10721000792F892F08E00E94728A59016A017B0147
:107220008C019101A201B4018B2F9A2F0E94A98A8F
:10723000122F932E842E052F1B012C0108C01AE05B
:10724000912C812C00E0212C312C412C512C0E94BE
:10725000D011212F392D482D502FB101C2012537D2
:10726000F3E63F07FDE64F0751056105710581050E
:10727000910511F40C9437472537E3E63E07EDE618
:107280004E075105610571058105910511F008F062
:10729000B2C12337F2E73F0741055105610571058A
:1072A0008105910511F40C94D0492337E2E73E079C
:1072B00041055105610571058105910511F008F041
:1072C000B9C02536F4E63F07410551056105710552
:1072D0008105910509F4D1C72536E4E63E0741054D
:1072E0005105610571058105910511F008F041C056
:1072F000A6E70E94D08A11F40C94BF430E94D08A62
:1073000009F070F4A8E60E94D08A11F40C948E4122
:10731000A5E70E94D08A11F40C94A9430C944D4C1B
:10732000212F392D482D502FB101C2012436F1E60D
:107330003F0741055105610571058105910511F46E
:107340000C94F8492537E2E63E07410551056105F1
:1073500071058105910509F431C52A33364241058D
:107360005105610571058105910509F430C30C943F
:107370004D4C212F392D482D502FB101C2012737F7
:10738000EFE63E074105510561057105810591054F
:1073900011F40C949D472737FFE63F07410551053F
:1073A000610571058105910509F0C8F42436E9E607
:1073B0003E0741055105610571058105910511F4EF
:1073C0000C94824325363E46410551056105710501
:1073D0008105910511F40C94D1470C944D4C212F4B
:1073E000392D482D502FB101C2012536E2E73E0765
:1073F00041055105610571058105910511F40C9454
:107400009D482936F2E73F074105510561057105A1
:107410008105910511F40C947F49233331474105CF
:107420005105610571058105910511F00C944D4CD4
:107430000C94F849212F392D482D502FB101C2014C
:107440002236F5E63F07F4E64F0751056105710561
:107450008105910509F411C72236E5E63E07E4E609
:107460004E075105610571058105910511F008F080
:107470005BC02133F4E63F07F1E64F075105610594
:1074800071058105910509F4B6C22133E4E63E0792
:10749000E1E64E075105610571058105910509F089
:1074A000C0F42337F3E73F07410551056105710536
:1074B0008105910511F40C94E449283734474105BE
:1074C0005105610571058105910509F480C20C948F
:1074D0004D4C212F392D482D502FB101C201283795
:1074E000F4E63F07F1E64F07510561057105810597
:1074F000910509F47CC22C36E5E73E07E2E64E072B
:107500005105610571058105910509F457C42336BC
:10751000344641465105610571058105910511F01B
:107520000C944D4C0C94F849212F392D482D502F97
:10753000B101C2012D36E5E73E07E8E64E075105E9
:10754000610571058105910511F40C940E4A2D36E3
:10755000F5E73F07F8E64F0751056105710581051D
:10756000910509F0E0F42237E2E73E07E5E64E0731
:107570005105610571058105910511F40C94E846EA
:1075800023363D4648465105610571058105910543
:1075900011F00C944D4C0E94A21C0C944F4C212FC6
:1075A000392D482D502FB101C2012436E3E63E07A4
:1075B000ECE64E075105610571058105910511F451
:1075C0000C944B462736FFE63F07FCE64F07510574
:1075D000610571058105910511F40C944E46233621
:1075E000324349465105610571058105910511F048
:1075F0000C944D4C20C2212F392D482D502FB10114
:10760000C2012037FCE63F07F5E64F07F8E65F07C3
:10761000610571058105910509F480C62037ECE606
:107620003E07E5E64E07E8E65E0761057105810560
:10763000910511F008F0E0C02437F8E73F07F4E7C0
:107640004F075105610571058105910511F40C94F1
:107650002B442437E8E73E07E4E74E075105610570
:1076600071058105910511F008F05DC02033F1E34B
:107670003F07F1E74F075105610571058105910548
:1076800011F40C94E8462033E1E33E07E1E74E07AE
:107690005105610571058105910509F0C0F421339B
:1076A000F2E63F07F0E74F075105610571058105D7
:1076B000910509F498C222333246404751056105CD
:1076C00071058105910509F4E3C20C944D4C212FFD
:1076D000392D482D502FB101C2012037F5E63F0763
:1076E000F2E74F075105610571058105910511F418
:1076F0000C949D482C36E4E73E074E075105610582
:1077000071058105910511F40C94734B21333143BC
:1077100041475105610571058105910511F00C94F2
:107720004D4C0C943747212F392D482D502FB10146
:10773000C2012B36ECE63E07E5E74E07E2E65E07C0
:10774000610571058105910509F438C32B36FCE606
:107750003F07F5E74F07F2E65F0761057105810511
:10776000910509F0E0F42437E4E63E07E7E74E0729
:107770005105610571058105910511F40C94C14B0A
:1077800024373F464F4652466105710581059105F4
:1077900011F00C944D4C0C9400000C944F4C212F84
:1077A000392D482D502FB101C2012E36E1E63E079A
:1077B000E8E64E07E3E65E07610571058105910580
:1077C00011F40C94FF432633F9E63F07F5E74F0722
:1077D000F5E65F07610571058105910509F4A2C50C
:1077E00029363C46414653466105710581059105A0
:1077F00011F00C944D4C7FC3212F392D482D502F63
:10780000B101C2012437F3E73F07F5E64F07F2E77E
:107810005F07610571058105910511F40C944D48D0
:107820002437E3E73E07E5E64E07E2E75E0761053A
:1078300071058105910511F008F062C02337F5E666
:107840003F07F2E74F07F0E75F0761057105810524
:10785000910511F40C94BE4A2337E5E63E07E2E7B2
:107860004E07E0E75E07610571058105910509F0A6
:10787000D0F42136FDE63F07F5E74F07F8E65F074E
:10788000610571058105910511F40C94BB47223700
:10789000374740475047610571058105910509F457
:1078A0005CC20C944D4C212F392D482D502FB10125
:1078B000C2012436FDE63F07F3E64F07F2E75F0714
:1078C000610571058105910509F437C62136ECE69D
:1078D0003E07E5E64E07E2E75E07610571058105B3
:1078E000910509F43CC523373247474750476105A6
:1078F00071058105910511F00C944D4C0C94504884
:10790000212F392D482D502FB101C2012437E2E734
:107910003E07E1E64E07E5E75E0761057105810573
:10792000910509F465C62437F2E73F07F1E64F07F2
:10793000F5E75F07610571058105910509F0C8F458
:107940002437E3E73E07E5E64E07E4E75E07610517
:1079500071058105910509F4A9C7273730474847C4
:107960005447610571058105910509F41EC70C9402
:107970004D4C212F392D482D502FB101C2012F36EA
:10798000ECE63E07EFE54E07E6E75E0761057105A9
:107990008105910509F47CC52C36F1E63F07F4E733
:1079A0004F07F8E75F07610571058105910511F43F
:1079B0000C94404B223737464047554761057105C7
:1079C0008105910511F00C944D4C0C94274683E0F1
:1079D00080937C3510927E3510927D354CE755E3CF
:1079E00062E182E492E00E9485700C944F4C0E9408
:1079F0002B1C0C944F4C21E042E161E080ED0E9491
:107A0000426221E042E161E080ED0E94426221E0B9
:107A100042E161E080ED0E94426221E042E161E0EA
:107A200080ED0E94426221E042E161E080ED0E942F
:107A300042620C944F4C60917E0270917F0280E014
:107A400090E00E940E9360E875E00E942F93892BCE
:107A500009F0C5C060917E0270917F0280E090E0E5
:107A60000E940E938C01009709F497C064E673E0BE
:107A70000E942F93892BE1F488EE93E0A0E0B0E020
:107A80008093600290936102A0936202B0936302BC
:107A900068EE73E080E090E00E94656044E050E0B2
:107AA00067E170E080E692E00E94B9960C944F4C3A
:107AB00066E875E0C8010E942F93892BE1F480E10C
:107AC00097E2A0E0B0E08093600290936102A093FF
:107AD0006202B093630260E177E280E090E00E948E
:107AE000656044E050E067E170E080E692E00E946B
:107AF000B9960C944F4C69E875E0C8010E942F9329
:107B0000892BE1F480EA96E8A1E0B0E0809360027E
:107B100090936102A0936202B093630260EA76E8F8
:107B200081E090E00E94656044E050E067E170E031
:107B300080E692E00E94B9960C944F4C6DE875E097
:107B4000C8010E942F93892BE1F480E89AE1A6E016
:107B5000B0E08093600290936102A0936202B093C0
:107B6000630260E87AE186E090E00E94656044E0AC
:107B700050E067E170E080E692E00E94B9960C94D4
:107B80004F4C8EE994E09F938F930E94EE930E9456
:107B9000D0110F900F900C944F4C60916002709137
:107BA0006102809162029091630228EE33E040E02E
:107BB00050E00E949D885F934F933F932F938AE9F3
:107BC00094E09F938F930E94EE930E94D0110F90A8
:107BD0000F900F900F900F900F900C944F4C0E94AD
:107BE00062160C944F4C60917E0270917F0280E08F
:107BF00090E00E940E938C0169E175E00E942F9342
:107C0000892BA1F48091660290916702A09168028D
:107C1000B0916902A2608093660290936702A0937C
:107C20006802B0936902299A0C944F4C6CE175E09C
:107C3000C8010E942F93892BB1F480916602909124
:107C40006702A0916802B0916902AD7F80936602DD
:107C500090936702A0936802B093690280E00E944B
:107C60000E290C944F4C299903C08CE195E002C079
:107C700089E195E09F938F9382E994E09F938F939E
:107C80000E94EE930F900F900F900F900C944F4C1A
:107C900060917E0270917F0280E090E00E940E93DE
:107CA0008C0169E175E00E942F93892BE1F48091AA
:107CB000660290916702A0916802B0916902A46087
:107CC0008093660290936702A0936802B093690262
:107CD0002A9A44E050E06EE170E086E692E00E946D
:107CE000B9960C944F4C6CE175E0C8010E942F933B
:107CF000892BF1F48091660290916702A09168024D
:107D0000B0916902AB7F8093660290936702A09363
:107D10006802B093690280E00E94142944E050E0B8
:107D20006EE170E086E692E00E94B9960C944F4CAA
:107D30002A9903C08CE195E002C089E195E09F9308
:107D40008F938AE894E09F938F930E94EE930F9015
:107D50000F900F900F900C944F4C60917E02709199
:107D60007F0280E090E00E940E938C0169E175E053
:107D70000E942F93892B19F477980C944F4C6CE147
:107D800075E0C8010E942F93892B19F4779A0C94FF
:107D90004F4C779B03C08CE195E002C089E195E0F0
:107DA0009F938F9380E596E09F938F930E94EE932D
:107DB0000F900F900F900F900C944F4C60917E029B
:107DC00070917F0280E090E00E940E938C0161E947
:107DD00075E00E942F93892BD1F48091AE1D1F92E4
:107DE0008F938091B01D1F928F938091AF1D1F9232
:107DF0008F931F9284E18F9380E694E09F938F93FB
:107E00000E94EE930FB6F894DEBF0FBECDBF66E9B9
:107E100075E0C8010E942F93892B19F40E949D37A9
:107E200066C06EE975E0C8010E942F93892BF1F5B9
:107E300060917E0270917F0280E090E00E940E933C
:107E4000009709F454C00E94FB918531910528F5F3
:107E5000909396138093951342E050E062E070E0B7
:107E600085E993E10E94B99660917E0270917F024C
:107E700080E090E00E940E930097C9F10E94FB9170
:107E8000909394138093931342E050E060E070E08D
:107E900083E993E10E94B9962AC08EE494E09F930F
:107EA0008F930E94EE930F900F9021C080919613B4
:107EB0008F93809195138F9385E494E09F938F9394
:107EC0000E94EE930E94D011809194138F93809121
:107ED00093138F9386E394E09F938F930E94EE9386
:107EE0000E94D0110FB6F894DEBF0FBECDBF0E9426
:107EF000D0110C944F4C60917E0270917F0280E013
:107F000090E00E940E938C016EED74E00E942F931E
:107F1000892B09F077C060917E0270917F0280E02A
:107F200090E00E940E938C01009711F40C944F4C3A
:107F30006CE975E00E942F93892BB1F482E29FEFE8
:107F4000ACECBBE38093850290938602A0938702FA
:107F5000B093880244E050E06EE470E085E892E07F
:107F60000E94B9960C944F4C62EA75E0C8010E94D9
:107F70002F93892BB1F482E29FEFACECBAE38093AC
:107F8000850290938602A0938702B093880244E012
:107F900050E06EE470E085E892E00E94B9960C949F
:107FA0004F4CC8010E94F7912B013C0120E030E0CA
:107FB000A9010E94BB8B8823D9F081E00E94711037
:107FC0009B01AC01C301B2010E94C08B609385028A
:107FD00070938602809387029093880244E050E079
:107FE0006EE470E085E892E00E94B9960C944F4CE4
:107FF00089E294E09F938F930E94EE930F900F90ED
:108000000C944F4C61EE74E0C8010E942F93892BB1
:1080100009F077C060917E0270917F0280E090E06D
:108020000E940E938C01009711F40C944F4C6CE954
:1080300075E00E942F93892BB1F482E29FEFACECA4
:10804000BBE38093810290938202A0938302B0935A
:10805000840244E050E06AE470E081E892E00E942B
:10806000B9960C944F4C62EA75E0C8010E942F93B8
:10807000892BB1F482E29FEFACECBAE380938102EA
:1080800090938202A0938302B093840244E050E074
:108090006AE470E081E892E00E94B9960C944F4C3B
:1080A000C8010E94F7912B013C0120E030E0A901BA
:1080B0000E94BB8B8823D9F082E00E9471109B0143
:1080C000AC01C301B2010E94C08B60938102709326
:1080D0008202809383029093840244E050E06AE439
:1080E00070E081E892E00E94B9960C944F4C8CE1CC
:1080F00094E09F938F930E94EE930F900F900C94B7
:108100004F4C69ED74E0C8010E942F93892B09F050
:1081100073C060917E0270917F0280E090E00E94C7
:108120000E938C01009711F40C944F4C6CE975E0A0
:108130000E942F93892BB1F487ED94E3AFEEBCE35B
:108140008093890290938A02A0938B02B0938C0251
:1081500044E050E062E570E089E892E00E94B99660
:108160000C944F4C62EA75E0C8010E942F93892B52
:1081700051F48DE094E09F938F930E94EE930F90C3
:108180000F900C944F4CC8010E94F7912B013C01B9
:1081900020E030E0A9010E94BB8B882319F180E028
:1081A0000E9471104B015C0121EE3AE744E95EE365
:1081B000C301B2010E94DC8AA50194010E94C08B18
:1081C0006093890270938A0280938B0290938C0251
:1081D00044E050E062E570E089E892E00E94B996E0
:1081E0000C944F4C80E094E09F938F930E94EE9309
:1081F0000F900F900C944F4C0E94BF109F938F9341
:108200007F936F9389EF93E09F938F930E94EE93F8
:1082100082E00E947110209181023091820240918F
:108220008302509184020E946C8E162F072FF82E25
:10823000E92E81E00E947110EF92FF920F931F933D
:1082400020918502309186024091870250918802E8
:108250000E946C8E9F938F937F936F938DEE93E02C
:108260009F938F930E94EE930E94D0110FB6F894C3
:10827000DEBF0FBECDBF0C944F4C60917E0270915B
:108280007F0280E090E00E940E93009711F10E941F
:108290000D2A00919F131091A0132091A1133091EA
:1082A000A213601771078207930739F160939F1338
:1082B0007093A0138093A1139093A21344E050E015
:1082C0006AE570E08FE993E10E94B99689E496E04F
:1082D00002C082E496E09F938F930E94EE93609198
:1082E0009F137091A0138091A1139091A2130E94EB
:1082F0001A290E94D0110F900F9087E396E09F9368
:108300008F930E94EE936FEF7FEFCB010E941A29AB
:108310000E94D0110F900F900C944F4C0E94FD259D
:108320000C944F4CF3018481843329F440E061E0E4
:1083300080E00E94451880918002882311F40C94FB
:108340004F4C1F928F9384E396E09F938F930E94EC
:10835000EE930F900F900F900F900C944F4CF301F1
:108360008481893709F080C060917E0270917F021C
:1083700080E090E00E940E938C0169E175E00E941C
:108380002F93892B51F48091660290916702A091FE
:108390006802B0916902906410C06CE175E0C80198
:1083A0000E942F93892BD1F48091660290916702ED
:1083B000A0916802B09169029F7B809366029093BE
:1083C0006702A0936802B093690244E050E06EE156
:1083D00070E086E692E00E94B99646C067EA75E0D2
:1083E000C8010E942F93892B21F58091A71C8F93A0
:1083F0008091A61C8F938091A51C8F938091A41CC3
:108400008F938091A31C8F938091A21C8F93809156
:10841000A11C8F938091A01C8F9382EC93E09F937B
:108420008F930E94EE930FB6F894DEBF0FBECDBFC0
:108430001BC08091660290916702A0916802B09182
:10844000690296FD03C08CE195E002C089E195E0E8
:108450009F938F938EEB93E09F938F930E94EE9365
:108460000F900F900F900F9080918002882311F44D
:108470000C944F4C1F928F9381E396E09F938F93C0
:108480000E94EE930F900F900F900F900C944F4C12
:10849000F30184818737E9F560917E0270917F0254
:1084A00080E090E00E940E930097D9F00E94F7912F
:1084B0002B013C0120E030E0A9010E94BB8B882306
:1084C00081F040928D0250928E0260928F027092E3
:1084D000900244E050E066E570E08DE892E00E9492
:1084E000B996809190028F9380918F028F938091A3
:1084F0008E028F9380918D028F9380EB93E09F93F8
:108500008F930E94EE930F900F900F900F900F900B
:108510000F9080918002882311F40C944F4C1F928D
:108520008F938EE296E09F938F930E94EE930F902D
:108530000F900F900F900C944F4C60917E027091B1
:108540007F0280E090E00E940E938C0169E175E06B
:108550000E942F93409066025090670260906802DC
:1085600070906902892B19F4689457F809C06CE17E
:1085700075E0C8010E942F93892B99F4E89457F86D
:10858000409266025092670260926802709269029D
:1085900044E050E06EE170E086E692E00E94B99619
:1085A00013C057FC03C08CE195E002C089E195E05F
:1085B0009F938F938CEA93E09F938F930E94EE9307
:1085C0000F900F900F900F9080918002882311F4EC
:1085D0000C944F4C1F928F938BE296E09F938F9356
:1085E0000E94EE930F900F900F900F900C944F4CB1
:1085F00060917E0270917F0280E090E00E940E9375
:108600008C016DEA75E00E942F93892B11F489E1AA
:1086100008C061EB75E0C8010E942F93892B49F4D3
:1086200080E18093C4001092C50082E08093C00076
:1086300055C065EB75E0C8010E942F93892B11F49A
:1086400088E0EFCF6AEB75E0C8010E942F93892B79
:1086500039F06FEB75E0C8010E942F93892B11F45C
:1086600083E0DFCF8091C400893141F487EA93E051
:108670009F938F930E94EE930F900F908091C40070
:10868000803141F482EA93E09F938F930E94EE93AE
:108690000F900F908091C400883041F48CE993E0F2
:1086A0009F938F930E94EE930F900F908091C40040
:1086B000833041F486E993E09F938F930E94EE9379
:1086C0000F900F908091C400883041F480E993E0CE
:1086D0009F938F930E94EE930F900F908091800252
:1086E000882311F40C944F4C1F928F9388E296E0EC
:1086F0009F938F930E94EE930F900F900F900F9087
:108700000C944F4C60917E0270917F0280E090E06B
:108710000E940E936CE975E00E942F93892B11F44F
:1087200081E001C080E00E94DE28809180028823E1
:1087300011F40C944F4C1F928F9385E296E09F9317
:108740008F930E94EE930F900F900F900F900C94C8
:108750004F4C0E94042780918002882311F40C94CE
:108760004F4C1F928F9382E296E09F938F930E94CB
:10877000EE930F900F900F900F900C944F4C0E941F
:10878000002780918002882311F40C944F4C1F9293
:108790008F938FE196E09F938F930E94EE930F90BB
:1087A0000F900F900F900C944F4C60917E0270913F
:1087B0007F0280E090E00E940E930E94FB91803146
:1087C00070F480939C130E94D56A41E050E06DE103
:1087D00070E08CE993E10E94B9960C944F4C809123
:1087E0009C131F928F9386E893E09F938F930E9430
:1087F000EE930F900F900F900F900C944F4C609150
:108800007E0270917F0280E090E00E940E930E94B1
:10881000FB9195EF980F903170F4809365020E9460
:10882000AE6941E050E06CE170E085E692E00E94C4
:10883000B9960C944F4C809165021F928F938DE7EF
:1088400093E09F938F930E94EE930F900F900F9061
:108850000F900C944F4C60917E0270917F0280E0EB
:1088600090E00E940E93009789F04AE050E0BC012E
:108870008FE89CE10E943F934AE050E064E070E0A2
:108880008FE89CE10E94B9960C944F4C8FE89CE1D4
:108890009F938F9384EC95E09F938F930E94DA933C
:1088A0000F900F900F900F900C944F4C60917E02A0
:1088B00070917F0280E090E00E940E938C0164E64C
:1088C00073E00E942F93892BD9F4219A809166023C
:1088D00090916702A0916802B091690280618093D3
:1088E000660290936702A0936802B093690244E025
:1088F00050E06EE170E086E692E00E94B996CFC744
:1089000062EE74E0C8010E942F93892BD9F4229A59
:108910008091660290916702A0916802B09169020D
:1089200080628093660290936702A0936802B0937E
:10893000690244E050E06EE170E086E692E00E9459
:10894000B996ADC766E473E0C8010E942F93892BE6
:10895000D9F4239A8091660290916702A0916802EF
:10896000B091690280648093660290936702A0933D
:108970006802B093690244E050E06EE170E086E680
:1089800092E00E94B9968BC765E874E0C8010E9426
:108990002F93892BD9F4239A8091660290916702D4
:1089A000A0916802B09169028068809366029093FA
:1089B0006702A0936802B093690244E050E06EE160
:1089C00070E086E692E00E94B99669C76AE779E0AE
:1089D000C8010E942F93892B71F581E08093E030CC
:1089E00088EA9CE19093E2308093E1301092E43089
:1089F0001092E3308091660290916702A091680224
:108A0000B091690291608093660290936702A0938F
:108A10006802B093690244E050E06EE170E086E6DF
:108A200092E00E94B99640EE50E362E182E492E067
:108A30000E94857034C76DE673E0C8010E942F93D1
:108A4000892B11F5E8EDFCE1119211922CE1E83F40
:108A5000F207D1F78091660290916702A0916802B7
:108A6000B091690292608093660290936702A0932E
:108A70006802B093690244E050E06EE170E086E67F
:108A800092E00E94B9960BC76CE175E0C8010E94A4
:108A90002F93409166025091670260916802709135
:108AA0006902892BC1F44F705C7F4093660250933A
:108AB000670260936802709369022B9A44E050E069
:108AC0006EE170E086E692E00E94B996809185356D
:108AD0000E94C369E4C644FD03C08CE195E002C076
:108AE00089E195E09F938F9382E793E09F938F9323
:108AF0000E94EE93809166020F900F900F900F905E
:108B000085FD03C08CE195E002C089E195E09F936B
:108B10008F9387E693E09F938F930E94EE938091CB
:108B200066020F900F900F900F9086FD03C08CE1AE
:108B300095E002C089E195E09F938F938CE593E0E7
:108B40009F938F930E94EE93809166020F900F90F7
:108B50000F900F9087FD03C08CE195E002C089E182
:108B600095E09F938F9381E593E09F938F930E946D
:108B7000EE938091660290916702A0916802B09195
:108B800069020F900F900F900F9090FD03C08CE141
:108B900095E002C089E195E09F938F9386E493E08E
:108BA0009F938F930E94EE9380916602909167024B
:108BB000A0916802B09169020F900F900F900F90F2
:108BC00091FD03C08CE195E002C089E195E09F939F
:108BD0008F938BE393E09F938F930E94EE9380910A
:108BE000660290916702A0916802B09169020F90AD
:108BF0000F900F900F9091FF52C68CEC95E00E9461
:108C0000169498EDE92E9CE1F92E00E010E024ED99
:108C1000822E25E0922EF70180819181F2E0EF0E05
:108C2000F11C9F938F93C8010B969F938F939F92F4
:108C30008F920E94DA930F5F1F4F0F900F900F904B
:108C40000F900F900F900031110529F728C68BE186
:108C500096E09F938F930E94EE93809180020F90F5
:108C60000F90882361F01F928F9388E196E09F9385
:108C70008F930E94EE930F900F900F900F90F894A7
:108C800098E088E10FB6F894A895809360000FBE35
:108C900090936000FFCF0E94F36101C660917E0255
:108CA00070917F0280E090E00E940E938C0169E158
:108CB00075E00E942F93892BE9F40E94B26880919D
:108CC000660290916702A0916802B09169028D7F5F
:108CD00081608093660290936702A0936802B093CC
:108CE000690244E050E06EE170E086E692E00E94A6
:108CF000B996D5C56CE175E0C8010E942F93892B08
:108D0000E1F40E94E8678091660290916702A09169
:108D10006802B09169028C7F80936602909367022B
:108D2000A0936802B093690244E050E06EE170E005
:108D300086E692E00E94B996B2C56FED75E0C80173
:108D40000E942F93892BE9F40E94E86780916602C4
:108D500090916702A0916802B09169028E7F826053
:108D60008093660290936702A0936802B0936902B1
:108D700044E050E06EE170E086E692E00E94B99631
:108D80008EC58091660281FF0FC08FED95E09F93A5
:108D90008F9387E393E09F938F930E94EE930F90BE
:108DA0000F900F900F907BC580FD03C08CE195E084
:108DB00002C089E195E09F938F9383E393E09F93B3
:108DC0008F930E94EE930F900F900F900F9067C5B6
:108DD0008091DE308F938091DD308F938091DC30F5
:108DE0008F938091DB308F938091DA308F938091D5
:108DF000D9308F938091D8308F938091D7308F93D3
:108E00008091D6308F938091D5308F938091D430DC
:108E10008F938091D3308F938091D2308F938091B4
:108E2000D1308F938091D0308F938091CF308F93BA
:108E30008CEE95E09F938F930E94EE930E94D01149
:108E4000809180020FB6F894DEBF0FBECDBF88239D
:108E500009F425C51F928F9389EE95E09F938F9318
:108E60000E94EE930F900F900F900F9018C5F894FA
:108E700089E021E030E0F90180935700C895E02CAB
:108E800020E030E0F90180935700C895F02C7894E9
:108E9000F89423E030E0F90180935700C895002D45
:108EA00022E030E0F90180935700C895102D7894A6
:108EB0008091B8288F938091B7288F938091B6289E
:108EC0008F938091B5288F938FED95E09F938F932B
:108ED0000E94EE931F92EF921F92FF921F920F93A8
:108EE0001F921F9388EB95E09F938F930E94EE93C0
:108EF0000E949E27809166001F928F938CEA95E0D6
:108F00009F938F930E94EE930E94D01180918002D4
:108F10000FB6F894DEBF0FBECDBF882309F4BFC4DF
:108F20001F928F9389EA95E09F938F930E94EE930F
:108F30000F900F900F900F90B2C460E070E080E04F
:108F400090E00E94D91160E070E081E090E00E9422
:108F5000D91180918002882309F4A1C41F928F93B4
:108F600086EA95E09F938F930E94EE930F900F9067
:108F70000F900F9094C40E94C0250E94D011809140
:108F80008002882309F48BC41F928F9383EA95E0B3
:108F90009F938F930E94EE930F900F900F900F90DE
:108FA0007EC460917E0270917F0280E090E00E941A
:108FB0000E9366E975E00E942F93892B31F5F894A2
:108FC00081E99AE00E945E718C01892B69F0C801E9
:108FD0000F960E94CB6DB80188E092E00E940F725C
:108FE000C8010E94C371F0CF81E99AE00E94B67176
:108FF000892B29F081E99AE00E947271F5CF81E90D
:109000009AE00E945A71789436C081E99AE00E94F1
:109010005E718C0184EEE82E85E0F82E01151105B5
:1090200051F1F80186811F928F9380851F928F9353
:1090300085811F928F9381851F928F9387811F92C5
:109040008F9384811F928F9383811F928F9382814C
:109050001F928F9382851F928F93FF92EF920E94AF
:10906000DA93C8010E94C3718C010FB6F894DEBF79
:109070000FBECDBFD3CF80918002882309F40FC4E7
:109080001F928F9380EA95E09F938F930E94EE93B7
:109090000F900F900F900F9002C40E945F35FFC396
:1090A00060917E0270917F0280E090E00E940E93BA
:1090B0008C0163E276E00E942F93892BD1F480919A
:1090C000660290916702A0916802B0916902977F51
:1090D0008093660290936702A0936802B09369023E
:1090E00044E050E06EE170E086E692E00E94B996BE
:1090F000D6C362EA75E0C8010E942F93892BD1F490
:109100008091660290916702A0916802B091690215
:1091100098608093660290936702A0936802B09370
:10912000690244E050E06EE170E086E692E00E9461
:10913000B996B5C30E94530EB2C360917E0270917E
:109140007F0280E090E00E940E93FC012081233298
:10915000C1F44AE050E060E070E001960E94958F13
:109160007B836A8360917E0270917F0280E090E051
:109170000E940E932A813B81243031050CF096C069
:1091800002C01B821A82009709F490C01982BE01A6
:109190006F5F7F4F0E947D2E19013A014B01B82F5E
:1091A000A92F8AE02A813B81829FF001839FF00DE5
:1091B0001124E855F34E4080518032813C838381F5
:1091C0008D8394819E8325812F8336813887878183
:1091D00089879101A301B4018B2F9A2F5201CC8072
:1091E000DD80EE80FF80088519850E94C78A09F41A
:1091F00060C08981811103C0208231822AC0181683
:1092000084F4422853289C81692A2D81722A3E8148
:10921000832A8F81982A9885B92B2985A22B408291
:1092200017C0209430946094709480949094B0957A
:10923000A095242053203C8163228D8178229E8139
:1092400089222F8192223885B3238985A823208201
:1092500051826282738284829582B683A78348E2B8
:1092600050E062E270E088EA9CE10E94B99688E9E9
:1092700095E09F938F930E94EE938AE02A813B8131
:10928000829FF001839FF00D1124E855F34E208159
:1092900031814281538164817581868197810E94E9
:1092A000C62A0E94D0110F900F9003C082E00E9446
:1092B00033308CE895E09F938F930E94EE932FEFCD
:1092C0003FEF4FEF5FEF6FEF7FEF8FEF9FEF0E946A
:1092D000C62A0E94D011809180020F900F9088239F
:1092E00009F4DDC21F928F9389E895E09F938F93D5
:1092F0000E94EE930F900F900F900F90D0C260914C
:109300007E0270917F0280E090E00E940E93FC014B
:1093100020812332A1F44AE050E060E070E0019641
:109320000E94958F8B0160917E0270917F0280E098
:1093300090E00E940E9304301105ECF402C000E0AE
:1093400010E00097C1F04AE050E060E070E00E9459
:10935000C0902AE0209FF001219FF00D1124E855D4
:10936000F34E7187608748E250E062E270E088EA7D
:109370009CE10E94B99681E00E9433308091800286
:10938000882309F48CC21F928F9386E895E09F93FF
:109390008F930E94EE930F900F900F900F907FC2CB
:1093A0000E94527280918002882309F478C21F9231
:1093B0008F9383E895E09F938F930E94EE930F9095
:1093C0000F900F900F906BC20E94F8308091800236
:1093D000882309F464C21F928F9380E895E09F93DD
:1093E0008F930E94EE930F900F900F900F9057C2A3
:1093F00080E090E00E94BA2780918002882309F4DF
:109400004EC21F928F938DE795E09F938F930E949A
:10941000EE930F900F900F900F9041C28091C52C4A
:1094200081FF2DC00E944625892B49F58091BC28DB
:109430008F938091BB288F938091BA288F938091CE
:10944000B9288F9382E795E09F938F930E94EE93C4
:1094500080919D358F9380919C358F9380919B3522
:109460008F9380919A358F9385E695E09F938F93A4
:109470000E94EE930FB6F894DEBF0FBECDBF0E94E0
:10948000D0118091C52C9091C62C90FF63C081E0D3
:1094900090E00E94BE247B011C0180E090E00E94CD
:1094A000BE244B018C010E941C243F922F92FF92FC
:1094B000EF9284E595E09F938F930E94EE931F9324
:1094C0000F939F928F9284E495E09F938F930E94D5
:1094D000EE93240138019401A80147018101B701ED
:1094E000C1010E94BB229F938F937F936F9389E367
:1094F00095E09F938F930E94EE93242D352D462D5A
:10950000572D6E2D792D822D912F0E941C239F9314
:109510008F937F936F938BE295E09F938F930E943D
:10952000EE93242D352D462D572D6E2D792D822D20
:10953000912F0E947D239F938F937F936F9388E158
:1095400095E09F938F930E94EE930FB6F894DEBF41
:109550000FBECDBF0E94D01180918002882309F4F4
:109560009EC11F928F9385E195E09F938F930E94F8
:10957000EE930F900F900F900F9091C18091C52C9A
:1095800082FF2BC021E048E061E083E00E94B01937
:109590008091AC1D8F938091AB1D8F938091AA1DFC
:1095A0008F938091A91D8F938091A81D8F93809197
:1095B000A71D8F938091A61D8F938091A51D8F93DA
:1095C0008EEF94E09F938F930E94EE930E94D011B0
:1095D0000FB6F894DEBF0FBECDBF8091C52C909121
:1095E000C62C91FF3BC00E94151E20E030E048ECE5
:1095F00052E4162F072FF82EE92E0E946C8E20E8D9
:1096000036EE45EC57E40E94C08B21E03EED42E48B
:109610005EE30E94D98E9B01AC0160E070E080E8BF
:109620009FE30E94DC8A2BE43AE34DEB57E30E9470
:10963000C08B9F938F937F936F93EF92FF920F93C3
:109640001F9385EE94E09F938F930E94EE930E9468
:10965000D0110FB6F894DEBF0FBECDBF809180024F
:10966000882309F41CC11F928F9382EE94E09F938C
:109670008F930E94EE930F900F900F900F900FC159
:1096800060917E0270917F0280E090E00E940E93D4
:1096900068E276E00E942F93892B99F460917E0214
:1096A00070917F0280E090E00E940E93009709F491
:1096B000F6C00E94FB9190915201892B8093520138
:1096C000EEC0809152018F701F928F9386E293E0DB
:1096D0009F938F930E94EE930E94D0110F900F9052
:1096E0000F900F90DCC060917E0270917F0280E04D
:1096F00090E00E940E93009711F14AE050E060E084
:1097000070E00E94958F603198F4609364021F921C
:109710006F9385ED94E09F938F930E94EE9341E0C9
:1097200050E06BE170E084E692E00E94B99611C0CF
:10973000809164021F928F938CEC94E006C080911C
:1097400064021F928F9383EC94E09F938F930E9407
:10975000EE930F900F900F900F900E94D011809178
:109760008002882309F49BC01F928F9380EC94E0C1
:109770009F938F930E94EE930F900F900F900F90F6
:109780008EC060917E0270917F0280E090E00E9426
:109790000E938C0169E175E00E942F93892BE1F40F
:1097A0000E94DB668091660290916702A091680238
:1097B000B091690290618093660290936702A093D2
:1097C0006802B093690244E050E06EE170E086E622
:1097D00092E00E94B99663C06CE175E0C8010E94F6
:1097E0002F93892B99F5F8940E94E8660FB6F894A8
:1097F000A89580916000886180936000109260005D
:109800000FBE84B7877F84BF80916000886180939A
:1098100060001092600078948091660290916702D7
:10982000A0916802B09169029F7E80936602909336
:109830006702A0936802B093690244E050E06EE1D1
:1098400070E086E692E00E94B99629C06DE276E06B
:10985000C8010E942F934091660250916702609167
:10986000680270916902892B21F454FF18C0F894A2
:10987000FFCF54FD03C08CE195E002C089E195E083
:109880009F938F9382E293E09F938F930E94EE9336
:109890000F900F900F900F9002C00E94E425EA8570
:1098A000FB851182108283E02B960FB6F894DEBF01
:1098B0000FBECDBFDF91CF911F910F91FF90EF9021
:1098C000DF90CF90BF90AF909F908F907F906F90E0
:1098D0005F904F903F902F900895CF93DF93EC01CE
:1098E00088819981009741F08530924109F48CC0BC
:1098F0001982188283E093C00E94B236809166027A
:1099000080FD05C081FF01C01D9B0E94E86780911A
:1099100070008C7F809370008091B600806280938D
:10992000B6001092B20082E08093B1008091B60040
:109930008770E1F78091700081608093700061E72B
:109940007EE080E090E00E94B5660E94002780E003
:109950000E94DE288CEE91E19F938F930E94EE93FC
:109960000E9462168091C52C0F900F9086FD0E9478
:109970009F618091C52C9091C62C90FD0E94D423AC
:109980008091C52C87FF06C021E04CE061E080EDAE
:109990000E94426280919C130E94D56A8091650268
:1099A0000E94AE690E94AB698093810A8091650232
:1099B0000E94AE6980919C131F928F938091810ABF
:1099C0001F928F9382E396E09F938F930E94DA9386
:1099D0001092830A1092820A0F900F900F900F90AE
:1099E0000F900F9086E592E090939835809397358D
:1099F00083E290E0909398138093971385E092E12F
:109A00009983888381E00BC06332E1F744EF50E330
:109A100060E070E082E89AE00E942238E3CFDF91B4
:109A2000CF9108950F931F93CF93DF93EC018A0199
:109A300088819981009711F18A31924121F0198230
:109A4000188283E020C06231E9F4A80162E170E08D
:109A500082E89AE00E94223884E080937C3510925C
:109A60007E3510927D351093803500937F354CE71D
:109A700055E362E182E492E00E9485708AE192E11E
:109A80009983888381E0DF91CF911F910F91089591
:109A90008436910514F19F938F9388E896E09F9305
:109AA0008F930E94DA938091CF309091D030A09123
:109AB000D130B091D2300196A11DB11D8093CF302D
:109AC0009093D030A093D130B093D2300F900F90BC
:109AD0000F900F9081E090E0089580E090E008956D
:109AE0002F923F924F925F926F927F928F929F92AE
:109AF000AF92BF92CF92DF92EF92FF920F931F939C
:109B0000CF93DF93CDB7DEB7CC59D1090FB6F89418
:109B1000DEBF0FBECDBFCB56DF4F99838883C559BB
:109B2000D0408A01633871F486E89AE0C456DF4F6A
:109B30006883CC59D0400E94A373C456DF4F68811C
:109B4000CC59D040CB56DF4FA881B981C559D04000
:109B50002D913C91223BB1E13B0711F40C943D5B0C
:109B600040F42115310581F0283D3F4009F43BC404
:109B70002FC4243C41E1340709F409C42B3C314192
:109B800011F40C94455B24C44AE259E061E870E0AA
:109B900086E89AE00E94887388ED9FE0EFC35A013F
:109BA000E3E0F0E0EC0FFD1FE40FF51F1082CA01A7
:109BB0000E94484D892B81F720E030E040E050E0E2
:109BC000CC56DF4F6881C459D040627070E080E0AD
:109BD00090E0A0E00E94D08A09F0A0C6212F287052
:109BE00030E040E050E060E070E080E090E0A0E035
:109BF0000E94D08A99F127E04AE250E06BE270E0DF
:109C000089E290E00E94205E8EE895E30E94F15F79
:109C1000BC01990F880B990B0E94748C20E030E0F6
:109C200048EC52E40E94C08B9F938F937F936F9375
:109C30008CEB96E09F938F931F9287E78F93CE01D3
:109C40008A0D9B1D03969F938F930E944694A80EA6
:109C5000B91E0FB6F894DEBF0FBECDBF212F207105
:109C600030E040E050E060E070E080E090E0A0E0B4
:109C70000E94D08AE9F126E04AE250E06BE270E00F
:109C800089E290E00E94205E81E090E00E946811ED
:109C900080939B1381E09DE10E94F15FBC01990FCD
:109CA000880B990B0E94748C20E030E048EC52E461
:109CB0000E94C08B9F938F937F936F9386EC96E067
:109CC0009F938F931F9287E78F93C501029621E0A0
:109CD00030E02C0F3D1F820F931F9F938F930E94A4
:109CE0004694A80EB91E0FB6F894DEBF0FBECDBFC6
:109CF000C257DF4F2881CE58D04030E040E050E0DE
:109D000060E070E080E090E0A0E00E94D08A01F185
:109D10000E9424119F938F937F936F9381ED96E020
:109D20009F938F931F9287E78F93C5010296A1E0BF
:109D3000B0E0AC0FBD1F8A0F9B1F9F938F930E94B3
:109D40004694A80EB91E0FB6F894DEBF0FBECDBF65
:109D5000212F207430E040E050E060E070E080E0CF
:109D600090E0A0E00E94D08A31F18091CA308F93B8
:109D70008091C9308F938091C8308F938091C73084
:109D80008F938FED96E09F938F931F9287E78F932A
:109D9000C501029621E030E02C0F3D1F820F931F7A
:109DA0009F938F930E944694A80EB91E0FB6F89405
:109DB000DEBF0FBECDBF212F207830E040E050E065
:109DC00060E070E080E090E0A0E00E94D08A41F185
:109DD000F8948091743590917535A0917635B09155
:109DE00077357894BF93AF939F938F938DEE96E0E2
:109DF0009F938F931F9287E78F93C5010296A1E0EF
:109E0000B0E0AC0FBD1F8A0F9B1F9F938F930E94E2
:109E10004694A80EB91E0FB6F894DEBF0FBECDBF94
:109E200020E0302F317040E050E060E070E080E0F2
:109E300090E0A0E00E94D08A09F082C520E0302F97
:109E4000327040E050E060E070E080E090E0A0E040
:109E50000E94D08A09F0F2C520E0302F347040E033
:109E600050E060E070E080E090E0A0E00E94D08AE6
:109E700009F015C620E0302F387040E050E060E077
:109E800070E080E090E0A0E00E94D08A09F036C641
:109E900020E0302F307140E050E060E070E080E082
:109EA00090E0A0E00E94D08A09F0A6C620E0302F02
:109EB000307240E050E060E070E080E090E0A0E0D0
:109EC0000E94D08A09F0C8C620E030E040E050E0AF
:109ED000CC56DF4F6881C459D040647070E080E098
:109EE00090E0A0E00E94D08A09F0E4C620E0C856C5
:109EF000DF4F3881C859D04040E050E060E070E06A
:109F000080E090E0A0E00E94D08A09F040C720E005
:109F1000C756DF4F3881C959D04040E050E060E07B
:109F200070E080E090E0A0E00E94D08A09F05DC778
:109F3000CE56DF4F5881C259D0405170952E20E047
:109F400030E0452F50E060E070E080E090E0A0E07D
:109F50000E94D08A09F077C720E030E0CE56DF4F6C
:109F60004881C259D040427050E060E070E080E02B
:109F700090E0A0E00E94D08A09F098C720E030E08D
:109F8000C657DF4F4881CA58D04050E060E070E0CB
:109F900080E090E0A0E00E94D08A09F0BAC720E0FB
:109FA00030E040E050E0CC56DF4F6881C459D040EB
:109FB000687070E080E090E0A0E00E94D08A09F034
:109FC000D2C720E030E040E050E0CC56DF4F68815F
:109FD000C459D040607170E080E090E0A0E00E9441
:109FE000D08A09F0ECC720E030E0CE56DF4F488140
:109FF000C259D040487050E060E070E080E090E0EE
:10A00000A0E00E94D08A11F00C940B5820E030E0C0
:10A01000CE56DF4F4881C259D040407150E060E0D9
:10A0200070E080E090E0A0E00E94D08A11F00C94F3
:10A030003E5820E030E0CE56DF4F4881C259D04034
:10A04000407250E060E070E080E090E0A0E00E94AC
:10A05000D08A11F00C94715820E030E0CE56DF4FDA
:10A060004881C259D040407450E060E070E080E028
:10A0700090E0A0E00E94D08A11F00C94A458CE5633
:10A08000DF4FF881C259D040F0787F2E20E030E0D9
:10A090004F2F50E060E070E080E090E0A0E00E9490
:10A0A000D08A11F00C94D758CD56DF4F2881C35970
:10A0B000D0402170622E20E030E040E0562D60E07C
:10A0C00070E080E090E0A0E00E94D08A11F40C944F
:10A0D000585B8091C52C82FD02C00C941F5921E071
:10A0E00046E061E083E00E94B01920E030E0472DB7
:10A0F00050E060E070E080E090E0A0E00E94D08A54
:10A1000011F40C941F598091C52C82FF02C00C944D
:10A11000E45820E030E040E0CD56DF4F5881C3598D
:10A12000D040527060E070E080E090E0A0E00E94DB
:10A13000D08A11F00C94545920E030E040E0CD5624
:10A14000DF4F5881C359D040547060E070E080E028
:10A1500090E0A0E00E94D08A11F00C94875920E092
:10A1600030E040E0CD56DF4F5881C359D0405071A8
:10A1700060E070E080E090E0A0E00E94D08A11F002
:10A180000C94BA5920E030E040E0CD56DF4F5881C2
:10A19000C359D040507260E070E080E090E0A0E0F1
:10A1A0000E94D08A11F00C94F95920E030E040E090
:10A1B000CD56DF4F5881C359D040507460E070E0F5
:10A1C00080E090E0A0E00E94D08A11F00C94385A10
:10A1D00020E030E040E0CD56DF4F5881C359D040F9
:10A1E000587060E070E080E090E0A0E00E94D08ACB
:10A1F00011F00C94775A20E030E040E0C656DF4F73
:10A200005881CA59D04060E070E080E090E0A0E062
:10A210000E94D08A11F00C94A85A20E030E0492D19
:10A2200050E060E070E080E090E0A0E00E94D08A22
:10A2300011F00C94DF5A212F302FCE56DF4F48817A
:10A24000C259D040CD56DF4F5881C359D040CC566B
:10A25000DF4F6881C459D0407D2DC956DF4F8881BA
:10A26000C759D0409C2DA0E00E94D08A11F00C94D8
:10A27000EA5A809164028061898380917A0A8A8394
:10A28000FE01EA0DFB1D138280919F139091A01394
:10A29000A091A113B091A21385010D5F1F4F80FF04
:10A2A0000CC01F930F938DE898E09F938F930E94AB
:10A2B000DA930F900F900F900F90B801CE01019696
:10A2C0000E9492758091660282FF0AC024E731E302
:10A2D000A801BE016F5F7F4F8EE692E00E9405618C
:10A2E00080919F139091A013A091A113B091A213FC
:10A2F00082FD73980E94B26886E89AE00E94A57376
:10A300008091660290916702A0916802B091690203
:10A3100090FD02C00C94215B3FEFA31AB30A0E9488
:10A32000AB69F82E89E10E94C36980916602909121
:10A330006702A0916802B091690290FD02C00C947E
:10A340001D5B739880917A0A8F5F80937A0A8A8363
:10A35000B5016F5F7F4FCE0101960E94927586E82E
:10A360009AE00E94A57340E050E065E88091E11416
:10A370009091E2140E94857082EB91E1CB56DF4F01
:10A38000A881B981C559D0408D939C931EC08EE69B
:10A390009AE00E94136F892BC1F00E94B2688091ED
:10A3A000660287FD2B9840E450E060E070E08EE6A6
:10A3B0009AE00E94F56E8BEC91E1CB56DF4FE8817D
:10A3C000F981C559D0409183808381E00C94685B0A
:10A3D000CB56DF4FA881B981C559D0401D921C9240
:10A3E00083E00C94685B623181F780906602909004
:10A3F0006702A0906802B090690291FCCDCBF80191
:10A400008081813021F50180F281E02D1081018170
:10A410002281CE56DF4F2883C259D0403381CD569A
:10A42000DF4F3883C359D0404481CC56DF4F488337
:10A43000C459D040D5805681C956DF4F5883C7597B
:10A44000D040C780E084F184212C312C52C082306E
:10A45000B9F423803480E12CF12C11E000E0CE56D9
:10A46000DF4F1882C259D040B0E8CD56DF4FB883D5
:10A47000C359D040CC56DF4F1882C459D04032C0A7
:10A480008330D1F0843009F087CBE12CF12C212CE2
:10A49000312C15E000E0CE56DF4F1882C259D04073
:10A4A000CD56DF4F1882C359D040E2E0CC56DF4F83
:10A4B000E883C459D04016C0E12CF12C212C312C5A
:10A4C00015E000E0CE56DF4F1882C259D040CD567D
:10A4D000DF4F1882C359D040F1E0CC56DF4FF883EC
:10A4E000C459D040D12CC956DF4F1882C759D0402B
:10A4F000C12C4090C7305090C8306090C9307090E7
:10A50000CA3020918D0230918E0240918F0250917D
:10A510009002C657DF4F288339834A835B83CA582A
:10A52000D0402DEC3CEC4CE45EE3C657DF4F688135
:10A5300079818A819B81CA58D0400E94DD8A9B0123
:10A54000AC01C301B2010E94998D87FD0BC0E89454
:10A55000A0F88092660290926702A0926802B09280
:10A56000690246C0C657DF4F288139814A815B8125
:10A57000CA58D040C301B2010E94BB8B87FF38C0CC
:10A580008091D3309091D430A091D530B091D63015
:10A590000196A11DB11D8093D3309093D430A09328
:10A5A000D530B093D630A0FCF7CA6894A0F880925A
:10A5B000660290926702A0926802B092690215E466
:10A5C00000E2CE56DF4F1882C259D040CD56DF4F41
:10A5D0001882C359D04034E0CC56DF4F3883C45979
:10A5E000D040D12CC956DF4F1882C759D040C12C5A
:10A5F000CE56DF4F4881C259D0404470C657DF4F16
:10A600004883CA58D04020E030E050E060E070E07D
:10A6100080E090E0A0E00E94D08A09F08C9A512F4F
:10A620005072C257DF4F5883CE58D040252F30E0AC
:10A6300040E050E060E070E080E090E0A0E00E9448
:10A64000D08A11F00E942411802F8074C856DF4FE9
:10A650008883C859D04020E0382F40E050E060E0C7
:10A6600070E080E090E0A0E00E94D08A11F00E94AB
:10A670004625902F9078C756DF4F9883C959D04010
:10A6800020E0392F40E050E060E070E080E090E0B2
:10A69000A0E00E94D08A51F00E94BF1060938135E3
:10A6A000709382358093833590938435212F217068
:10A6B00030E040E050E060E070E080E090E0A0E05A
:10A6C0000E94D08AF1F08FE89CE19F938F938CE9F0
:10A6D00096E09F938F931F9287E78F93CE01039607
:10A6E0009F938F930E9446944C010E94484D0FB651
:10A6F000F894DEBF0FBECDBF892B09F04DCA5401BF
:10A7000002C0A12CB12C212F227030E040E050E09B
:10A7100060E070E080E090E0A0E00E94D08AD1F19B
:10A72000C501029664EA76E0E1E0F0E0EC0FFD1F7F
:10A730008E0F9F1F0E943893F3E0AF0EB11C2EE8DE
:10A74000622E25E3722E36E7832E33E0932E47E701
:10A75000542ED3018D913D011F928F939F928F9222
:10A760001F925F92C5010296E1E0F0E0EC0FFD1F41
:10A770008E0F9F1F9F938F930E944694A80EB91E21
:10A780000FB6F894DEBF0FBECDBF36E9631635E3D2
:10A790007306F9F6212F247030E040E050E060E0CD
:10A7A00070E080E090E0A0E00E94D08A09F450C000
:10A7B000C501029668EA76E041E050E04C0F5D1F6B
:10A7C000840F951F0E94389354E0A50EB11C2E01F2
:10A7D0008AE7480E511C80E1D2011D928A95E9F763
:10A7E00028E0A20168E980EB0E94FB173201B8E083
:10A7F0006B0E711C96E7892E93E0992E27E7F201E4
:10A8000081912F011F928F939F928F921F922F936E
:10A81000C501029641E050E04C0F5D1F840F951F6B
:10A820009F938F93C556DF4F2883CB59D0400E940A
:10A830004694A80EB91E0FB6F894DEBF0FBECDBF6A
:10A84000C556DF4F2881CB59D04046145704B9F67E
:10A85000CD56DF4F9881C359D0409078C656DF4F10
:10A860009883CA59D04020E030E040E0592F60E0A2
:10A8700070E080E090E0A0E00E94D08AE1F4809156
:10A880009D1390919E139F938F938DEA96E09F93D3
:10A890008F931F9287E78F93CE018A0D9B1D03969E
:10A8A0009F938F930E944694A80EB91E0FB6F894FA
:10A8B000DEBF0FBECDBF20E030E040E050E0CC5620
:10A8C000DF4F6881C459D040617070E080E090E053
:10A8D000A0E00E94D08A09F46FC9E3E0F0E0EC0F39
:10A8E000FD1FEA0DFB1D80E28083A50183E090E05F
:10A8F0008A199B09FC01E40FF51FEC50FF4C2081E5
:10A900004F5F5F4F222309F44AC92081E1E0F0E064
:10A91000EC0FFD1FE40FF51F2283ECCFCE018A0D53
:10A920009B1D64EB76E003960E943893B7E0AB0E74
:10A93000B11CC5010E94484D892B09F02DC94EC993
:10A94000E114F10409F47ACAF894409074355090F7
:10A950007535609076357090773578948091F91CD4
:10A960009091FA1CA091FB1CB091FC1CA3019201D8
:10A97000281B390B4A0B5B0BCA01B9010E94728C70
:10A98000C257DF4F688379838A839B83CE58D04038
:10A99000B70180E090E00E94728C9B01AC01C2572D
:10A9A000DF4F688179818A819B81CE58D0400E9497
:10A9B000C08B4C019F928F937F936F9388EF96E0AB
:10A9C0009F938F931F9287E78F939E012A0D3B1DC4
:10A9D0002D5F3F4F3F932F93C456DF4F6883CC5971
:10A9E000D040C556DF4F7883CB59D0400E94469463
:10A9F000A80EB91EC456DF4F6881CC59D040C55649
:10AA0000DF4F7881CB59D040862F972FA82DB92DB5
:10AA10008093863590938735A0938835B093893598
:10AA20004092F91C5092FA1C6092FB1C7092FC1C24
:10AA30000FB6F894DEBF0FBECDBF00CAE114F1041B
:10AA400009F40ACAF8948091D01C9091D11CA0916D
:10AA5000D21CB091D31C78949F938F9380916D02F8
:10AA60008F9380916C028F9385E097E09F938F93F3
:10AA70001F9287E78F93C5010296A1E0B0E0AC0F6B
:10AA8000BD1F8A0F9B1F9F938F930E944694A80E11
:10AA9000B91E0FB6F894DEBF0FBECDBFDDC9F89466
:10AAA0008091783590917935A0917A35B0917B3548
:10AAB0007894BF93AF939F938F9385E197E09F9393
:10AAC0008F931F9287E78F93C501029621E030E0B4
:10AAD0002C0F3D1F820F931F9F938F930E944694CC
:10AAE000A80EB91EC5010E94484D0FB6F894DEBFEE
:10AAF0000FBECDBF892B09F04FC8BCC9E114F104CA
:10AB000009F4C6C9F8944090783550907935609032
:10AB10007A3570907B3578948091FD1C9091FE1C65
:10AB2000A091FF1CB091001DA3019201281B390BBD
:10AB30004A0B5B0BCA01B9010E94728CC257DF4FEE
:10AB4000688379838A839B83CE58D040B70180E0A5
:10AB500090E00E94728C9B01AC01C257DF4F68816C
:10AB600079818A819B81CE58D0400E94C08B4C0154
:10AB70009F928F937F936F9380E297E09F938F9341
:10AB80001F9287E78F939E012A0D3B1D2D5F3F4F3C
:10AB90003F932F93C456DF4F6883CC59D040C5569E
:10ABA000DF4F7883CB59D0400E944694A80EB91E3F
:10ABB000C456DF4F6881CC59D040C556DF4F7881ED
:10ABC000CB59D040862F972FA82DB92D80938A3549
:10ABD00090938B35A0938C35B0938D354092FD1CAE
:10ABE0005092FE1C6092FF1C7092001D0FB6F894EC
:10ABF000DEBF0FBECDBF4CC9EF2809F457C9F8948A
:10AC00008091D41C9091D51CA091D61CB091D71CDA
:10AC100078949F938F9380916B028F9380916A02B7
:10AC20008F938DE297E09F938F931F9287E78F9387
:10AC3000C5010296A1E0B0E0AC0FBD1F8A0F9B1FBB
:10AC40009F938F930E944694A80EB91E0FB6F89456
:10AC5000DEBF0FBECDBF2AC98091CB309091CC30E2
:10AC6000A091CD30B091CE30BF93AF939F938F938F
:10AC70008DE397E09F938F931F9287E78F93C50192
:10AC8000029621E030E02C0F3D1F820F931F9F930F
:10AC90008F930E944694A80EB91EC5010E94484D8C
:10ACA0000FB6F894DEBF0FBECDBF892B11F00C9408
:10ACB000CC4D0AC98091D6308F938091D5308F9337
:10ACC0008091D4308F938091D3308F938091D23004
:10ACD0008F938091D1308F938091D0308F938091DA
:10ACE000CF308F9388E497E09F938F931F9287E7ED
:10ACF000982E9F92C5010296A1E0B0E0AC0FBD1F57
:10AD00008A0F9B1F9F938F930E944694A80EB91E93
:10AD1000C5010E94484D0FB6F894DEBF0FBECDBFEF
:10AD2000892B11F00C94CC4D8091C52C9091C62CA0
:10AD300090FFDCC88091DA308F938091D9308F9367
:10AD40008091D8308F938091D7308F938CE697E0A5
:10AD50009F938F931F929F92C501029621E030E04E
:10AD60002C0F3D1F820F931F9F938F930E94469439
:10AD7000A80EB91EC5010E94484D0FB6F894DEBF5B
:10AD80000FBECDBF892B11F00C94CC4DAFC8809174
:10AD9000BC288F938091BB288F938091BA288F9382
:10ADA0008091B9288F938EE797E09F938F931F929E
:10ADB00087E78F93C5010296A1E0B0E0AC0FBD1FFD
:10ADC0008A0F9B1F9F938F930E944694A80EB91ED3
:10ADD000C5010E94484D0FB6F894DEBF0FBECDBF2F
:10ADE000892B11F00C94CC4D92C8809184358F93AF
:10ADF000809183358F93809182358F9380918135B7
:10AE00008F9389E897E09F938F931F9287E78F93A3
:10AE1000C501029621E030E02C0F3D1F820F931FE9
:10AE20009F938F930E944694A80EB91EC5010E945D
:10AE3000484D0FB6F894DEBF0FBECDBF892B11F081
:10AE40000C94CC4D75C881E00E9471102091850250
:10AE50003091860240918702509188020E946C8E48
:10AE60009F938F937F936F9386E997E09F938F9340
:10AE70001F9287E78F93C5010296A1E0B0E0AC0F67
:10AE8000BD1F8A0F9B1F9F938F930E944694A80E0D
:10AE9000B91EC5010E94484D0FB6F894DEBF0FBE23
:10AEA000CDBF892B11F00C94CC4D56C882E00E9486
:10AEB0007110209181023091820240918302509161
:10AEC00084020E946C8E9F938F937F936F9383EA8B
:10AED00097E09F938F931F9287E78F93C501029608
:10AEE00021E030E02C0F3D1F820F931F9F938F9323
:10AEF0000E944694A80EB91EC5010E94484D0FB687
:10AF0000F894DEBF0FBECDBF892B11F00C94CC4D51
:10AF100035C883E00E9471109F938F937F936F9346
:10AF200080EB97E09F938F931F9287E78F93C501E4
:10AF30000296A1E0B0E0AC0FBD1F8A0F9B1F9F934C
:10AF40008F930E944694A80EB91E8C98C5010E944A
:10AF5000484D0FB6F894DEBF0FBECDBF892B11F060
:10AF60000C94CC4D1CC8299903C08CE195E002C01B
:10AF700089E195E09F938F938DEB97E09F938F935B
:10AF80001F9287E78F93C501029621E030E02C0FD6
:10AF90003D1F820F931F9F938F930E944694A80E8C
:10AFA000B91EC5010E94484D0FB6F894DEBF0FBE12
:10AFB000CDBF892B11F00C94CC4D0C94E14F2A9904
:10AFC00003C08CE195E002C089E195E09F938F93E7
:10AFD00085EC97E09F938F931F9287E78F93C5012E
:10AFE0000296A1E0B0E0AC0FBD1F8A0F9B1F9F939C
:10AFF0008F930E944694A80EB91EC5010E94484D29
:10B000000FB6F894DEBF0FBECDBF892B11F00C94A4
:10B01000CC4D0C94F34F8091C52C87FD02C00C944D
:10B02000065021E042E161E080ED0E9442629F9380
:10B030008F937F936F938DEC97E09F938F931F92E5
:10B0400087E78F93C501029621E030E02C0F3D1F6A
:10B05000820F931F9F938F930E944694A80EB91E50
:10B06000C5010E94484D0FB6F894DEBF0FBECDBF9C
:10B07000892B11F00C94CC4D0C9406508091C52C6A
:10B0800087FD02C00C94195021E042E162E080ED9E
:10B090000E9442629F938F937F936F938BED97E013
:10B0A0009F938F931F9287E78F93C5010296A1E02C
:10B0B000B0E0AC0FBD1F8A0F9B1F9F938F930E9420
:10B0C0004694A80EB91EC5010E94484D0FB6F894CB
:10B0D000DEBF0FBECDBF892B11F00C94CC4D0C946C
:10B0E00019508091C52C87FD02C00C942C5021E092
:10B0F00042E163E080ED0E9442629F938F937F93D1
:10B100006F9389EE97E09F938F931F9287E78F93BA
:10B11000C501029621E030E02C0F3D1F820F931FE6
:10B120009F938F930E944694A80EB91EC5010E945A
:10B13000484D0FB6F894DEBF0FBECDBF892B11F07E
:10B140000C94CC4D0C942C508091C52C87FD02C0E2
:10B150000C943F5021E042E164E080ED0E944262A5
:10B160009F938F937F936F9387EF97E09F938F9336
:10B170001F9287E78F93C5010296A1E0B0E0AC0F64
:10B18000BD1F8A0F9B1F9F938F930E944694A80E0A
:10B19000B91EC5010E94484D0FB6F894DEBF0FBE20
:10B1A000CDBF892B11F00C94CC4D0C943F50809165
:10B1B000C52C82FD02C00C94545046E061E083E04F
:10B1C0000E94B0190C9454508091A81D8F938091C7
:10B1D000A71D8F938091A61D8F938091A51D8F939E
:10B1E00085E098E09F938F931F9287E78F93C50127
:10B1F000029641E050E04C0F5D1F840F951F9F9316
:10B200008F930E944694A80EB91EC5010E94484D16
:10B210000FB6F894DEBF0FBECDBF892B11F00C9492
:10B22000CC4D20E030E040E0562D60E070E080E062
:10B2300090E0A0E00E94D08A11F40C948950809193
:10B24000C52C82FD02C00C9489508091AC1D8F9357
:10B250008091AB1D8F938091AA1D8F938091A91D22
:10B260008F938DE098E09F938F931F9287E78F9342
:10B27000C5010296E1E0F0E0EC0FFD1F8E0F9F1F6D
:10B280009F938F930E944694A80EB91EC5010E94F9
:10B29000484D0FB6F894DEBF0FBECDBF892B11F01D
:10B2A0000C94CC4D0C9489508091C52C9091C62C57
:10B2B00090FD02C00C949C5080E090E00E94BE245F
:10B2C0009F938F937F936F9388E198E09F938F93E1
:10B2D0001F9287E78F93C501029641E050E04C0F23
:10B2E0005D1F840F951F9F938F930E944694A80E15
:10B2F000B91EC5010E94484D0FB6F894DEBF0FBEBF
:10B30000CDBF892B11F00C94CC4D0C949C508091A6
:10B31000C52C9091C62C90FD02C00C94AF5081E0DA
:10B3200090E00E94BE249F938F937F936F9388E257
:10B3300098E09F938F931F9287E78F93C5010296A2
:10B34000E1E0F0E0EC0FFD1F8E0F9F1F9F938F93A6
:10B350000E944694A80EB91EC5010E94484D0FB622
:10B36000F894DEBF0FBECDBF892B11F00C94CC4DED
:10B370000C94AF508091C52C9091C62C90FD02C0CA
:10B380000C94C25081E090E00E94BE242B013C014D
:10B3900080E090E00E94BE249B01AC01C301B20199
:10B3A0000E94BB229F938F937F936F9389E398E0D2
:10B3B0009F938F931F9287E78F93C501029641E079
:10B3C00050E04C0F5D1F840F951F9F938F930E9439
:10B3D0004694A80EB91EC5010E94484D0FB6F894B8
:10B3E000DEBF0FBECDBF892B11F00C94CC4D0C9459
:10B3F000C2508091C52C9091C62C90FD02C00C9437
:10B40000D55081E090E00E94BE242B013C0180E0F9
:10B4100090E00E94BE249B01AC01C301B2010E94D6
:10B420001C239F938F937F936F9384E498E09F9363
:10B430008F931F9287E78F93C5010296E1E0F0E0BA
:10B44000EC0FFD1F8E0F9F1F9F938F930E944694BA
:10B45000A80EB91EC5010E94484D0FB6F894DEBF74
:10B460000FBECDBF892B11F00C94CC4D0C94D55050
:10B470008091C52C9091C62C90FD02C00C94E85090
:10B4800081E090E00E94BE242B013C0180E090E02E
:10B490000E94BE249B01AC01C301B2010E947D2326
:10B4A0009F938F937F936F9382E598E09F938F9301
:10B4B0001F9287E78F93C501029641E050E04C0F41
:10B4C0005D1F840F951F9F938F930E944694A80E33
:10B4D000B91EC5010E94484D0FB6F894DEBF0FBEDD
:10B4E000CDBF892B11F00C94CC4D0C94E850809179
:10B4F000C52C9091C62C91FD02C00C94FB500E946B
:10B50000151E9F938F937F936F9385E698E09F938B
:10B510008F931F9287E78F93C5010296E1E0F0E0D9
:10B52000EC0FFD1F8E0F9F1F9F938F930E944694D9
:10B53000A80EB91EC5010E94484D0FB6F894DEBF93
:10B540000FBECDBF892B11F00C94CC4D0C94FB5049
:10B55000D10116968C9116971F928F9315968C9108
:10B5600015971F928F9313968C9113971F928F9319
:10B5700012968C911F928F9386E798E09F938F93FA
:10B580001F9287E78F93C5010296E1E0F0E0EC0F90
:10B59000FD1F8E0F9F1F9F938F930E944694A80EAE
:10B5A000B91EC5010E94484D0FB6F894DEBF0FBE0C
:10B5B000CDBF892B11F00C94CC4D0C940D51779A82
:10B5C00080919F139091A013A091A113B091A21309
:10B5D00092FD749A80919F139091A013A091A11352
:10B5E000B091A21382FD0CC08091660280FD08C05C
:10B5F00081FD02C00C9439511D9902C00C9439513F
:10B6000040E050E060E070E0CE0101960E94DC0E68
:10B610008091AE1D90E02091951330919613821782
:10B62000930710F40C94395140E050E062E180E15E
:10B6300092E00E9485700C9439518F2D0E94C3694D
:10B64000739A80919D1390919E13892B11F00E9403
:10B65000E86780917A0A8F5F80937A0A80919F13BE
:10B660009091A013A091A113B091A21382FD02C0EA
:10B670000C94CC4D739A0C94CC4D653811F00C940D
:10B68000E551A12CB12C0C9495518EE69AE00E94C4
:10B69000136F892B11F40C94E5510E94E867809197
:10B6A000660287FD02C00C94CC4D2B9A0C94CC4DB5
:10B6B00020E030E0472D50E060E070E080E090E076
:10B6C000A0E00E94D08A11F00C9483500C94895011
:10B6D000C456DF4F0FB6F894DEBF0FBECDBFDF916B
:10B6E000CF911F910F91FF90EF90DF90CF90BF907F
:10B6F000AF909F908F907F906F905F904F903F9012
:10B700002F9008950C943B734F925F926F927F92AB
:10B710009F92AF92BF92CF92DF92EF92FF920F93E0
:10B720001F93CF93DF93CDB7DEB760970FB6F89432
:10B73000DEBF0FBECDBF5B010E94AB69E82FF0E01A
:10B74000EE0FFF1FEE53F34E80819181019691839E
:10B75000808380919F139091A013A091A113B09129
:10B76000A21381FD74984090660250906702609029
:10B770006802709069020E94EE746C01FC01808185
:10B78000982F92959F70913099F48F7051F4809119
:10B79000A61C9091A71C01969093A71C8093A61CB1
:10B7A0003CC1B50183EA97E30E94A774892B51F04D
:10B7B0008091A41C9091A51C01969093A51C809348
:10B7C000A41C2BC1D301C2013EE0B695A795979565
:10B7D00087953A95D1F7F82FF1709F2E81E99AE07D
:10B7E0000E945E717C01892B09F44BC0B501C70131
:10B7F00002960E94A774892B09F43FC087012BE8A9
:10B800003EE040E054E660E070E0C7010F960E9421
:10B81000936DF6019181F7018481981321C082858F
:10B820008F5F82878091A21C9091A31C01969093B8
:10B83000A31C8093A21C84E00E94DE75F701208582
:10B8400030E02817390708F078C184E00E94DE75DF
:10B85000F7018087F60180818F70F7018187DDC055
:10B86000F701128684E00E94DE75F7018087F601F9
:10B8700080818F70F701818761C1C7010E94C37108
:10B88000B1CF88E092E00E94EA717C01892B09F433
:10B89000C4C0B501C70102960E94A074F60181815F
:10B8A0008150F701848380E091E0A0E0B0E08387DD
:10B8B0009487A587B687128684E00E94DE75F7011B
:10B8C0008087F60180818F70F7018187B70181E958
:10B8D0009AE00E949D7187012BE83EE040E054E62B
:10B8E00060E070E0C7010F960E94936D11E0F601D1
:10B8F0008181F7018483F60180818F70F70187834E
:10B9000084E00E94DE75F701858383E00E94DE7586
:10B91000F701868387818F3009F010E0F6014180BE
:10B92000F7018481481A512C612C712C86E0440C5B
:10B93000551C661C771C8A95D1F72385348545856F
:10B940005685A0ECB0E00E940489BB27A92F982F50
:10B95000872F480E591E6A1E7B1E438654866586B5
:10B960007686A501B701C6010E94DC0E8091AE1D4E
:10B9700090E020919513309196138217930738F039
:10B9800040E050E062E180E192E00E9485708091A9
:10B99000951390919613029708F44BC08091C52C93
:10B9A00086FF2AC00E949161C60105960E945D61D2
:10B9B000F60181811F928F93F70186811F928F93E9
:10B9C00085811F928F938EE998E09F938F931F92AA
:10B9D00080E18F93CE0101965C019F938F930E942B
:10B9E000469482E00E947761C5010E945D610FB6B6
:10B9F000F894DEBF0FBECDBF8091660290916702C2
:10BA0000A0916802B091690297FD4DC08091951395
:10BA100090919613029708F47AC080919F139091A9
:10BA2000A013A091A113B091A21381FF89C0749AB1
:10BA300087C08091660290916702A0916802B091E0
:10BA4000690296FFABCF992009F4A8CFF601808157
:10BA5000982F9F709230E8F09150807F892B8083DF
:10BA600086E89AE00E94825B8091A01C9091A11CC4
:10BA700001969093A11C8093A01C80919F1390919C
:10BA8000A013A091A113B091A21396FF87CF739832
:10BA900085CF8091A61C9091A71C01969093A71C1E
:10BAA0008093A61C7BCF8FE89CE120918F1C2223E2
:10BAB00009F4ACCF9F938F9381EB98E09F938F9382
:10BAC000CE0101963C019F938F930E9483945C0169
:10BAD000B301C60102960E9459930F900F900F90E8
:10BAE0000F900F900F90009709F490CFEFEFAE1AE0
:10BAF000BE0A8A0D9B1DAC010196FA0120812032FD
:10BB0000D1F362E18AE192E00E9485707FCF112338
:10BB100009F483CF82E08093E0301092E2301092FB
:10BB2000E130F092E430E092E33040EE50E362E145
:10BB300082E492E00E94857070CF912C10E0D7CE05
:10BB400060960FB6F894DEBF0FBECDBFDF91CF91E8
:10BB50001F910F91FF90EF90DF90CF90BF90AF902B
:10BB60009F907F906F905F904F9008958115910501
:10BB700011F00197F1F70895E091A135F091A23508
:10BB800090818091A03589230895E0919E35F091B0
:10BB90009F3590818091A035892B8083E091A335DA
:10BBA000F091A43590818091A035892B80830895F0
:10BBB0001F93CF93DF93E0919E35F0919F35908155
:10BBC0008091A035809589238083E091A335F09101
:10BBD000A43590818091A035892B80838FE897E0F0
:10BBE0000E94B65D1FB7F894E091A335F091A4359B
:10BBF00090818091A03580958923808389E091E0B0
:10BC00000E94B65DE091A135F091A235D081C0913E
:10BC1000A0351FBF789485E896E00E94B65DE0915C
:10BC2000A135F091A23580819091A035982319F02B
:10BC30008D2F8C2301C081E0DF91CF911F9108955A
:10BC40005093A4354093A33570939F3560939E35F0
:10BC50009093A2358093A13581E001C0880F2A9589
:10BC6000EAF78093A0350C94D85DCF93DF93C82F6B
:10BC7000DFB7F894E091A335F091A43590818091DD
:10BC8000A035892B808387E090E00E94B65DCC23AD
:10BC900051F0E091A335F091A43590818091A035C9
:10BCA00080958923808384E390E00E94B65DE091D3
:10BCB000A135F091A23590818091A035892309F4B6
:10BCC000C0E085EB90E00E94B65DE091A335F09175
:10BCD000A43590818091A035809589238083DFBF32
:10BCE00088E790E00E94B65D8C2FDF91CF91089598
:10BCF000CF93DF93C82FD8E08C2F81700E94355EE0
:10BD0000C6958111C068D150B9F78C2FDF91CF91C2
:10BD100008958FEF0C94785EDF92EF92FF920F936D
:10BD20001F93CF93DF93E82E8B010E94D85D811182
:10BD300035C080EF0E94785ED0E0C0E488EFD82E56
:10BD4000DC0E81E00E94355EF82E81E00E94355EB7
:10BD5000882319F0FF2071F023C0F1100BC0CE151D
:10BD600030F0F801808180FF05C0EC1619F0DC2F5F
:10BD7000FF24F3948F2D0E94355EF80190819695F3
:10BD8000FF2011F09068F8019083C150CD11D9CFF8
:10BD90000F5F1F4FC111D2CF8D2F03C08FEF01C096
:10BDA0008EEFDF91CF911F910F91FF90EF90DF9079
:10BDB0000895EF92FF921F93CF93DF93182FEB011B
:10BDC0000E94D85D209771F085E50E94785E7E0123
:10BDD00088E0E80EF11C89910E94785ECE15DF059F
:10BDE000D1F703C08CEC0E94785E812FDF91CF9158
:10BDF0001F91FF90EF900C94785E0F931F93CF9359
:10BE0000DF93DB01EC9111969C911197F0E0F92BF7
:10BE1000803179F4EE7F63E0EE0FFF1F6A95E1F762
:10BE200016969C9116976CE070E0691B7109E60FFD
:10BE3000F71FF7FF07C091E0EA019883F195E195BC
:10BE4000F10902C0EA011882883279F414968C91C3
:10BE5000982F9076903649F086FF02C0EE7F05C09D
:10BE600085FF02C0EC7F01C0E87FCF0144E09695DA
:10BE700087954A95E1F7D9018C93EF70E801E88343
:10BE800080E0DF91CF911F910F9108950F931F9341
:10BE9000CF93DF93EC018B01B80188810E948C5E07
:10BEA00088839FEF980F9D3F30F4F801908198327E
:10BEB00011F0903189F7DF91CF911F910F91089583
:10BEC000CF93DF93EC010E94D85DBE0184EB0E940A
:10BED000D95E81E00E94355EC82F0E94D85D81E066
:10BEE000C11101C080E0DF91CF9108951F93CF93DE
:10BEF000DF931F921F92CDB7DEB7182F69837A8325
:10BF00000E94D85D0E94BC5D69817A81882341F0DE
:10BF100084E40E94D95E113029F00E94C55D02C000
:10BF200082E001C080E00F900F90DF91CF911F91D0
:10BF300008955F926F927F928F929F92AF92BF927D
:10BF4000CF92DF92EF92FF920F931F93CF93DF93E5
:10BF5000CDB7DEB729970FB6F894DEBF0FBECDBFC1
:10BF60005C014B013A0189010E94D85DB5018EEB5D
:10BF70000E94D95ECE0101967C016C0199E0592E98
:10BF80005E0C0E94895EF60181936F015E12F9CF0B
:10BF900069E070E0C7010E947D79D82E811108C048
:10BFA0009301A401B701F50180810E94FD5E02C0EA
:10BFB00083E0D82E8D2D29960FB6F894DEBF0FBEE4
:10BFC000CDBFDF91CF911F910F91FF90EF90DF9048
:10BFD000CF90BF90AF909F908F907F906F905F9029
:10BFE00008950F931F93CF93DF93CDB7DEB72B97B1
:10BFF0000FB6F894DEBF0FBECDBF182F092F682FE4
:10C00000792F88E0810F0E94765F882319F084E3FE
:10C0100091E243C06CE872E88EE190E00E945860C3
:10C020009E01275F3F4FAE01465F5F4FBE01655FD8
:10C030007F4F812F902F0E94995F8111E8CF88E078
:10C04000E1EEF2E0DE01119601900D928A95E1F7A2
:10C05000298541E752E0249FC001259F900D1124BE
:10C0600064E670E00E9489888A8594E6899F600D65
:10C07000711D1124FE01319688E08E0F91912913D4
:10C0800003C06F5F7F4F02C08E13F8CF8B8588236C
:10C0900019F0719561957109CB012B960FB6F89443
:10C0A000DEBF0FBECDBFDF91CF911F910F910895DD
:10C0B000DC01CB0181159105A105B10529F0815065
:10C0C0009040A040B040D9F708959B01AC01109278
:10C0D000B90060E074E284EF90E00E949D88DA018C
:10C0E000C9014097A109B109B695A795979587957C
:10C0F0008093B800089594EA9093BC0040EA56E813
:10C1000061E070E09091BC0097FD07C0415051097B
:10C1100061097109B9F781E008959091B900987F9C
:10C12000983011F09031B9F78093BB0084E8809388
:10C13000BC0080EA96E8A1E0B0E02091BC0027FDB9
:10C1400005C00197A109B109C1F7E5CF8091B900F8
:10C15000887F883111F08034F1F680E0089524EA78
:10C1600034E844E92093BC009091BC0097FFFCCFD9
:10C170009091B900987F983011F0903199F78093A1
:10C18000BB003093BC009091BC0097FFFCCF909116
:10C19000B900987F903211F0983539F44093BC0083
:10C1A0009091BC0094FDFCCFDDCF08950C947B6092
:10C1B00084E98093BC008091BC0084FDFCCF08958D
:10C1C0008093BB0084E88093BC008091BC0087FF13
:10C1D000FCCF9091B900987F81E0983209F480E01B
:10C1E000089584EC8093BC008091BC0087FFFCCF55
:10C1F0008091BB00089584E88093BC008091BC00CE
:10C2000087FFFCCF8091BB000895CF93DF93FC01A3
:10C210007096EC01A991CE01A0933F01CE17DF07E4
:10C22000C1F780913C018F7D80933C0180913C015E
:10C23000877F80933C01DB015096FB0181918093C5
:10C240003E01EA17FB07D1F780913C01806880939B
:10C250003C0180913D0180FFFCCF4051510980910C
:10C260003C01806280933C0180913C01877F8093F8
:10C270003C01141615069CF4FB01819180933E014C
:10C28000EA17FB07D1F780913C01806880933C015D
:10C2900080913D0180FFFCCF40515109EACFF90167
:10C2A000C901409620913E012193E817F907D1F783
:10C2B00081E090E0DF91CF9108950F931F93CF938A
:10C2C000DF93EC018CE70E94AF608CE70E94E06096
:10C2D0008E01005F1F4F89910E94E060C017D10757
:10C2E000D1F7DF91CF911F910F910C94D8608130DD
:10C2F00019F440E050E002C040EC50E060E070E033
:10C300008CE790E00C94E317813019F44EE050E094
:10C3100002C048E050E060E070E08CE790E00C94F0
:10C32000E31741E050E060E070E08CE790E00E94AD
:10C33000E31764ED74E180E090E00C94586048E30A
:10C3400050E060E070E08CE790E00E94E31749E382
:10C3500050E060E070E08CE790E00E94E31744E179
:10C3600050E060E070E08CE790E00E94E31748E75F
:10C3700050E060E070E08CE790E00E94E3174EE54B
:10C3800050E060E070E08CE790E00E94E3174DE63B
:10C3900050E060E070E08CE790E00E94E31768E313
:10C3A00074E38CE090E00E9458604CE050E060E064
:10C3B00070E08CE790E00E94E31741E050E060E01D
:10C3C00070E08CE790E00E94E31746E050E060E008
:10C3D00070E08CE790E00E94E31764ED74E180E088
:10C3E00090E00C945860CF93DF93CDB7DEB7A2975F
:10C3F0000FB6F894DEBF0FBECDBF81E1E0E4F9E0F7
:10C40000DE01529601900D928A95E1F781E1E1E516
:10C41000F9E0DE01119601900D928A95E1F70E94F4
:10C420009F61CE0142960E945D6182E00E94776129
:10C4300064ED74E180E090E00E945860CE010196C6
:10C440000E945D6160E27CE581E590E00E945860B9
:10C4500080E00E94846160E27CE581E590E00E94DA
:10C4600058604EE050E060E070E08CE790E00E94A1
:10C47000E317A2960FB6F894DEBF0FBECDBFDF91D3
:10C48000CF910895CF92DF92EF92FF920F931F9377
:10C49000CF93DF9300D0CDB7DEB7042F122F21301A
:10C4A00061F0223031F0243031F0283031F493E063
:10C4B00005C091E003C092E001C090E0E82FF0E0F9
:10C4C0008160F82E0C3009F4E0C00E3011F4946055
:10C4D000DCC0003111F49860D8C0023109F0D5C039
:10C4E000613009F4B7C09C60623011F4906207C0FB
:10C4F000633011F4906403C0643009F4906690686E
:10C50000692F70E023E030E0AE014F5F5F4FCF0155
:10C510000E94FB1762E174E380E090E00E945860A3
:10C520008F2D0E947B600E94F16089830E94F160E0
:10C530008A83023119F40E94F1608B830E94F160BA
:10C5400087FDF1CF0E94FB600E94D86062E174E336
:10C5500080E090E00E9458608F2D0E947B600E94D6
:10C56000F16089830E94F1608A83023119F40E948C
:10C57000FB608B830E94FB600E94D86069812A81E6
:10C58000023139F5862F90E0A0E0B0E04B81DC016C
:10C590009927882730E0322F2227820F931FA11D71
:10C5A000B11D61FF09C0840F911DA11DB11DBC010A
:10C5B000CD018C6F9F6F06C0BC01CD01640F711D52
:10C5C000811D911D0E94748C20E83FEF4FEF57E4CE
:10C5D0001FC070E0762F6627620F711D072E000CBA
:10C5E000880B990B0E94748C0C3029F420E030EEFB
:10C5F0004FEF54E40DC00E3029F420E038EF4FEF38
:10C6000055E406C0003131F420E03EEF4FEF56E430
:10C610000E94C08B2FE632E143E050E40E946C8E12
:10C620006B017C01612F70E080E090E00E94748CCF
:10C630009B01AC01C701B6010E94C08B0F900F9007
:10C640000F90DF91CF911F910F91FF90EF90DF90AE
:10C65000CF9008959C68692F70E023E030E0AE0130
:10C660004F5F5F4FCF010E94FB1762E174E380E0F0
:10C6700090E00E9458608F2D0E947B600E94F160C4
:10C6800089830E94F1608A8356CF613009F02CCFF4
:10C690009068692F70E023E030E0AE014F5F5F4F9C
:10C6A000CF010E94FB1762E174E380E090E00E94FA
:10C6B00058608F2D0E947B600E94F16089830E94E8
:10C6C000F1608A833BCFCF93E6E4F1E02081908153
:10C6D0008081C081C295C695C695C370207CC20F6B
:10C6E000969596959073C90F82958C70C80F1F927E
:10C6F000CF9389E093E19F938F930E94EE930F90E5
:10C700000F900F900F908C2FCF9108951F93CF9380
:10C71000DF9346E069E180E00E946E6680E00E945F
:10C72000C3660E94516504B600FE08C088EF92E11E
:10C730009F938F930E94EE930F900F9004B601FE8B
:10C7400008C087EE92E19F938F930E94EE930F9023
:10C750000F9004B602FE08C086ED92E19F938F937E
:10C760000E94EE930F900F9004B603FE08C085EC74
:10C7700092E19F938F930E94EE930F900F9004B6D7
:10C7800004FE08C088EB92E19F938F930E94EE9382
:10C790000F900F9082E699E09F938F938DE992E13D
:10C7A0009F938F930E94EE930E94E0700E941170FD
:10C7B00060E070E085EB92E00E94B3700E94876DAC
:10C7C000E091A609F091A70919950E94636390E092
:10C7D0000E94F4660E94B87482E08093A33780932D
:10C7E000A4370E94496543EA57E3BC018DEC9BEAFC
:10C7F0000E94C8690E94B9640E94AE690E944D659A
:10C800000E94D56A0E94F775E0911C0AF0911D0AFA
:10C810001995E091F409F091F5091995E091E6096F
:10C82000F091E70919950E94D76A182FC091280A3C
:10C83000D091290AFE0119950F900F900F900F903B
:10C84000892B49F0FE011995BC0180E890E00E9417
:10C850007588EB0102C0C0E8D0E00E94AB691F926E
:10C860001F93DF93CF931F928F9380911B0A8F9317
:10C8700080911A0A8F938091F3098F938091F20926
:10C880008F938BE692E19F938F930E94EE938EE5B8
:10C8900092E19F938F930E94EE938DE492E19F9398
:10C8A0008F930E94EE9360E070E087ED92E00E942B
:10C8B000B3708EE299E00E94126D85E492E19F933D
:10C8C0008F930E94EE938DB79EB742960FB6F89461
:10C8D0009EBF0FBE8DBFDF91CF911F91089580E85D
:10C8E00080936100109261000E948663C3E3D2E1ED
:10C8F00002E212E181E1E82E82E1F82E90E0C92EF9
:10C9000092E1D92E22EFA22E21E1B22E04B600FE32
:10C9100006C0DF93CF930E94EE930F900F9004B662
:10C9200001FE06C01F930F930E94EE930F900F908D
:10C9300004B602FE06C0FF92EF920E94EE930F90A3
:10C940000F9004B603FE06C0DF92CF920E94EE93D2
:10C950000F900F9004B604FE06C0BF92AF920E94E3
:10C96000EE930F900F9014BE0E9421700E94E66615
:10C97000CDCFDF92EF92FF920F931F93CF93DF9370
:10C98000CDB7DEB7A0970FB6F894DEBF0FBECDBF10
:10C9900083E690E00E94B396182F282F35EF380FCA
:10C9A000303108F0982F9095291709F463C088E179
:10C9B00093E19F938F930E94EE93EDE5F3E18E0157
:10C9C0000F5F1F4F0F900F90D801D02EE12EF02E49
:10C9D00088E0800F94919D9331968A13FBCFF89451
:10C9E00048E050E06FE770E0C8010E94B996EFE4BC
:10C9F000F3E1D8018EE08F0D94919D9331968A13C7
:10CA0000FBCF4EE050E061E770E0C8010E94B996AC
:10CA1000E5E4F3E12AE02F0D8491D8018D938D0197
:10CA200031962A13F9CF4AE050E067E670E08D2D89
:10CA30009E2D0E94B9966DEC7BEA81E690E00E9403
:10CA4000D19660E070E08FE590E00E94D19660E0C2
:10CA50008EE590E00E94C39660E070E085E690E08D
:10CA60000E94D1961AE16AE175EE83E690E00E9499
:10CA7000D1967894812FA0960FB6F894DEBF0FBEA2
:10CA8000CDBFDF91CF911F910F91FF90EF90DF907D
:10CA900008958FE590E00C94B3968EE590E00C94A9
:10CAA000AB96F8941092B60016BC89E787BD82E079
:10CAB00084BD95E095BD95B395BB80936E00789449
:10CAC00008950F931F936091A5137091A613809101
:10CAD000A7139091A8130091A5131091A61320916C
:10CAE000A7133091A813601771078207930759F7AE
:10CAF0001F910F9108950F931F936091AD35709121
:10CB0000AE358091AF359091B0350091AD35109133
:10CB1000AE352091AF353091B0356017710782077F
:10CB2000930759F71F910F9108951F920F920FB617
:10CB30000F9211240BB60F922F933F934F935F9355
:10CB40006F937F938F939F93AF93BF93EF93FF93D5
:10CB50008091A5139091A613A091A713B091A8134B
:10CB60000196A11DB11D8093A5139093A613A093C8
:10CB7000A713B093A8138091A4138F5F8093A4137D
:10CB800087FF15C01092A4138091AD359091AE35FA
:10CB9000A091AF35B091B0350196A11DB11D809324
:10CBA000AD359093AE35A093AF35B093B03580914D
:10CBB0004C378823E1F08091A3138F5F8093A313F8
:10CBC00087FF15C01092A3138091A5359091A635CB
:10CBD000A091A735B091A8350196A11DB11D8093F4
:10CBE000A5359093A635A093A735B093A8350E949C
:10CBF0001E6F892B11F00E943F6EFF91EF91BF9144
:10CC0000AF919F918F917F916F915F914F913F91E4
:10CC10002F910F900BBE0F900FBE0F901F90189585
:10CC20001F920F920FB60F9211240BB60F922F93F3
:10CC30003F934F935F936F937F938F939F93AF93A4
:10CC4000BF93EF93FF938091C600E091B335F091CD
:10CC5000B435309709F01995FF91EF91BF91AF91DD
:10CC60009F918F917F916F915F914F913F912F9104
:10CC70000F900BBE0F900FBE0F901F9018951F9234
:10CC80000F920FB60F9211240BB60F922F933F9372
:10CC90004F935F936F937F938F939F93AF93BF93C4
:10CCA000EF93FF938091CE00E091B135F091B235D2
:10CCB000309709F01995FF91EF91BF91AF919F9136
:10CCC0008F917F916F915F914F913F912F910F9035
:10CCD0000BBE0F900FBE0F901F90189581110EC0C4
:10CCE0001092C5006093C40088E98093C10040930E
:10CCF000C2001092B4351092B3350895813069F4B2
:10CD00001092CD006093CC0088E98093C9004093D5
:10CD1000CA001092B2351092B1350895811107C042
:10CD20008091C00085FFFCCF6093C60008958130DC
:10CD300031F48091C80085FFFCCF6093CE00089548
:10CD4000CF93C82F8A3031F46DE08091A9130E94EF
:10CD50008E6602C08D3029F06C2F8091A9130E943D
:10CD60008E6680E090E0CF910895811105C07093A8
:10CD7000B4356093B3350895813021F47093B235A2
:10CD80006093B13508958093A91383E992E090935D
:10CD9000F8398093F739089584B7877F84BF0FB639
:10CDA000F894A8958091600088618093600010924B
:10CDB00060000FBE08959FE088E10FB6F894A89533
:10CDC000809360000FBE909360000895A895089529
:10CDD0000FB6F894A89580916000886180936000F8
:10CDE000109260000FBE08950C948A8F0C94868F69
:10CDF0008091BA3590E008958091390181FF09C092
:10CE0000809139018D7F8093390189E190E001970C
:10CE1000F1F723E040E06FE182E491E00E94326CA0
:10CE200085E090E00197F1F708959091390191FD27
:10CE30000AC0282F803108F02FE040E06FE085E441
:10CE400091E00C94326C08958091390181FD0EC0FF
:10CE500040E06FE181E491E00E94276C282F2F7E53
:10CE600081E090E0213021F080E0089580E090E0C2
:10CE700008958091390181FF02C081E0089540E06A
:10CE80006FE181E491E00E94276C8F3121F08F7E69
:10CE90008150823090F780E008958091390181FDC2
:10CEA00004C00E9439678823C1F3089510924C375B
:10CEB0008091390181FD8BC00E944D6780913901BD
:10CEC00081FD85C00E94FC6680913901826080935B
:10CED0003901809184378823D9F180919400909111
:10CEE0009500409195375091963784179507A0F497
:10CEF0008091613790916237A0916337B091643728
:10CF0000875F924CAF4FBF4F8093613790936237EA
:10CF1000A0936337B09364372091940030919500CB
:10CF2000241B350B8091613790916237A091633754
:10CF3000B0916437820F931FA11DB11D809361379B
:10CF400090936237A0936337B0936437109284371D
:10CF5000809186378823D9F1809194009091950033
:10CF60004091993750919A3784179507A0F4809192
:10CF7000693790916A37A0916B37B0916C37875FB2
:10CF8000924CAF4FBF4F8093693790936A37A0930D
:10CF90006B37B0936C372091940030919500241B2F
:10CFA000350B8091693790916A37A0916B37B091BA
:10CFB0006C37820F931FA11DB11D80936937909329
:10CFC0006A37A0936B37B0936C3710928637089509
:10CFD00080914C37882321F00E9439670E94566760
:10CFE00080E090E0089522E0260F27FF0CC080919A
:10CFF0004A3790914B37019690934B3780934A373D
:10D000008FEF9FEF0895AB01BC018AEA93E10E9484
:10D010001F9380E090E0089540E06FE181E491E0AB
:10D020000C94276C282F40E06FEF86E591E00E947A
:10D03000326C0895CF93DF9398EF980F923038F0C9
:10D04000982F9F7E963019F0893109F049C0909150
:10D05000390191FD48C0C82F0E944D670E940C689D
:10D06000D82FC81709F442C0C83029F4809139017B
:10D070000E94FC6627C0C93119F4863181F404C0CE
:10D08000C63169F4893159F429E040E06FE182E466
:10D0900091E00E94326C85E090E00197F1F72C2F2F
:10D0A00040E06FE182E491E00E94326CD83031F4CC
:10D0B0008FEF0E94126881ED92E002C085E090E05F
:10D0C0000197F1F70E940C688C1781F0C63019F4B3
:10D0D000813079F40BC0C63161F4813151F406C05E
:10D0E00082E490E008C084E490E005C080E490E031
:10D0F00002C083E490E0DF91CF9108958091940085
:10D100009091950090939A378093993781E080931E
:10D11000863780934C379091390191FF1EC0209142
:10D1200094003091950030939637209395378093F3
:10D130008437809347372FB7789480913901809155
:10D1400039018D7F8093390180E197E23091473733
:10D15000332311F00197D1F72FBF86E10E941A689F
:10D160000C944D6780914C37811102C00E947E68FB
:10D1700081E090E008950F931F93CF93DF931F9268
:10D18000CDB7DEB780914C37882361F080913901AB
:10D1900081FF02C080E07BC00E9439678823D1F301
:10D1A00000E003C00E94B26801E080919400909179
:10D1B0009500909394378093933711E010938337C1
:10D1C00080E88093550186E00E941A681093BB3571
:10D1D0008FB789837894109247018091BB35811174
:10D1E000FCCF89818FBF8091470111E08E3008F01C
:10D1F00010E0119586E10E941A6810925501809105
:10D2000083378823D9F180919400909195004091C3
:10D2100093375091943784179507A0F480915D3728
:10D2200090915E37A0915F37B0916037875F924CE5
:10D23000AF4FBF4F80935D3790935E37A0935F37BA
:10D24000B09360372091940030919500241B350BEA
:10D2500080915D3790915E37A0915F37B0916037D4
:10D26000820F931FA11DB11D80935D3790935E3790
:10D27000A0935F37B09360371092833701110E94FB
:10D28000E867812F8295869586958370817090E0FE
:10D290000F90DF91CF911F910F9108958FEF8093A1
:10D2A0004E0121E044E060EF8CE691E00E94326C98
:10D2B00025E041E06EE08CE691E00E94326C80E86F
:10D2C00080936F018091460180936D0121E045E0DC
:10D2D00060E284E491E00C94326CCF93DF93C9EF69
:10D2E000D7E0CE010197F1F70E94266C1092C1356C
:10D2F000109243361092C5361092C0351092BF3549
:10D30000E9E3F1E080818E7F808380818D7F80835F
:10D3100081EC93E00197F1F780818160808323E0C5
:10D3200040E06FE182E491E00E94326C2197F1F7D6
:10D3300080915D0180915E010E944E6960E070E025
:10D3400081EA92E00E94B3700E947E6881E090E0E2
:10D35000DF91CF91089580912B140895CF93DF939F
:10D360001F92CDB7DEB789830E944D678981809374
:10D370002B14282F40E06FE188E491E00F90DF91BB
:10D38000CF910C94326C0E94AE6986E00C941A68BE
:10D39000EF92FF920F931F93CF93DF931F921F92F1
:10D3A000CDB7DEB78C017A017F936F931F938F9374
:10D3B0008CE799E09F938F9369837A830E94DA9335
:10D3C00000936201109363016981609360017A8127
:10D3D000709361010F900F900F900F900F900F902E
:10D3E000E114F104C9F0F701808180936B01818120
:10D3F00080936A01828180936901838180936801AF
:10D400008481809367018581809366018681809302
:10D4100065018781809364010F900F90DF91CF9118
:10D420001F910F91FF90EF90089581EA92E00E9482
:10D43000D47081E08093BA358091BC359091BD3530
:10D4400001969093BD358093BC3581E090E00895BE
:10D450000F931F93CF932091C035C2E8C29F9001D4
:10D460001124F901EF53FA4C4081442309F451C0CF
:10D4700047FD09C0433038F050E08A0102501109DD
:10D480006017710710F4108244C0B9016E537A4CD2
:10D490000E941F938091C035C89FF0011124EF5363
:10D4A000FA4CDF01A058BF4F9C919093B535108284
:10D4B0008F5F833018F48093C03502C01092C0355E
:10D4C000E091C03582E8E89FF0011124EF53FA4C57
:10D4D0008081882319F00E94156A02C01092BA3523
:10D4E000809147018093B6359091B935992311F019
:10D4F000891710F48093B9356091B63570E084E0F7
:10D500000E94D3756091B53570E083E00E94D375B9
:10D5100002C000E010E0C801CF911F910F91089563
:10D520000F931F93CF93DF931F92CDB7DEB78C017C
:10D53000FC0180819181009709F18334954029F0A5
:10D54000F8011182108283E02AC06238E1F40E945F
:10D550007F758FB78983F8940E94EE7460E870E05D
:10D560000E94286A29812FBF1816190674F40E9498
:10D57000E974E091220AF091230A199583E495E079
:10D58000F8019183808381E00AC08091B735909142
:10D59000B83501969093B8358093B735EFCF0F909B
:10D5A000DF91CF911F910F9108950C941567809191
:10D5B000390181FD06C040E06FE085E491E00C9404
:10D5C000276C80E10895EF92FF921F93CF93DF9332
:10D5D0001F92CDB7DEB7182F8091390181FD07C0AA
:10D5E0000E944D6780914C3781111CC05AC08091B8
:10D5F000940090919500909396378093953781E0B1
:10D600008093843780934737809139018D7F809351
:10D61000390180E197E220914737222309F30197EE
:10D62000D1F7DECF809186378823D9F1809194009D
:10D63000909195004091993750919A3784179507AA
:10D64000A0F48091693790916A37A0916B37B091BF
:10D650006C37875F924CAF4FBF4F80936937909381
:10D660006A37A0936B37B0936C3720919400309158
:10D670009500241B350B8091693790916A37A091F2
:10D680006B37B0916C37820F931FA11DB11D809332
:10D69000693790936A37A0936B37B0936C371092C9
:10D6A000863789E10E941A6886E00E94DE75892B20
:10D6B00051F00E94D76AE82E86E00E94DE75815004
:10D6C0000E94156702C0E12CF12C8091940090918A
:10D6D0009500909398378093973781E080938537B2
:10D6E0008FB78983F89480913901826080933901E2
:10D6F000809139018D7F8093390162E0610F8AEA60
:10D7000093E10E94796C89818FBF80914837909115
:10D710004937019690934937809348370E944D6767
:10D7200045E060EE82E491E00E94276C182F86E0CD
:10D730000E94DE75892B19F08E2D0E94156780914D
:10D7400085378823D9F1809194009091950040917C
:10D7500097375091983784179507A0F480916537D3
:10D7600090916637A0916737B0916837875F924C88
:10D77000AF4FBF4F8093653790936637A09367375D
:10D78000B09368372091940030919500241B350B9D
:10D790008091653790916637A0916737B09168376F
:10D7A000820F931FA11DB11D80936537909366373B
:10D7B000A0936737B09368371092853780914C37C4
:10D7C000882371F0809194009091950090939A37FE
:10D7D0008093993781E0809386370E947E6802C0EB
:10D7E0000E945667123028F48CE00E94DE7510E02B
:10D7F0000BC0133031F0153031F0173029F411E03F
:10D8000003C012E001C013E0812F90E00F90DF9180
:10D81000CF911F91FF90EF900895CF93DF93EB018D
:10D820000E94F367009729F4CE010E94E36A0097F3
:10D8300051F020914A3730914B372F5F3F4F309353
:10D840004B3720934A37DF91CF9108950895FC011B
:10D8500080816823862F90E002C0959587954A9530
:10D86000E2F70895CF93DF931F92CDB7DEB7FC01A7
:10D87000922F8FB78983F8942081362F3095522FBD
:10D880005323292F01C0220F4A95EAF72623252B7F
:10D89000208389818FBF0F90DF91CF910895CF931F
:10D8A000DF93E0917B012DEF2E0F2D3740F0FC012F
:10D8B0001082E058FF4F10823196108217C0EC01A1
:10D8C000E993A0E8B1E020E82E0F3C91399311963E
:10D8D0002A13FBCFE150F0E0E058FE4F2181FC011C
:10D8E000E058FF4F2083319681E08083DF91CF9114
:10D8F000089560938001E1E8F1E06158DC012D9129
:10D90000CD01208331966E13F9CF08951F920F92A7
:10D910000FB60F9211240BB60F922F933F934F9394
:10D920005F936F937F938F939F93AF93BF93EF9387
:10D93000FF93809147018093B6358091BF3522E8EF
:10D94000829FC00111248F539A4C0E944F6C80918A
:10D95000BF358F5F833018F48093BF3502C01092BB
:10D96000BF350E94156AFF91EF91BF91AF919F91D2
:10D970008F917F916F915F914F913F912F910F9078
:10D980000BBE0F900FBE0F901F9018951F920F9215
:10D990000FB60F9211240F900FBE0F901F90189585
:10D9A0001F920F920FB60F9211240F900FBE0F907F
:10D9B0001F9018951F920F920FB60F9211240F907F
:10D9C0000FBE0F901F9018951F920F920FB60F92D7
:10D9D0001124109247370F900FBE0F901F9018958B
:10D9E0001F920F920FB60F9211241092BE350F9016
:10D9F0000FBE0F901F9018951F920F920FB60F92A7
:10DA000011240F900FBE0F901F9018951F920F9228
:10DA10000FB60F9211241092BB350F900FBE0F90CE
:10DA20001F901895CF93DF93EC01899199910097FE
:10DA300029F060E070E00E94B370F7CFDF91CF91E2
:10DA40000895EF92FF920F931F93CF93DF938C0172
:10DA50007A01FC0180819181009741F08A3491051F
:10DA600011F1F8011182108283E04AC08DE294E145
:10DA70000E945E71EC01209761F04E815F816885A4
:10DA80007985CE0102960E94F56E0990D881C02D4D
:10DA9000F2CF81E080932C148AE490E0F801918326
:10DAA000808381E02DC06838E1F78DE294E10E9427
:10DAB0005E71EC01209781F3CE010296E816F9061B
:10DAC000D9F4BE018DE294E10E947E71E090E114F0
:10DAD000F090E2148E859F859093E2148093E11478
:10DAE000E889F989309719F08A899B891995F0920C
:10DAF000E214E092E114D0CF0990D881C02DDACFA2
:10DB0000DF91CF911F910F91FF90EF9008951092A8
:10DB10002C148DE294E10E945A7160E070E08BEA6F
:10DB200092E00C94B370EF92FF920F931F93CF93F8
:10DB3000DF93EC01E090E114F090E214FF86EE86B2
:10DB4000398B288B1B8B0A8B80912C14882379F0BE
:10DB50008BEA92E09093E2148093E114CE01029656
:10DB60000E94F56EF092E214E092E11404C04E833C
:10DB70005F8368877987BE018DE294E10E947E71A0
:10DB8000BE018DE294E1DF91CF911F910F91FF9043
:10DB9000EF900C949D71CF93DF93EC0180912C1446
:10DBA000882329F0CE0102960E94296F04C01B86AB
:10DBB0001A861D861C86BE018DE294E1DF91CF910D
:10DBC0000C947E71CF92DF92EF92FF920F931F938E
:10DBD0008091331490913414892B49F410922F14AE
:10DBE00010923014109231141092321441C00E94DD
:10DBF00061658B019C01E0913314F09134144481F0
:10DC000055816681778180819181A281B381840F62
:10DC1000951FA61FB71F801B910BA20BB30B00848F
:10DC2000F185E02D3097C1F0C480D580E680F78083
:10DC300040815181628173814C0D5D1D6E1D7F1D80
:10DC4000401B510B620B730B481759076A077B0780
:10DC500030F7DB01CA01E3CF800F911FA21FB31F72
:10DC600080932F1490933014A0933114B0933214F6
:10DC70001F910F91FF90EF90DF90CF90089585EB6B
:10DC800092E00C94D470EF92FF920F931F93CF9376
:10DC9000DF938C01FC0180819181009799F0893597
:10DCA0009105D9F0F8011182108283E068C0828565
:10DCB00093858417950709F049C00084F185E02D0C
:10DCC0003097A9F7109234141092331489E590E03C
:10DCD000F8019183808381E052C0673891F1623806
:10DCE000A9F7C0913314D0913414E12CF12C209772
:10DCF00069F3CE010E942F71892BF1F0AE0168E823
:10DD00008A859B850E948570892BA1F41B861A86C3
:10DD100088859985E114F10421F0F70191878087C6
:10DD200004C09093341480933314198618860E948B
:10DD3000E26DD7CF0E943F6E7E010884D985C02D49
:10DD4000D6CFE0913314F0913414BACFF093341459
:10DD5000E0933314A085B185109709F4B7CF1A96D4
:10DD60008D919C911B978417950739F418968D9186
:10DD70009C91199791878087EDCFFD01EBCFDF91C3
:10DD8000CF911F910F91FF90EF900895CF93DF9364
:10DD9000EC010E943F6E2A853B859091331480915F
:10DDA0003414232B91F0E92FF82F309771F0EC17F2
:10DDB000FD0739F48091E1149091E21493878287F2
:10DDC00010C00084F185E02DF0CF2091E114309156
:10DDD000E2143B872A8798878987D0933414C093AD
:10DDE0003314DF91CF910C94E26DCF93DF93EC016C
:10DDF0000E940171CE01DF91CF910C94C66ECF933A
:10DE0000DF93EC010E941171CE01DF91CF910C9450
:10DE1000C66ECF93DF93EC010E942371CE01DF9198
:10DE2000CF910C94C66E21E030E0FC018285938591
:10DE3000892B11F020E030E0C901089581E090E0E5
:10DE40002091331430913414232B11F480E090E0AE
:10DE50000895CF93DF93EC01E0913314F0913414E3
:10DE60008E179F0769F48885998590933414809361
:10DE700033140DC0808591858C179D0721F0FC011E
:10DE80003097C1F706C088859985918780870E9461
:10DE9000E26D198618861B861A86DF91CF91089548
:10DEA0001F93CF93DF93DC011496ED91FC911597AE
:10DEB0003097E1F0162FEC019093E2148093E11477
:10DEC00082E08887CD0106961995082E000C990BE3
:10DED0000297029710F0133839F4BE01CE01DF919A
:10DEE000CF911F910C94806F81E08887DF91CF9153
:10DEF0001F910895FC01208520FD0C94506F08951A
:10DF0000CF92DF92EF92FF920F931F93CF93DF9305
:10DF1000E090E114F090E214C090E314D090E41487
:10DF2000F601E817F90739F0309709F44BC0019072
:10DF3000F081E02DF6CF009709F444C08B01EC018D
:10DF40008885882309F11886C114D10461F0CC15A5
:10DF5000DD0529F0AE0167E8C6010E947A6FF6017F
:10DF6000C080D180F1CFEC81FD81309769F0C0177E
:10DF7000D10751F0D093E214C093E11440E050E097
:10DF800063E8CE0106961995E091E314F091E4144C
:10DF9000CE17DF0741F4888199819093E414809330
:10DFA000E3140CC0FC01309749F0808191818C17FB
:10DFB0009D07C1F78881998191838083F092E21453
:10DFC000E092E114DF91CF911F910F91FF90EF90BC
:10DFD000DF90CF9008951F93CF93DF9310923D145D
:10DFE000C091E314D091E41411E0209779F0898571
:10DFF000882341F01887198640E050E062E8CE019E
:10E000000E94506F0990D881C02DEFCFDF91CF9142
:10E010001F9108958091E01491E0980F9093E0147F
:10E0200008958AE88093E0141092DE141092DF14B1
:10E030001092E4141092E3141092E2141092E1147E
:10E04000089580913D1481110E94EB6F5091DF146F
:10E05000552309F452C0E091DE142E2F30E085E004
:10E06000E89FF0011124E25CFB4E608160933C1458
:10E07000A181B281B0933B14A0933A14838194811F
:10E0800090933914809338142F5F3F4F2F713327AB
:10E090002093DE1451505093DF14009731F5809196
:10E0A000E3149091E4149093371480933614809184
:10E0B000361490913714892B01F180913D14811110
:10E0C0000E94EB6F40913A1450913B1460913C14C4
:10E0D00080913614909137140E947A6FE091361433
:10E0E000F091371480819181DECF613819F421E0FD
:10E0F000FC012087AD010E947A6F80913D14209130
:10E10000DF1490E0820F911D08959C019091DF141F
:10E110009032B9F0E091DE14E90FEF71E09335141D
:10E1200085E0E89FF0011124E25CFB4E608352839E
:10E130004183348323839F5F9093DF1480E090E0DA
:10E14000089581E090E00895CF93DF93C091E114AA
:10E15000D091E2140E947A6FD093E214C093E1143C
:10E16000DF91CF910895AB013091E3142091E41435
:10E17000E32FF22FE817F907B1F0309721F0019063
:10E18000F081E02DF7CF009771F0FC0130832183FF
:10E190009093E4148093E31421E020871782168281
:10E1A00061E80C94A4700895009749F0FC01208563
:10E1B0002150223020F421E0218720933D1408953E
:10E1C0000C940D7A8091E5149091E6140097C1F0BB
:10E1D0001092E6141092E514DC0114966D917C9176
:10E1E00015971296ED91FC9113971995E091E5140E
:10E1F000F091E614309721F0808191810C94277A78
:10E200000895CF93DF93EC014C835D836E837F830E
:10E210000E946165688379838A839B83DF91CF91B4
:10E220000895FC01408151816281738184819581CF
:10E23000A681B781840F951FA61FB71F8083918386
:10E24000A283B3830895CF93DF93EC010E946165AD
:10E25000688379838A839B83DF91CF910895CF92DE
:10E26000DF92EF92FF92CF93DF93EC010E94616502
:10E27000C880D980EA80FB80DC01CB018C199D0924
:10E28000AE09BF090196A11DB11D21E030E0CC808F
:10E29000DD80EE80FF80C816D906EA06FB0610F086
:10E2A00020E030E0C901DF91CF91FF90EF90DF9047
:10E2B000CF900895FC01118210820895FC018081A5
:10E2C00091810895DC01ED91FC91309741F08081BE
:10E2D0009181009711F0FC01FACFCF01089580E001
:10E2E00090E00895DC01ED91FC911197309721F0B9
:10E2F000208131812D933C93CF010895DC01ED9174
:10E30000FC913097C9F0A0E0B0E0E617F70761F4A0
:10E31000FB0120813181109709F4DC012D933C939E
:10E32000FB0111821082089520813181DF012115C6
:10E33000310511F0F901E9CF08950F931F93CF93A1
:10E34000DF938C01EB010E947E7119821882C80153
:10E350000E946271009711F4F80101C0FC01D183A1
:10E36000C083DF91CF911F910F910895DC01ED9152
:10E37000FC9180E090E0309729F001960190F081C7
:10E38000E02DF9CF0895009721F0FC018081918163
:10E39000089580E090E00895CF93DF93EC014A81E7
:10E3A0005B8160E070E08C819D810E9428932A81CE
:10E3B0003B8188819981289FA001299F500D389F1A
:10E3C000500D112460E070E08E819F81DF91CF912C
:10E3D0000C942893FC018281938120E030E028177F
:10E3E0003907D1F0A481B581A20FB31F4C9141111F
:10E3F00010C081E08C9380819181289FA001299F8A
:10E40000500D389F500D112486819781840F951FE0
:10E4100008952F5F3F4FE3CF80E090E00895FC0127
:10E42000868197814281538120E030E024173507AF
:10E43000D1F08617970781F4A481B581A20FB31F8D
:10E440008C91181614F481508C9384819581FC0171
:10E45000E20FF31F80810895A081B1818A0F9B1F75
:10E460002F5F3F4FE3CF8FEF0895FC012681378167
:10E4700062177307A0F0A081B18142815381A49FEC
:10E48000C001A59F900DB49F900D1124280F391F36
:10E4900081E090E06217730720F080E0089580E04B
:10E4A00090E008952F923F924F925F926F927F92E9
:10E4B0008F929F92AF92BF92CF92DF92EF92FF9294
:10E4C0000F931F93CF93DF93CDB7DEB768970FB647
:10E4D000F894DEBF0FBECDBFEDE4F7E324A535A56C
:10E4E00046A557A550A441A432A423A4948C858C9E
:10E4F000768C678C808D8983918D9A83828D8B83B6
:10E50000938D9C8384898D8395899E8386898F834F
:10E51000978998878089898791899A8782898B874B
:10E5200093899C8784858D8795859E8786858F872F
:10E530009785988B8085898B91859A8BB284A384EB
:10E54000F480E580D680C78080818F8B9181988F01
:10E55000128103812B8B3C8B4D8B5E8B0E947B65E4
:10E560005E895F934D894F933C893F932B892F930D
:10E570002F923F924F925F926F927F928F929F92D3
:10E580002C812F932B812F932A812F9329812F93D5
:10E5900028852F932F812F932E812F932D812F93B9
:10E5A0002C852F932B852F932A852F9329852F93A5
:10E5B00028892F932F852F932E852F932D852F9389
:10E5C000AF92BF922A892F9329892F93CF92DF92FE
:10E5D000EF92FF920F931F93288D2F932F892F93E4
:10E5E0009F938F937F936F93E3EAF7E381811F9269
:10E5F0008F9380811F928F9385E693E19F938F93F2
:10E600000E94EE930FB6F894DEBF0FBECDBF6896A2
:10E610000FB6F894DEBF0FBECDBFDF91CF911F9133
:10E620000F91FF90EF90DF90CF90BF90AF909F90B1
:10E630008F907F906F905F904F903F902F900895B4
:10E64000EF92FF920F931F93CF93DF938C01EB0117
:10E650007A010E94B673F801F086E78265ED79E0F1
:10E66000CE01DF91CF911F910F91FF90EF900C940D
:10E67000DA730C94BE730C947274DC011796ED91EE
:10E68000FC9118970190F081E02D309709F01994D2
:10E690000895DC011796ED91FC9118970280F381A3
:10E6A000E02D309709F019940895DC011996ED9149
:10E6B000FC911A970280F381E02D309709F01994AC
:10E6C00008950F931F93CF93DF931F921F92CDB79F
:10E6D000DEB78C0188E10E94F175BC01CE01019684
:10E6E0000E94A074D8011996ED91FC911A9701909F
:10E6F000F081E02D309729F0BE016F5F7F4FC80198
:10E7000019950F900F90DF91CF911F910F91089560
:10E71000EF92FF920F931F93CF93DF938C01EB0146
:10E720007A0147ED59E00E942073F801F286E186F4
:10E730006BED79E0CE01DF91CF911F910F91FF90AA
:10E74000EF900C94DA730C943973CF93DF93EC0150
:10E7500063EA77E388E10E94E775CE01DF91CF910C
:10E760000C943B7387EE94E10C945A71FC01738313
:10E770006283BC0187EE94E10C949D71BC0187EE2D
:10E7800094E10C947E71CF93DF93EC0187EE94E1DA
:10E790000E945E71009749F0FC01228133812C17A1
:10E7A0003D0729F00E94C371F5CF80E090E0DF9132
:10E7B000CF9108950F931F93CF93DF938B010E9406
:10E7C000C373EC01892B31F01D830C83C8010E94B7
:10E7D000DA838E83DF91CF911F910F910895CF92AD
:10E7E000DF92EF92FF920F931F93CF93DF937C0101
:10E7F0008B016A0189EE94E10E945E71EC01892B24
:10E8000051F0EC81FD81309711F0C8011995CE01CE
:10E810000E94C371F3CFA601B801C701DF91CF9168
:10E820001F910F91FF90EF90DF90CF900C94497360
:10E830000F931F93CF93DF931F921F92CDB7DEB735
:10E840000E94AC838C0189EE94E10E945E71009776
:10E8500079F0DC011296ED91FC911397309729F035
:10E8600089839A8319959A8189810E94C371EFCF18
:10E870000115110549F0C8010F900F90DF91CF915C
:10E880001F910F910C943D730F900F90DF91CF91DA
:10E890001F910F910895CF92DF92EF92FF920F9305
:10E8A0001F930E94F7750E947F750E9441820E940B
:10E8B000AA83C12C88E0D82E87E0E82EF12C00E056
:10E8C0001EE120E030E040E052E060E070E082E0F5
:10E8D00090E00E9471831F910F91FF90EF90DF9065
:10E8E000CF900895CF93DF93EC010E94BF830097F0
:10E8F00061F00E940775E091F609F091F709BE01F9
:10E900008FEE93E7199581E090E0DF91CF91089524
:10E91000E0911E0AF0911F0A1994E091E809F09124
:10E92000E9091994E091240AF091250A1994E091DB
:10E93000260AF091270A199480E090E0089508953E
:10E94000FB0120813181FC0131832083089542E065
:10E9500050E00E94129321E030E0892B11F020E07A
:10E9600030E0C9010895BC0183EA97E30C94A074D8
:10E97000E091A609F091A7091995E0911C0AF09180
:10E980001D0A1995E091F409F091F5091995E091A6
:10E99000E609F091E70919942091A2153091A31589
:10E9A0002817390798F04091A0155091A115480FEC
:10E9B000591F5093A1154093A015281B390B309374
:10E9C000A3152093A21581E090E0089580E090E0E7
:10E9D00008959093A3158093A21508958091A01592
:10E9E0009091A115835E9A4E089580919F1590E0B5
:10E9F00083519B4E089581E090E02091EB1430917B
:10EA0000EC142D51354111F480E090E008950E94FE
:10EA1000FB74892B61F06091EB147091EC144091C0
:10EA2000A2155091A3158DE195E10C941F932091AF
:10EA3000A0153091A11521153105B9F08091A215CD
:10EA40009091A315C096EDE1F5E1AF014D5E544103
:10EA50004817590734F4DF01A20FB31F4C914193BB
:10EA6000F4CF1092A1151092A01508958091A215CF
:10EA70009091A315089580919F1590E3981B209184
:10EA8000A2153091A315A901490F511DCA0108957E
:10EA90000F931F93CF938C01C0919F158C2F90E003
:10EAA000801791076CF00E943B75800F911F813891
:10EAB000910530F4C01BC0939F1581E090E002C027
:10EAC00080E090E0CF911F910F910895CF93DF9355
:10EAD000EDEAF7E31192119287E3ED3DF807D1F7E4
:10EAE000C5EAD7E360E07AE0CE010E94A0742296E6
:10EAF00087E3CD3AD807B1F7DF91CF91089510920F
:10EB0000A1151092A0151092A3151092A21580E3E2
:10EB100080939F158DE195E19093EC148093EB1415
:10EB20000C946675EF92FF920F931F93CF93DF9330
:10EB30001F921F92CDB7DEB78C0169837A830E9442
:10EB40007F756981E62E7A81F72E81E8E816F10457
:10EB500018F080E8E82EF12CA701B8018091EB14A1
:10EB60009091EC140E941F93F092A315E092A215CD
:10EB7000C7010F900F90DF91CF911F910F91FF90E0
:10EB8000EF900895FC0190E3ADEAB7E301900D9298
:10EB90009A95E1F788E0FB01A5EAB7E301900D92B1
:10EBA0008A95E1F70895E82FF0E0EE0FFF1FE35597
:10EBB000F84C7183608381E090E00895E82FF0E0E5
:10EBC000EE0FFF1FE355F84C80819181089590E08E
:10EBD000880F991F8B58984C0E94A07481E090E098
:10EBE000089590E0880F991F8B58984C08958FEBEB
:10EBF00092E00E94CC718FEC92E00E94CC7187EC85
:10EC000092E00C94CC710F931F93CF93DF93EC01A0
:10EC1000BC018FEC92E00E943572892BA9F009901B
:10EC2000D881C02DFE0161917191CF010E94927532
:10EC3000BE016E547F4FCE018E579F4FDF91CF9113
:10EC40001F910F910C94C275BE0187EC92E00E9457
:10EC50003572892BD1F00E947F75688179818A8114
:10EC60009B810E9492758CA990E00E9448750CA926
:10EC700010E00E94F574BE016C5F7F4FA801DF9128
:10EC8000CF911F910F910C941F93DF91CF911F9102
:10EC90000F91089587E19CE10E94136F892B21F069
:10ECA00087E19CE10C94096F0895E091031CF091B9
:10ECB000041C309709F0199480E00895EF92FF92B8
:10ECC0000F931F93CF93DF938C01EA01FC018081A6
:10ECD0009181009741F08A33934081F1F8011182CC
:10ECE000108283E0F8C080E024E0829FF0011124CC
:10ECF000EB5FF34E118210828F5F8430A9F780930F
:10ED0000021C8091E1149091E2149093161C809360
:10ED1000151C0E940A708093DD3740E450E060E0EB
:10ED200070E087E19CE10E94F56E0E94EE7A8AE332
:10ED300093E0F8019183808381E0CDC06230D9F403
:10ED40008091DE379091DF37892B89F38091EF37FF
:10ED5000863029F48091073881FD0E944A7681E04F
:10ED60000E94357B8091DE379091DF37892BF9F255
:10ED70000E94B877DCCF633060F5611114C0209732
:10ED8000B1F2D093DC38C093DB3883E00E94357B4E
:10ED90008091DE379091DF37892B11F00E945576F4
:10EDA0000E944A76C4CF613011F6209709F4BFCF94
:10EDB000D093D838C093D73885E00E94357B8091B6
:10EDC000DE379091DF37892B09F4B1CF0E94557659
:10EDD000AECF673809F040C01092011C85E0E82EE4
:10EDE0008CE1F82E8091011C8430C0F4F7018281FF
:10EDF00093818C179D0749F4808191810E941A7B31
:10EE0000F7011182108213821282F4E0EF0EF11CDE
:10EE10008091011C8F5F8093011CE4CFE6EFF8E343
:10EE2000838194818C179D0719F4148213821082B8
:10EE3000B09629E3E637F20799F7E3E7F9E381852E
:10EE400092858C179D0711F4158214823D9689E3F3
:10EE5000E53FF807A1F76BCF683809F068CFC751D5
:10EE6000DC4109F064CF87E19CE10E94136F892B9C
:10EE700009F45DCF1092011CE091011CE43008F010
:10EE800056CF20E2E29FF0011124E352F74C818D2E
:10EE90008823D9F087E19CE10E94096F8091011CD1
:10EEA000E0E28E9FC00111248352974C9093DC388E
:10EEB0008093DB3882E00E94357B8091DE37909131
:10EEC000DF37892B11F00E9455768091011C8F5FEE
:10EED0008093011CD1CFDF91CF911F910F91FF90B3
:10EEE000EF900895CF93DF93A091DB38B091DC3899
:10EEF000109719F0ED016C9605C0C091D738D091EC
:10EF0000D83829968091D63886FF23C01092001CED
:10EF100080E0E5E0FCE18430C1F04081518114964D
:10EF20002D913C9115974217530761F4228133814B
:10EF30002115310539F08093001C398328831B8209
:10EF40001A8205C034968F5FE6CF8093001C0E9422
:10EF50004A7688819981009741F04A815B8160916E
:10EF6000DD37DF91CF910C94A470DF91CF9108959C
:10EF70000F931F93CF93DF938091EF37863009F083
:10EF80007AC08091DE379091DF37803F910508F499
:10EF900072C08897EC01D695C7959E01220F331F4A
:10EFA0008E012817390710F40F5F1F4FCE01889686
:10EFB0009093DF378093DE379093E8378093E9377B
:10EFC00010920B3810920A380E94E87A809590953A
:10EFD00090930B3880930A381092F1371092F037E3
:10EFE0000E94D77A809590959093F1378093F0376F
:10EFF0000E945576C80188969093DF378093DE375C
:10F000009093E8378093E9378091D9389091DA3836
:10F01000BC016C0F7D1FA8010E941F93BE018EEFE3
:10F0200097E30E94847A8091E2378093FE37809143
:10F03000E3378093FF378091E437809300388091E5
:10F04000E5378093013810920B3810920A380E94ED
:10F05000E87A8095909590930B3880930A381092B7
:10F06000F1371092F0370E94D77A8095909590935F
:10F07000F1378093F037DF91CF911F910F910C946E
:10F080005576E091B609F091B709199480E090E0C7
:10F090000895AF92BF92CF92DF92EF92FF920F93BB
:10F0A0001F93CF93DF93CDB7DEB7E1970FB6F894F8
:10F0B000DEBF0FBECDBF7C016B01CE0101965C01AE
:10F0C00081E3F50111928A95E9F781E089838CE06B
:10F0D0000E94DE758C831D821F828091231C91E02B
:10F0E000980F9093231C898713E018878DEC9BEA77
:10F0F0009B878A8789E10E94F17560E07AE00E942F
:10F10000A774892B31F082E08E838FEF8C878D87F7
:10F1100009C089E10E94F175BC01CE010C960E94E4
:10F12000A0741E838DEC9BEA9D8B8C8B63EA77E346
:10F13000CE0146960E94A0740E94EE749FA78EA7EF
:10F140000E94367599AB88ABC5010E9422848C0160
:10F150001127C8010E944875892B31F10E94F5746E
:10F16000A801BC01C5010E9445840091AC09109121
:10F17000AD090E943B755C010E94F574B501F80170
:10F180001995E114F10481F0009739F0019761F4C9
:10F1900041E050E064E070E004C041E050E060E035
:10F1A00070E0C601F7011995E1960FB6F894DEBF3D
:10F1B0000FBECDBFDF91CF911F910F91FF90EF90C8
:10F1C000DF90CF90BF90AF9008950F931F93CF9390
:10F1D000DF934115510579F0FA018B01EC01828131
:10F1E00093810E940376B801CE01DF91CF911F91E8
:10F1F0000F910C944978DF91CF911F910F91089551
:10F200000F931F93CF93DF93CDB7DEB7E1970FB680
:10F21000F894DEBF0FBECDBF0E9436758C010E94F0
:10F22000EE74AE014F5F5F4FB8010E943885892BA5
:10F2300009F443C088A999A99801281B390BC90171
:10F240000E94CC74892BC9F18E8181110CC0BE0142
:10F250006A5E7F4F88E10E94E775E091F809F091BE
:10F26000F90919952AC02A853B852D3C9BEA390767
:10F2700019F02F3F3F4F09F5823019F088E090E0F8
:10F2800002C082E090E0019710F3E1E0F0E0EC0FC3
:10F29000FD1FE80FF91F23852F3FA9F3BE01645F0F
:10F2A0007F4F89E10E94E77589E10E94F17563EA69
:10F2B00077E30E94A774892B51F6E1960FB6F89474
:10F2C000DEBF0FBECDBFDF91CF911F910F9108958B
:10F2D0000E94F6668093231CE091B609F091B7096D
:10F2E0001994892B29F0E091B609F091B70904C06F
:10F2F000E091B809F091B9091994FC01680F791FE0
:10F3000080E048E1E617F70781F0219198E0322F7D
:10F310003827532F517030FD84278695513009F4DA
:10F3200080682695915099F7EDCF08951F920F921E
:10F330000FB60F9211240BB60F922F933F934F935A
:10F340005F936F937F938F939F93AF93BF93EF934D
:10F35000FF938091940090919500909390378093C3
:10F360008F3781E08093813780917100807D809319
:10F3700071000E94E270809181378823D9F18091D9
:10F3800094009091950040918F3750919037841759
:10F390009507A0F48091553790915637A091573733
:10F3A000B0915837875F924CAF4FBF4F809355371E
:10F3B00090935637A0935737B093583720919400C5
:10F3C00030919500241B350B80915537909156371D
:10F3D000A0915737B0915837820F931FA11DB11DCF
:10F3E0008093553790935637A0935737B09358373B
:10F3F00010928137FF91EF91BF91AF919F918F91C3
:10F400007F916F915F914F913F912F910F900BBE24
:10F410000F900FBE0F901F9018959FB7F894E1E7DB
:10F42000F0E08081807D808388B38F6288BB1092FA
:10F430009000E1E9F0E010821092920010929500A5
:10F44000109294008081856080839FBF08959C0105
:10F450009FB7F894309399002093980088B38F62F7
:10F4600088BBE1E7F0E08081826080839FBF0895E0
:10F47000FB0141505109460F571FE417F50778F477
:10F48000208130E0322F22276181260F311D820F2B
:10F49000931F8217930708F401963296EECFE41774
:10F4A000F50751F4208130E0322F2227820F931F7D
:10F4B0008217930708F401960895CF93DF93C091C4
:10F4C000E937D0E064972091E83730E0322F2227E7
:10F4D000C20FD31F48E050E062EF77E39E01280F90
:10F4E000311DC9010E94387AAE016AEF77E30E94AC
:10F4F000387A009721F098278927982702C08FEF44
:10F500009FEFDF91CF910895FC012381260F209377
:10F51000E537A72FBB2792819A0F9093E43731816B
:10F520003093E33740814093E237E92FF0E0EA1768
:10F53000FB0748F481E0830F8093E337811103C018
:10F540004F5F4093E23730E077272617370788F47C
:10F550009F5F9093E43791110CC08091E3378F5FE8
:10F560008093E337811105C08091E2378F5F8093EC
:10F57000E23708952091DB383091DC38BC01C901B5
:10F5800008960E94847AE091DB38F091DC38A2EE94
:10F59000B7E38C91808711968C9111978187129691
:10F5A0008C911297828713968C918387089544E1FA
:10F5B00050E066EE77E380E090E00E94387A0097B2
:10F5C00021F098278927982708958FEF9FEF0895B6
:10F5D00086E00C945D7A81E10C945D7A80E0E82FFE
:10F5E000F0E0EE0FFF1FE35AF64C118210828F5F9E
:10F5F0008430A9F780E090E2899FF0011124E35262
:10F60000F74C118E8F5F8430B1F780E094E09093D7
:10F61000291C8093281C80E09DE0989FF001112414
:10F62000ED58F64C158214828F5F8A30B1F78093C3
:10F63000271C08959C0190E09430A1F0E92FF0E0A0
:10F6400081E0890FEE0FFF1FE35AF64C4081518194
:10F650004217530729F49093271C118210820895B2
:10F66000982FEACF9093271C0895AF92BF92CF9224
:10F67000DF92EF92FF920F931F93CF93DF93C0918E
:10F68000DB38D091DC38843009F4DBC12EE038E37C
:10F690003093DA382093D9383093E1372093E0372C
:10F6A000833059F4898D8F70833009F06AC088895E
:10F6B0009989892B09F0D4C67EC0823009F07FC0B9
:10F6C00080912D1C8F5F80932D1C811113C0809120
:10F6D0002C1C8F5F80932C1C81110CC080912B1CE3
:10F6E0008F5F80932B1C811105C080912A1C8F5F36
:10F6F00080932A1C1092DF371092DE3710927239F5
:10F7000010927139898D982F9D7F953041F48A8DA3
:10F710008F5F8A8F843109F0A3C6198EA1C6882312
:10F7200009F49EC628893989232B09F440C09A8D93
:10F730002FEF290F2A8F911193C69B8D983031F0AE
:10F740002FEF280F223048F4953039F4198E80E8D5
:10F750008093D6380E9472773DC5953038F423E007
:10F76000092E01C0220F0A94EAF701C020E32A8F74
:10F770009F5F9B8F8F708330A1F048F4813009F434
:10F7800044C3823009F06CC61092073841C38630FA
:10F7900009F4BCC4883009F4B9C4843009F060C6E7
:10F7A000B5C484E08093D6380E94727745C58F70C7
:10F7B000833009F055C688E08093D63800C585307F
:10F7C00019F5E091D738F091D83884819581892B4B
:10F7D00009F446C61092DC381092DB3882E098E3D8
:10F7E0009093DA388093D9389093E1378093E0375B
:10F7F00010927239109271391092DF371092DE3701
:10F8000088E08093D6381BC18091E637853409F0B3
:10F8100027C60091E83710E0102F00278091E937C4
:10F82000080F111D8091DE379091DF378017910707
:10F8300008F416C61093DF370093DE378091EC375B
:10F840008F7309F00DC6F090ED37F11009C6809165
:10F850006D3990916E39C0912A0AD0912B0A8C177C
:10F860009D0759F440916F395091703920912C0ABD
:10F8700030912D0A42175307A1F02091F6373091AD
:10F88000F7372817390709F0EBC52091F837309181
:10F89000F93780916F39909170392817390709F03D
:10F8A000DFC50E94D77A019609F0DAC58091EF375B
:10F8B000863009F429C18131E9F1813009F0D0C5E0
:10F8C0008091FA37883009F0CBC51092FA378091D1
:10F8D000FC379091FD37873F6FEF960710F0099640
:10F8E00001C008969093FD378093FC378091F237E2
:10F8F0009091F337A091F437B091F5378093F637B4
:10F900009093F737A093F837B093F93780916D391A
:10F9100090916E39A0916F39B09170398093F23720
:10F920009093F337A093F437B093F53780E4809346
:10F93000EE3773C50C5111091093DF370093DE3792
:10F9400082E098E39093DA388093D9388091003838
:10F9500090910138892B29F00E94EB7A019609F0E9
:10F960007FC52091FC373091FD372115310509F411
:10F9700077C583E799E39093D8388093D738A090E0
:10F98000FA37B090FB3740912E0A50912F0A6091C0
:10F99000300A7091310AA091F237B091F33700919B
:10F9A000F4371091F537E0902C0AF0902D0AE09191
:10F9B000D738F091D83889E3E53FF80708F050C50B
:10F9C00084819581009721F12817390709F58681EF
:10F9D0009781009719F0A816B906D1F4808191811A
:10F9E0008C179D0729F4C280D380CE14DF04B1F0B8
:10F9F0008417950729F4C280D380C616D70671F004
:10FA0000A817B90729F4828193810817190731F0E3
:10FA10003D96F093D838E093D738C9CF1092DC38B0
:10FA20001092DB3882E08093D63882E098E390939E
:10FA3000E1378093E03710927239109271390E9449
:10FA400072778091713990917239009709F408C5E5
:10FA50009C01245E3F4F3093DF372093DE37309395
:10FA6000E8372093E937E091D738F091D8382085EE
:10FA70002093EE3721E12093EF37089698278927C6
:10FA800098279093FF378093FE3710920138109299
:10FA90000038848195819093FB378093FA37868173
:10FAA00097819093FD378093FC3780916D399091C9
:10FAB0006E39A0916F39B09170398093F23790937D
:10FAC000F337A093F437B093F53780819181A28109
:10FAD000B3818093F6379093F737A093F837B093BC
:10FAE000F9378EE098E39093DA388093D9380E9402
:10FAF000EB7A80959095009711F48FEF9FEF90939C
:10FB000001388093003889C40E94E87A019609F090
:10FB1000A7C44091FC375091FD374115510509F4B8
:10FB20009FC48091FA379091FB37009709F498C4ED
:10FB30006091F2377091F337E091F437F091F53737
:10FB4000CDEDD8E3298D2223A9F0AC81BD814A17E0
:10FB50005B0781F4AE81BF818A179B0759F4A881A6
:10FB6000B9816A177B0731F4AA81BB81EA17FB07C9
:10FB700009F466C1A09629E3CD35D20719F7809123
:10FB800007388F738230D9F45093251C4093241C7E
:10FB900080E0843091F0E82FF0E0EE0FFF1FE35A91
:10FBA000F64C208131818F5F4217530791F71092F5
:10FBB000271C80E0C0E0D0E07CC08093271C8091AF
:10FBC000073882FD4DC484E18093073888E290E0D5
:10FBD0009093DF378093DE3780E58093063830914D
:10FBE0000138809105388093013820910038809148
:10FBF000043880930038209304389091FF37809127
:10FC000003388093FF37909303388091FE378093B9
:10FC1000271C409102384093FE37809302383F5FA3
:10FC20003093053831110DC02F5F20930438211116
:10FC300008C09F5F90930338911103C08F5F80933A
:10FC400002388091FA379091FB379093251C80936E
:10FC5000241C2091FC373091FD373093FB372093E3
:10FC6000FA379093FD378093FC378091F23790916B
:10FC7000F337A091F437B091F5378093F63790932E
:10FC8000F737A093F837B093F93780916D39909199
:10FC90006E39A0916F39B09170398093F23790939B
:10FCA000F337A093F437B093F5379CC3973089F0BE
:10FCB0008F5F8430C1F060E2869F90011124F901CA
:10FCC000E352F74C918D9111F1CF8093271CEF01F6
:10FCD0000CC0209721F0428D9A8D941748F7E901C6
:10FCE000C352D74CE5CF8093271C209709F4B8C3A3
:10FCF000D093DC38C093DB3883E08A8F888F1E8AEC
:10FD000084E08F8B1B8E8091FC379091FD379D8313
:10FD10008C838091FA379091FB379F838E838091FB
:10FD2000F2379091F337A091F437B091F53788838B
:10FD30009983AA83BB8381E0898F80912A1C8C8759
:10FD400080912B1C8D8780912C1C8E8780912D1C7F
:10FD50008F8781E090E0998B888B809101388B8729
:10FD6000809100388A878091FF3789878091FE379C
:10FD7000888781E090E00E94BA7A80910638982FB7
:10FD8000907F913508F441C082958F7090E005977F
:10FD9000880F991F880F991F2091261CEF2DF0E0E6
:10FDA000E817F90774F5EA51F84C20A5211103C0B2
:10FDB0001092261C28C0213011F4F394EFCF22308A
:10FDC000D9F431A53430C1F42093261CF092271CBD
:10FDD00082A590E0982F882723A5822B9093251C3D
:10FDE0008093241C893C910510F088EC90E09B8B5B
:10FDF0008A8B9D8B8C8B09C031A5332311F0F30EB8
:10FE0000CDCF2093261CF092271C80E180930738E9
:10FE10008091073882608093073882E080930E38A3
:10FE200084E080930F381092103888EC809311385A
:10FE30008CE290E09093DF378093DE3780E680C2DB
:10FE4000D093DC38C093DB381092D63880910738D5
:10FE5000782F7470F72E82FF03C0198E80E219C2CA
:10FE60009091063892959F70990F990F9093271C47
:10FE7000091B1109045111091093DF370093DE3774
:10FE8000922F9F70923029F4982F9F73923139F4FA
:10FE90001FC0913021F4982F9F739230C9F0012B2D
:10FEA00019F4982F9370A1F02091FE3798852913AB
:10FEB0003DC22091FF379985291338C2209100381F
:10FEC0009A85291333C2209101389B8529132EC2AC
:10FED00084FF49C0688979896115710509F443C0B7
:10FEE000CE010C960E94847A309102388091E237DC
:10FEF000381339C0209103388091E337281333C079
:10FF0000909104388091E43798132DC08091053882
:10FF10004091E537841327C03C872D879E878F87C4
:10FF20008B8D811119C09E89888D2A8D821B292F66
:10FF3000269526952695821B980F9E8B87FD819589
:10FF40002F89322F36953695231B820F8F8B9695EE
:10FF500096959695890F888F81E08093D638888D05
:10FF60008A8F198A188A298DE22FEF708E2F90E0E0
:10FF7000FC013197E830F10508F072C28827E65697
:10FF8000FF4F8F4F0C94DE888091D63880FF14C0CD
:10FF900083E0898F80E48093D638198A188A80910B
:10FFA000DE379091DF37009709F405C122E42093F2
:10FFB000D6380E94BA7AFFC0809107388F7382309A
:10FFC00009F04EC222CF8091D63880FF6AC080915E
:10FFD00007388F73823109F064C080910638982FFA
:10FFE000907F913508F441C082958F7090E005971D
:10FFF000880F991F880F991F2091261CEF2DF0E084
:020000021000EC
:10000000E817F90774F5EA51F84C20A5211103C04F
:100010001092261C28C0213011F4F394EFCF223027
:10002000D9F431A53430C1F42093261CF092271C5A
:1000300082A590E0982F882723A5822B9093251CDA
:100040008093241C893C910510F088EC90E09B8BF8
:100050008A8B9D8B8C8B09C031A5332311F0F30E55
:10006000CDCF2093261CF092271C83E0898F8091AE
:10007000FE3788878091FF378987809100388A878B
:10008000809101388B8781E090E00E94BA7A82E407
:100090008093D638198A188A1092DF371092DE378B
:1000A0008AC080E28093D6380E947277E091DB3874
:1000B000F091DC38118E83CD8091073880FF28C005
:1000C00024FD26C088899989892B09F0C9C18091AE
:1000D000DE379091DF3701960E94BA7A8091D63848
:1000E000982F90619093D6382091DE373091DF378A
:1000F000232B19F082618093D6380E94727781E0B9
:1001000090E0998B888B88E0898F1B8E81E10FC1ED
:1001100085FF1DC080910C3890E0982F8827309182
:100120000D38832B4091D9385091DA38480F591F38
:100130005093DA384093D9384091DE375091DF3709
:10014000BA01681B790B7093DF376093DE374091FB
:10015000DE375091DF374115510551F024FD08C0BD
:100160009091D63892609093D638CA010E94BA7A9C
:100170008091083890E0982F882720910938820FC5
:10018000911D9093251C8093241C2C893D89281750
:10019000390710F0892B21F43093251C2093241C5F
:1001A0008091241C9091251C9B8B8A8B8091D63842
:1001B000837009F455C110927239109271390E94FE
:1001C00072778091D63885FF07C0109272391092ED
:1001D0007139198E84E1ABC084FF0AC01092723964
:1001E0001092713981E090E0998B888B84E08CCFFC
:1001F000209171393091723921153105E1F080FF7C
:1002000002C0198A188A88899989009781F48A8995
:100210009B898217930720F49093723980937139E8
:100220008091713990917239998B888B04C0909329
:100230007239809371391B8E8091E0379091E1374C
:100240009093DA388093D9388091713990917239CE
:10025000892B59F088899989009739F0889690936D
:10026000DF378093DE3788E10BC08091D63881FF7D
:10027000F7C088E290E09093DF378093DE3780E12B
:10028000809307385CC08091D63880FFE9C0198E12
:1002900080E18093D6380E947277E2C08091DE3789
:1002A0009091DF37009711F00E94BA7A9091073849
:1002B0008091D63890FF0BC080FF06C087E0898F01
:1002C0001A8E198A188A19C086E0898F16C080FF95
:1002D0001EC085E0898F198A188AC2C08091DE37D6
:1002E0009091DF37009711F00E94BA7A8091073819
:1002F00080FF0DC087E0898F1A8E81E090E00E9418
:10030000BA7A80E18093D6380E9472770FC08091CC
:10031000DE379091DF37892B49F4A2C08091D6381F
:1003200080FF9EC087E0898F1A8E9AC080E18093FB
:10033000073888E290E09093DF378093DE3780E5DE
:1003400080930638888580930238898580930338A6
:100350008A85809304388B85809305388C858093BB
:10036000FE378D858093FF378E85809300388F858B
:100370008093013886E08093EF378C819D81909344
:10038000FB378093FA378E819F819093FD3780935E
:10039000FC3780916D3990916E39A0916F39B09191
:1003A00070398093F2379093F337A093F437B0937A
:1003B000F53788819981AA81BB818093F637909324
:1003C000F737A093F837B093F937898D84FF05C0CC
:1003D000109209381092083805C01092083888EC3D
:1003E0008093093880E48093EE378091DE379091D6
:1003F000DF379093E8378093E93710920D381092E9
:100400000C3810920B3810920A380E94E87A8095C6
:10041000909590930B3880930A3885E48093E63763
:100420001092E7371092ED371092EC3780912E1C26
:1004300090912F1C019690932F1C80932E1C9093CB
:10044000EA378093EB371092F1371092F0370E9421
:10045000D77A809590959093F1378093F03704C0C8
:100460001092DF371092DE371092D638DF91CF919D
:100470001F910F91FF90EF90DF90CF90BF90AF90C2
:10048000089582E39CE10C945A719093311C8093FF
:10049000301C089582E39CE10C945E71EF92FF9210
:1004A0000F931F93CF93DF938C01EB017A0182E3CB
:1004B0009CE10E945E710097D9F0DC0112962D91AB
:1004C0003C9113972C173D0781F41696ED91FC9102
:1004D0001797309769F09701AE01B801DF91CF917E
:1004E0001F910F91FF90EF9019940E94C371E3CF79
:1004F000DF91CF911F910F91FF90EF900895089594
:100500000F931F93CF93DF93C3E7DCE148815981B9
:100510006A817B8100E010E02AEA32E883E59CE111
:100520000E94936D0E94F666BC0180E090E02881F5
:1005300039814A815B810E949D88AB01BC012FEC0F
:1005400032E88FE39CE10E94936DDF91CF911F9180
:100550000F9108958091731C9091741CA091751C4B
:10056000B091761C40916F1C5091701C6091711C71
:100570007091721C880F991FAA1FBB1F481759073B
:100580006A077B0710F4DB01CA018093731C909308
:10059000741CA093751CB093761C0C948082CF932E
:1005A000DF930E947F750E94EE74EC01198218821D
:1005B0000E944A8228813981009719F1FC01408507
:1005C0004423F9F0FC0142815381F901EE0FFF1F32
:1005D000EE0FFF1FEC0FFD1F53834283FC0144818C
:1005E00055812F5F3F4FF901EE0FFF1FEE0FFF1FE9
:1005F000EC0FFD1F51834083398328830E94C37110
:10060000D9CFC901880F991F880F991F02960E94A0
:10061000E97488819981892B31F084E39CE1DF9131
:10062000CF910C94A573DF91CF910895AF92BF92B3
:10063000CF92DF92EF92FF920F931F93CF93DF93AE
:100640001F921F92CDB7DEB75B010E94EE748C0142
:10065000FC01E080F180FA82E9820E943675970100
:10066000220F331F220F331F2E5F3F4F8217930736
:1006700098F0C12CD12CCE14DF0471F0F801448124
:10068000558162817381C5010E944E82FFEFCF1AAE
:10069000DF0A0C5F1F4FEFCF0F900F90DF91CF91CC
:1006A0001F910F91FF90EF90DF90CF90BF90AF9090
:1006B00008950F93013099F48091671C9091681C04
:1006C000A091691CB0916A1C8093731C9093741C58
:1006D000A093751CB093761C0F910C9480820F919F
:1006E00008954F925F926F927F928F929F92AF92F6
:1006F000BF92CF92DF92EF92FF920F931F932A0146
:100700003B014801590142E35AE0BC0184E39CE10A
:100710000E948873E4E3FCE143AA54AA65AA76AA7E
:1007200087AA90AEA1AEB2AEC3AED4AEE5AEF6AE81
:1007300089E593E81F910F91FF90EF90DF90CF90A4
:10074000BF90AF909F908F907F906F905F904F90F1
:100750000C9445820C94B273CF93DF93E091360AE8
:10076000F091370A1995EC01892B29F06A817B8178
:1007700081E00E94D375CE01DF91CF9108950F9350
:100780001F93CF93DF93EC01E091380AF091390A7F
:1007900019958C016A817B8181E00E94D37581E08B
:1007A00090E0012B11F480E090E0DF91CF911F9158
:1007B0000F910895E0913A0AF0913B0A1994CF9372
:1007C000DF93FC01DB0185E0EB0119928A95E9F7E3
:1007D0008581837011F082E08C938781837021F092
:1007E00082E012968C9312978581837081F08781C5
:1007F000837069F0238934898185928528173907A8
:1008000031F481E0848312961C92129701C0148205
:1008100085818370823029F0833011F488E001C033
:1008200080E011968C93119787818370823029F034
:10083000833011F488E001C080E013968C93DF913F
:10084000CF910895CF93DF9300D01F921F92CDB721
:10085000DEB7BE016F5F7F4F0E94DF83898190E02A
:1008600003962A81820F911D2B81820F911D2C816D
:10087000820F911D2D81820F911D0F900F900F906F
:100880000F900F90DF91CF9108953F924F925F921A
:100890006F927F928F929F92AF92BF92CF92DF9290
:1008A000EF92FF920F931F93CF93DF9300D01F928D
:1008B0001F92CDB7DEB78C017B013A01BE016F5F9D
:1008C0007F4F0E94DF8369817A81472F50E0EB815F
:1008D0003C80232D30E0862F90E00396840F951FF7
:1008E0008E0F911D820F931FAD818A0F911D681687
:1008F00079060CF4A4C0D80111968C91119780FB55
:10090000882480F8912C83E0880C991C8A95E1F763
:1009100012968C91129780FBAA24A0F8B12C94E037
:10092000AA0CBB1C9A95E1F78A288C918770882ABB
:1009300013968C91139780FBCC24C0F8D12CF5E052
:10094000CC0CDD1CFA95E1F7C82814968C9180FB3D
:10095000442440F8512CA6E0440C551CAA95E1F71C
:100960004C28D7014C92D80115968C918370B4E035
:100970008B9F60011124D80116969C919370B0E171
:100980009B9FC00111248C29D8011796FC9190E4FB
:10099000F99FD00111248A2BD70111968C93D8018D
:1009A00018968C91D70112968C93623071F4D8010D
:1009B00019968C91D70113968C93D8011A968C9125
:1009C000D70114968C9385E001C083E0780F872FC0
:1009D000972F941B4115510561F041505109D801E1
:1009E000A40FB51F1B968C91D701A90FB11D8C9335
:1009F000EECFE23071F4D701A70FB11DF801938952
:100A00009C9391E0970FD701A90FB11D8E5F948938
:100A10009C93F32DF80F8F2F821B2115310561F068
:100A200021503109D801A20FB31F55969C91D701CF
:100A3000A80FB11D9C93EFCF8F2F90E002C080E0F4
:100A400090E00F900F900F900F900F90DF91CF914B
:100A50001F910F91FF90EF90DF90CF90BF90AF90DC
:100A60009F908F907F906F905F904F903F900895F0
:100A7000AF92BF92CF92DF92EF92FF920F931F93AC
:100A8000CF93DF93633071050CF4B3C0EA016B01BF
:100A90007C01FC01908196FBAA24A0F88181282F7B
:100AA000269526952370B82EB294B694B69453E04A
:100AB000B522392F3770388393FB332730F93983C8
:100AC00094FB332730F93A8395FB992790F99B8360
:100AD000AC822D83829583708E83BF8282818887CA
:100AE000222379F13381848190E0982F8827830F26
:100AF000911D9A87898787010B5F1F4F223071F400
:100B000060E07AE0CE010B960E94A074F701868126
:100B10008B8785818C870E5F1F4F1EC02330E1F4C9
:100B2000F7013D96DE011B969E012D5E3F4F9E2FE5
:100B30008F2F42914D93A217B307D9F7092F182F82
:100B40000BC087010D5F1F4F60E07AE0CE010B966E
:100B50000E94A0741A861986BB20A1F1A1100DC0B5
:100B6000F8012081818190E0982F8827820F911DC4
:100B70009C8B8B8B0E5F1F4F04C089859A859C8B45
:100B80008B8BF2E0BF120EC060E07AE0CE0145969A
:100B90000E94A074F80181818D8B80818E8B0E5F05
:100BA0001F4F18C0F3E0BF1215C0085F1F4FD801D8
:100BB000FE017596CE014D962E912193E817F90707
:100BC000D9F708C060E07AE0CE0145960E94A07493
:100BD0001C8A1B8A98012E193F09C601821B930BA0
:100BE00098AB8FA71EA70DA7C216D30614F0C90194
:100BF00002C080E090E0DF91CF911F910F91FF90B4
:100C0000EF90DF90CF90BF90AF90089520E030E05C
:100C10000296FC0132974081442331F0FC01319768
:100C20004081240F311DF4CFC9010895FC012081BA
:100C300030E0322F22278181282B02C0220F331F60
:100C40006A95E2F7232F3327FA01E45CF54F8081A0
:100C500090E08223932328E030E0241B350B02C070
:100C6000969587952A95E2F708956F927F928F92D5
:100C70009F92AF92BF92CF92DF92EF92FF920F932B
:100C80001F93CF93DF937C018B015A01E901283038
:100C9000310544F4A901B501C8010E941686F70187
:100CA000808346C0690183E0D594C7948A95E1F7B3
:100CB000452B21F04701612C712C06C0FB01D701A7
:100CC000CB018C0D9D1D1FC048E050E0B501C8014F
:100CD000860D971D0E941686F40181934F01FFEF48
:100CE0006F1A7F0A6C147D0479F7AE01477055279F
:100CF00041155105E9F0E701C60DD71DB501C80141
:100D0000860D971D12C0E817F90719F021912D9350
:100D1000FACFAE01477055274115510549F0E7015B
:100D2000CC0DDD1D60E070E0CF010E941686888347
:100D3000DF91CF911F910F91FF90EF90DF90CF90B7
:100D4000BF90AF909F908F907F906F9008958F92FB
:100D50009F92AF92BF92CF92DF92EF92FF920F934A
:100D60001F93CF93DF931F921F92CDB7DEB70E94E0
:100D7000EE748C0182E090E00E94CC74892B19F40F
:100D800080E090E05FC0F801218130E0322F22271F
:100D90008081A901480F511DCA010E94C3737C01C3
:100DA000892B71F30E94EE744C01F7019681292F73
:100DB00026952695269530E0977041E050E011F495
:100DC00040E050E0C901840F951F0E94CC74892B2C
:100DD000B9F2F70104811581A12CB12CF8018081B1
:100DE000882379F1F801C180D12CA50147705527DE
:100DF000B50193E0759567959A95E1F7680D791DB2
:100E0000883168F09601CE0101960E943586BE01B8
:100E10006F5F7F4FF80180810E94E7750DC01A82D5
:100E200019829601CE0101960E94358669817A81E8
:100E3000F80180810E94D375AC0CBD1C0E5F1F4F62
:100E4000CDCFC7010F900F90DF91CF911F910F91E0
:100E5000FF90EF90DF90CF90BF90AF909F908F90DA
:100E60000895DC0150E0E0E1F0E0CF01861B970B34
:100E7000821B930B02C0440F551F8A95E2F78C9199
:100E8000852B8C9311968C911197482B11964C932E
:100E900008956F927F928F929F92AF92BF92CF925E
:100EA000DF92EF92FF920F931F93CF93DF9328303F
:100EB00031051CF4FA0140815AC05901E3E0B594B0
:100EC000A794EA95E1F76115710541F03901EA014E
:100ED0008B017C014A01C12CD12C05C0EA01FC0127
:100EE0004A0D5B1D2AC0F40141914F0128E030E01A
:100EF000B801C7018C0D9D1D0E943187FFEFCF1AED
:100F0000DF0ACA14DB0479F7930127703327211510
:100F10003105E9F1CC0DDD1D488150E0021B130BBA
:100F2000085F1F4F02C0559547950A95E2F760E0AC
:100F300070E0C7018C0D9D1D1AC0C417D50719F0AC
:100F400069916193FACF2770332721153105F9F0A4
:100F5000488150E068E070E0621B730B02C0559559
:100F600047956A95E2F760E070E08A0D9B1DDF917E
:100F7000CF911F910F91FF90EF90DF90CF90BF9096
:100F8000AF909F908F907F906F900C943187DF91FE
:100F9000CF911F910F91FF90EF90DF90CF90BF9076
:100FA000AF909F908F907F906F9008956F927F92F7
:100FB0008F929F92AF92BF92CF92DF92EF92FF9269
:100FC0000F931F93CF93DF931F921F92CDB7DEB77E
:100FD0007C01FC018681082F069506950695202F39
:100FE00030E0877001E010E011F400E010E0020F43
:100FF000131FC80102960E944875009709F448C063
:101000000E94F574F7012281FC012083F7012381FE
:10101000FC0121830E94F57402965C01A80160E046
:1010200070E00E942893F701048115810F5F1F4F24
:10103000812C912CF80131978081882339F1F801B6
:10104000C080D12C3401F7E06F227724740193E043
:10105000F594E7949A95E1F7EA0CFB1C883128F0A7
:101060000E94F1759601AC0108C00E94DE759A835A
:1010700089839601AE014F5F5F4FB301C7010E94A4
:1010800049878C0C9D1C0E5F1F4FD4CF81E090E0F0
:101090000F900F90DF91CF911F910F91FF90EF90E4
:1010A000DF90CF90BF90AF909F908F907F906F9088
:1010B0000895DB018F939F930E940489BF91AF91A4
:1010C000A29F800D911DA39F900DB29F900D1124A2
:1010D0000895991B79E004C0991F961708F0961B94
:1010E000881F7A95C9F780950895AA1BBB1B51E10B
:1010F00007C0AA1FBB1FA617B70710F0A61BB70B88
:10110000881F991F5A95A9F780959095BC01CD012C
:10111000089597FB072E16F4009407D077FD09D0A9
:101120000E94758807FC05D03EF4909581959F4FED
:101130000895709561957F4F0895A1E21A2EAA1B1C
:10114000BB1BFD010DC0AA1FBB1FEE1FFF1FA21777
:10115000B307E407F50720F0A21BB30BE40BF50B74
:10116000661F771F881F991F1A9469F760957095FD
:10117000809590959B01AC01BD01CF010895052E8E
:1011800097FB1EF400940E94D68857FD07D00E945A
:101190009D8807FC03D04EF40C94D688509540955A
:1011A000309521953F4F4F4F5F4F08959095809513
:1011B000709561957F4F8F4F9F4F0895EE0FFF1FE2
:1011C000881F8BBF0790F691E02D19940E94EE883E
:1011D000332312F48A1B9B0B0C94FF88A29FB0014F
:1011E000B39FC001A39F700D811D1124911DB29F5B
:1011F000700D811D1124911D08950E94EE88B7FF86
:101200000895821B930B08950E94EE88A59F900D70
:10121000B49F900DA49F800D911D11240895B7FFD8
:101220000C9404890E940489821B930B0895DF9318
:10123000CF931F930F939A9DF02D219FF00D8B9DBF
:10124000F00D8A9DE02DF10D039FF00D029FE00D42
:10125000F11D4E9DE00DF11D5E9DF00D4F9DF00DB9
:101260007F936F93BF92AF925F934F93D5010E948C
:10127000EE888B01AC01D7010E94EE88EB01E80FEC
:10128000F91FD6010E9467892F913F91D6010E94D4
:10129000EE88C60FD71FE81FF91FAF91BF910E94BC
:1012A00067892F913F910E94EE88C60FD71FE81FD4
:1012B000F91FD6010E94EE88E60FF71F9801BE01C4
:1012C000CF0111240F911F91CF91DF9108950E94BA
:1012D000EE88460F571FC81FD91F08F4319608958E
:1012E000E894DF93CF93FC01DB010E94EE887F93AB
:1012F0006F93E9019A01AC01BF93AF933F932F9392
:10130000DF010E94EE8826F46C1B7D0B820B930B91
:101310009E01EB01FC010E946789AF91BF912F9163
:101320003F910E946789BE01CF01F9012F913F9142
:10133000CF91DF910895689401C0E894F92FF12BC3
:1013400012F00C94CF89A0E0B0E0E9EAF9E80C943F
:10135000418A092E059422F40E942B8A112392F4CB
:10136000F0E80F26FFEFE094F09400951095B0940C
:10137000C094D094A194BF0ACF0ADF0AEF0AFF0AF3
:101380000F0B1F0B0E94DA8907FC0E942B8ACDB736
:10139000DEB7ECE00C945D8A689401C0E8948F920B
:1013A0009F92CF93DF930E94DA89DF91CF919F9034
:1013B0008F90089588249924F401E401B0E49F9368
:1013C000AA279A158B049C04ED05FE05CF05D007CE
:1013D000A10798F4AD2FDC2FCF2FFE2FE92D982CED
:1013E000892E982F872F762F652F542F432F322F3A
:1013F0002227B85031F7BF9127C01B2EBF91BB27C2
:10140000220F331F441F551F661F771F881F991F08
:10141000881C991CEE1FFF1FCC1FDD1FAA1FBB1FBE
:101420008A149B04EC05FD05CE05DF05A007B10776
:1014300048F08A189B08EC09FD09CE09DF09A00BCA
:10144000B10B21601A94E1F62EF49401AF01BE01B4
:10145000CD01000C0895609570958095909530951C
:101460004095509521953F4F4F4F5F4F6F4F7F4FA6
:101470008F4F9F4F08952F923F924F925F926F929E
:101480007F928F929F92AF92BF92CF92DF92EF9214
:10149000FF920F931F93CF93DF93CDB7DEB7CA1B95
:1014A000DB0B0FB6F894DEBF0FBECDBF19942A88B0
:1014B000398848885F846E847D848C849B84AA8468
:1014C000B984C884DF80EE80FD800C811B81AA81F5
:1014D000B981CE0FD11D0FB6F894DEBF0FBECDBFC0
:1014E000ED0108950F93083090F0982F872F762FF5
:1014F000652F542F432F322F22270850F4CF220F6D
:10150000331F441F551F661F771F881F991F0A9599
:10151000B2F70F91089597FB10F8169400080F93F7
:10152000083098F00850232F342F452F562F672F5F
:10153000782F892F902DF4CF0594979587957795DF
:10154000679557954795379527950A95AAF70F916F
:1015500008952A0D3B1D4C1D5D1D6E1D7F1D801FB6
:10156000911F08950024A7FD00942A0F301D401DEF
:10157000501D601D701D801D901D08952A193B0986
:101580004C095D096E097F09800B910B08952A159E
:101590003B054C055D056E057F05800791070895A5
:1015A0000024A7FD00942A1730054005500560056A
:1015B00070058005900508955058BB27AA270E9402
:1015C000F48A0C945F8D0E94518D38F00E94588DE2
:1015D00020F039F49F3F19F426F40C94178D0EF483
:1015E000E095E7FB0C94118DE92F0E94708D58F364
:1015F000BA17620773078407950720F079F4A6F5F8
:101600000C94928D0EF4E0950B2EBA2FA02D0B01A9
:10161000B90190010C01CA01A0011124FF27591B37
:1016200099F0593F50F4503E68F11A16F040A22F3D
:10163000232F342F4427585FF3CF469537952795AE
:10164000A795F0405395C9F77EF41F16BA0B620BAD
:10165000730B840BBAF09150A1F0FF0FBB1F661FF4
:10166000771F881FC2F70EC0BA0F621F731F841F37
:1016700048F4879577956795B795F7959E3F08F05D
:10168000B0CF9395880F08F09927EE0F979587951F
:1016900008950E94518D60F080E891E009F49EEF7A
:1016A0000E94588D28F040E851E071F45EEF0CC0C4
:1016B0000C94178D0C94928DE92FE0780E94708D18
:1016C00040F3092E052AB1F32617370748075907B3
:1016D00038F00E2E07F8E02569F0E025E0640AC036
:1016E000EF6307F8009407FADB01B9019D01DC0103
:1016F000CA01AD01EF930E94D78B0E945F8D0E94BB
:101700008C8B5F91552339F02BED3FE049E450FD80
:1017100049EC0C94DD8A0895DF93DD27B92FBF775C
:1017200040E85FE31616170648075B0718F4D92F41
:101730000E949E8D9F938F937F936F930E94298F1A
:10174000E4E4F1E00E942A8D0E945F8D2F913F9189
:101750004F915F910E947F8EDD2351F09058A2EA55
:101760002AED3FE049EC5FE3D0785D270E94F48AE0
:10177000DF910C945F8D0E94ED8C08F481E0089558
:101780000E94D48B0C945F8D0E94588D58F00E945B
:10179000518D40F029F45F3F29F00C94118D5111C7
:1017A0000C94938D0C94178D0E94708D68F399237F
:1017B000B1F3552391F3951B550BBB27AA2762174D
:1017C0007307840738F09F5F5F4F220F331F441F5A
:1017D000AA1FA9F335D00E2E3AF0E0E832D091508E
:1017E0005040E695001CCAF72BD0FE2F29D0660F7B
:1017F000771F881FBB1F261737074807AB07B0E8BE
:1018000009F0BB0B802DBF01FF2793585F4F3AF0C3
:101810009E3F510578F00C94118D0C94938D5F3F91
:10182000E4F3983ED4F3869577956795B795F79549
:101830009F5FC9F7880F911D9695879597F9089531
:10184000E1E0660F771F881FBB1F621773078407CD
:10185000BA0720F0621B730B840BBA0BEE1F88F7DC
:10186000E095089529F416F00C94118D0C94928D46
:101870000C94178D0E94788DA8F39638A0F707F87E
:101880000F92E8942BE33AEA48EB5FE70E94828EDE
:101890000F920F920F924DB75EB70F920E94388E43
:1018A000E1E7F1E00E942A8D4F915F91EF91FF9166
:1018B000E595EE1FFF1F49F0FE57E0684427EE0F45
:1018C000441FFA95E1F74195550B0E94AA8D0F90A0
:1018D00007FE0C949E8D089597FB16F40E941A8DB6
:1018E0000C94B08CE89409C097FB3EF490958095D9
:1018F000709561957F4F8F4F9F4F9923A9F0F92FD6
:1019000096E9BB279395F695879577956795B79553
:10191000F111F8CFFAF4BB0F11F460FF1BC06F5F39
:101920007F4F8F4F9F4F16C0882311F096E911C04B
:10193000772321F09EE8872F762F05C0662371F06C
:1019400096E8862F70E060E02AF09A95660F771F80
:10195000881FDAF7880F9695879597F90895E89488
:10196000F92F96EBFF2381F0121613061406440B91
:101970009395F69587957795679557954040FF2302
:10198000B9F71BC099270895882351F49850D2F7CE
:10199000872B762F652F542F432F322F20E0B1F362
:1019A000121613061406440B88233AF09A95440F36
:1019B000551F661F771F881FCAF755234AF4440F27
:1019C000551F11F460FF04C06F5F7F4F8F4F9F4F13
:1019D000880F9695879597F90895990F0008550FE8
:1019E000AA0BE0E8FEEF16161706E807F907C0F0A5
:1019F00012161306E407F50798F0621B730B840BAD
:101A0000950B39F40A2661F0232B242B252B21F486
:101A100008950A2609F4A140A6958FEF811D811D26
:101A2000089597F99F6780E870E060E008959FEF60
:101A300080EC0895909580957095609550954095AF
:101A4000309521953F4F4F4F5F4F6F4F7F4F8F4FD7
:101A50009F4F0895DF93CF931F930F93FF92EF92C1
:101A6000DF927B018C01689406C0DA2EEF010E94A0
:101A70007F8EFE01E894A591259135914591559170
:101A8000A6F3EF010E94F48AFE019701A801DA94FF
:101A900069F7DF90EF90FF900F911F91CF91DF9149
:101AA000089500240A9416161706180609060895C4
:101AB00000240A9412161306140605060895092E2A
:101AC0000394000C11F4882352F0BB0F40F4BF2B99
:101AD00011F460FF04C06F5F7F4F8F4F9F4F0895D9
:101AE00057FD9058440F551F59F05F3F71F04795CF
:101AF000880F97FB991F61F09F3F79F087950895B4
:101B0000121613061406551FF2CF4695F1DF08C0D2
:101B1000161617061806991FF1CF869571056105EF
:101B200008940895E894BB2766277727CB0197F997
:101B300008950E94ED8C08F48FEF08959B01AC018D
:101B400060E070E080E89FE30C94C08B0C94118DF2
:101B50000C942D8F0E94788DD8F39923C9F3940F9C
:101B6000511DA3F39150504094F059F0882332F066
:101B7000660F771F881F91505040C1F79E3F510557
:101B80002CF7880F911D9695879597F908955F3FDB
:101B9000ACF0983E9CF0BB27869577956795B795F6
:101BA00008F4B1609395C1F7BB0F58F711F460FFCB
:101BB000E8CF6F5F7F4F8F4F9F4FE3CF0C94938D94
:101BC0000E94F08D29ED3BE54EED5EE30C946C8EAA
:101BD00016F00C942D8F0C94178D68940C94118D25
:101BE0000E94788DA8F39923C1F3AEF3DF93CF93CE
:101BF0001F930F93FF92C92FDD2788232AF0219787
:101C0000660F771F881FDAF720E030E040E85FEBCF
